:020000040000FA
:107800005469616E59696E673130300000000000C4
:1078100054593230302E303830303030625F747925
:10782000424154333247313339474B3634464200B4
:1078300043414E5F5354440000000000000000002C
:1078400043414E5F43485F300000000000000000ED
:1078500043414E5F3530304B6270730000000000D2
:10786000E8070000E0070000DF070000000000005C
:020000040000FA
:1080000028330020DD800000E5800000E7800000CC
:108010000000000000000000000000000000000060
:10802000000000000000000000000000EF800000E1
:108030000000000000000000F380000075C2010095
:10804000F91201003D1301006D1301009D130100A1
:10805000CD130100FD1301002D1401005D1401007A
:108060008D140100BD140100F1140100051501007B
:108070001515010049150100591501006915010088
:108080009D150100E115010029160100711601007E
:10809000B916010001170100111701004517010071
:1080A00079170100A9170100DD170100111801005F
:1080B000211801003118010065180100991801000C
:1080C000EF3FE8FF0448854600F02CFA00480047DF
:1080D0007D060200C046C04628330020164880476F
:1080E00016480047FEE7FEE7FEE7FEE7FEE7FEE78D
:1080F000FEE7FEE7FEE7FEE7FEE7FEE7FEE7FEE758
:10810000FEE7FEE7FEE7FEE7FEE7FEE7FEE7FEE747
:10811000FEE7FEE7FEE7FEE7FEE7FEE7FEE7FEE737
:10812000FEE7FEE7FEE7FEE7FEE7FEE7FEE7FEE727
:10813000FEE7FEE7FEE7000075C80100C58000000D
:1081400030B50B46014600202022012409E00D46EF
:10815000D5409D4205D31D469540491B2546954077
:1081600040191546521E002DF1DC30BD70B50024BB
:108170002546002801DA01244042002901DA0125C0
:108180004942FFF7DDFFAC4200D04042002C00D056
:10819000494270BDF0B51FB40646002082B00546C6
:1081A0004024019100901BE0019922460F46304681
:1081B00000F066F9049A059B801A994110D3104685
:1081C0001946224600F04CF9361A8F410197224693
:1081D00001200021009F00F043F938184D41009024
:1081E0002046641E0028DFDC019B009829463246A9
:1081F00007B0F0BDF0B51FB486B00020009001902C
:1082000002900698069980B204900798090C02041F
:108210000014114307900027089D099806913E46D7
:108220003C4603900398A9B20204000C0390049802
:108230002D0C154348430021224600F011F9C719BF
:10824000714110340E46402CECDB3846029A00F0A7
:1082500007F9009A019B80180090594102980191FA
:10826000103002904028CCDB00980BB0F0BD0346E4
:108270000B439B0703D009E008C9121F08C0042A5A
:10828000FAD203E00B780370401C491C521EF9D24D
:108290007047D2B201E00270401C491EFBD2704709
:1082A0000022F6E710B513460A4604461946FFF7C2
:1082B000F0FF204610BD30B504460020034600E024
:1082C0005B1C934203D2E05CCD5C401BF8D030BD18
:1082D0000321001D401E037812021A43491EF9D5DE
:1082E00010467047034603220870000A491C521EBC
:1082F000FAD518467047024670B54A40D30FDB07DF
:1083000040002DD04A002AD0010E140E00021202A5
:108310000919400A520A8418E50104465443000A28
:10832000120A2E045043A4194219200CC543AA185E
:10833000120C0125AD03521C521912047F3924047A
:1083400000D0521C104301D44000491EC2B20C069A
:10835000C0092018401C4008802A02D003E00020F9
:1083600070BD40084000002900DA0020184370BDAD
:1083700070B502464A40D50F40004A00ED0740085C
:108380005208002814D0002A12D0C40DD30D410287
:108390000120C0055202490A520AE41A09181218AB
:1083A0007D34914201D3641C00E04900002C01DAC5
:1083B000002070BD0023914201D3891A0343400875
:1083C00049000028F7D100290AD0914202D10121A9
:1083D000C90705E0914201D2012101E00121C94311
:1083E000E005C018401900F05CF870BD10B500221F
:1083F0009623114600F05DF810BDC20FD207400071
:1084000040080BD0C10D0723DB01C9184002090544
:10841000400A1143C208400711437047002001463B
:108420007047000010B5002904DB0124E407404236
:108430008C412146002B04DB1C460123DB07524202
:10844000A341994200D1904210BD00000122D20701
:10845000002800DB101A002900DB511A88427047FF
:1084600010B5202A04DB0146203A9140002010BDBF
:10847000914020239C1A0346E3401943904010BDCD
:1084800010B5202A04DB0846203AD040002110BD58
:108490000B46D340D0402024A21A914008431946ED
:1084A00010BD002904DA401C490001D140084000F9
:1084B000704770B40024050C05D11024000402D1CB
:1084C000002921D01124050E01D100020834050F26
:1084D00001D10001241D850F01D18000A41C0028BA
:1084E00001DB4000641C002908D020252E1B0D460E
:1084F000F540A14000D001212943084301061B1B80
:10850000000ADB1D02D5002070BC7047DB0518187F
:1085100080180029F8DA401C4900F5D170BC4008E9
:1085200040007047064C0125064E05E0E36807CC85
:108530002B430C3C98471034B442F7D3FFF7C6FDE9
:10854000B41A0200D41A020070B58C180578401CC9
:108550006B075B0F01D10378401C2A1106D102780A
:10856000401C03E006780E70401C491C5B1EF9D1CC
:108570002B0705D40023521E0DD40B70491CFAE7BB
:108580000378401CCB1A921C03E01D780D70491C27
:108590005B1C521EF9D5A142D8D3002070BD70B526
:1085A00007F022F80524204618F022F80025284676
:1085B00007F00EF8204618F01BF80126304606F0AA
:1085C000E3FF204618F014F8284606F0DDFF2046A9
:1085D00018F00EF8304606F0FBFF204618F008F8B9
:1085E00070BDB0B507F000F80524204618F000F87B
:1085F0000125284606F0ECFF204617F0F9FF284633
:1086000006F0C2FF204617F0F3FF002006F0BCFF83
:10861000204617F0EDFFB0BDF0B581B006F0D0FFF9
:10862000052017F0E5FF08270026012006F0ACFF23
:108630000524204617F0DCFF204617F0D9FF06F08E
:10864000B5FF0546204617F0D3FF002006F09CFF3B
:10865000204617F0CDFF76002E437F1E3806E4D16A
:10866000F0B201B0F0BD70B50446002006F08CFFFA
:1086700006F0BAFF052017F0BBFF0826E0B2C009DC
:1086800006F0A6FF0525284617F0B2FF012006F0E8
:108690007BFF284617F0ACFF002006F075FF284648
:1086A00017F0A6FF284617F0A3FF6400761E3006D9
:1086B000E4D1052017F09CFF012070BDF0B583B018
:1086C000019314460E4607460120384302900325C5
:1086D00004E000F08EF86D1E280631D000F067F837
:1086E0003846FFF7C0FF00F0A7F80028F1D1304668
:1086F000FFF7B9FF00F0A0F80028EAD100F057F822
:108700000298FFF7B0FF00F097F80028E1D1019838
:1087100002280BD3451E0026FFF77EFF2070FFF7CF
:108720003EFF641C761CF0B28542F5DCFFF774FF57
:108730002070FFF756FF00F05CF8202003B0F0BD7A
:10874000102003B0F0BDF0B583B01C46009201913B
:108750000290032504E000F04CF86D1E280623D09B
:1087600000F025F80298FFF77EFF00F065F800287A
:10877000F1D10198FFF777FF00F05EF80028EAD109
:10878000002C0CD00026009F3878FFF76CFF00F01B
:1087900053F80028DFD1761C7F1CA642F4D300F0EA
:1087A00028F8082003B0F0BD102003B0F0BDB0B52C
:1087B00006F01AFF0524204617F01AFF0125284667
:1087C00006F0E2FE204617F013FF284606F000FFF1
:1087D000204617F00DFF0025284606F0F9FE20463A
:1087E00017F006FF284606F0CFFE642017F000FFC2
:1087F000B0BDB0B506F0F8FE0524204617F0F8FE2F
:108800000025284606F0C0FE204617F0F1FE284657
:1088100006F0DEFE204617F0EBFE0125284606F0A6
:10882000B3FE204617F0E4FE284606F0D1FE642091
:1088300017F0DEFEB0BD0000B0B506F0C1FE0524A5
:10884000204617F0D5FE012006F09EFE204617F0C8
:10885000CFFE0B4D06F0AAFE044606F08FFE002C5C
:1088600002D06D1E2804F5D10525284617F0C0FE5C
:10887000002006F089FE284617F0BAFE2046B0BD5B
:1088800033210000034801780B2901D8491C0170ED
:108890007047C046172F002070B584B0002503959F
:1088A00002950195009506F069FE0F20C6430E4C17
:1088B0001036F1B2A0206A461023FFF744FF20468D
:1088C00017F096FE204617F093FE912EF0D3A020CD
:1088D000B0216A461023FFF736FF204617F088FEC6
:1088E0000248058004B070BD581B00000A2F00200C
:1088F00070B5022902D2EB24E0B270BD891EEB25CF
:108900000022134605E0401C5B1CDDB2A94225464F
:108910000EDB04786C40154604E034466E1C072DCF
:108920003546F0D26608E407F7D09A246640F4E7AB
:10893000E0B270BDF0B591B00C91417810AA117001
:1089400083781B025918C37804792402E3181B04A6
:1089500059180B0ED3700C0C94700D0A55700B91B6
:1089600008956918099409190A93C9180278D2431D
:108970008918427983791B029A18C379047A2402F0
:10898000E3181B049A188918130A0693C918130CC4
:108990000593C9180792120E04928918827AC37A35
:1089A0001B029A18037B0F90447B2402E3181B04DC
:1089B00098180918020A02928918020C0192891863
:1089C0000D910390000E0E9000200346014606E034
:1089D00032409A40D2B211435B1C082B0ED00126C4
:1089E00035469D400746024602E07F1C042FEFD02B
:1089F00010ACE45D2542F8D0521CF6E70E9C0D98B1
:108A00000019C3B20F98827B934205D0427A9142FB
:108A100002D1002011B0F0BD1021FFF769FF0C99C1
:108A2000CC72019A8A72029A4A72039A0A72049A62
:108A3000CA71059A8A71069A4A71079A0A710A9A46
:108A4000CA70099A8A70089A4A700B9A0A7011B013
:108A5000F0BDF0B58DB055220270002747720B783B
:108A60004370CA79059202728A790492C2714A7976
:108A7000039282710A7902924271CA7A0892427311
:108A80008A7A019202734E7AC6720C7A84720CAAA8
:108A900013704D782D02EB188D78C97809024919A9
:108AA0000904CB18190E01711D0CC57009931B0A1E
:108AB0000B90837038460A91D17007959570069394
:108AC000537031020919089A1202019BD21812043C
:108AD0005118089103990902029A8918059A1202FD
:108AE000049BD2181204511805913D463A4605E000
:108AF0002640AE4032436D1C082D0ED00124214685
:108B0000A9400346064602E05B1C042BF0D00CAFE4
:108B1000FF5C3942F8D0761CF6E70B9B5A72099835
:108B200006994018079940180A994018059A801824
:108B3000110A4018110C4018110E4018089A80189C
:108B4000110A4018110C4018110E4018563898732D
:108B500010211846FFF7CCFE0DB0F0BDF0B58FB078
:108B60000446FF20E070A07060700F20C0430290A8
:108B70000F302070704817F03BFD7049086863287B
:108B800001D8642008606E4F002038806D4E01903F
:108B9000308008E00B99814222D338881030388029
:108BA00080B2A1286DD206F0E9FC3978A02003AA92
:108BB0001023FFF783FD30802028EED103AD0BA9F1
:108BC0002846FFF7B7FEE97B8842E6D1287855288A
:108BD000E3D15D48017800290298DBD10846D9E746
:108BE0003888A0284DD8C0B20021019105E006F0D8
:108BF000C5FC3988C8B2A12943D2C1B2A02003AABA
:108C00001023FFF75BFD3080398810313980202830
:108C100037D103AD07A92846FFF78CFEE97B8842D0
:108C2000E5D128785528E2D14748007800280299F4
:108C300000D1014607988842D9D240490A68962156
:108C400051430B9A824208D90818904219D30BA9B4
:108C50000E222046FFF70BFBC9E78918814210D38B
:108C600007A90E222046FFF702FB0BA80A99818173
:108C700007980B9008980C9009980D9038880190EF
:108C8000B5E72078617809020818A178E278120225
:108C9000511809040818401C24D100200190388084
:108CA000A020B02103AA1023FFF708FD3080202860
:108CB00018D103AD0BA92846FFF73CFEE97B88429B
:108CC00010D1287855280DD11F480078002800D1F0
:108CD00002900B980299884204D20BA90E222046DA
:108CE000FFF7C5FA2078617809020818A178E278C0
:108CF0001202511809040818401C0CD10020E0721F
:108D0000A07260722072E071A07160712071E070D9
:108D1000A070607020700198388020786178090216
:108D20000818A178E27812025118090408180749B6
:108D3000086030880FB0F0BD70110100042F0020D2
:108D40000A2F0020002F0020032F0020102F0020CA
:108D5000F0B581B000910646214800250570002A33
:108D60002ED01446C036631B71190F200840102204
:108D7000101A834200D303461A480278102A01D001
:108D8000042A1AD1C809FE2707405F2F13D80127EC
:108D9000B8436038C0B29E3282420CD3009A521956
:108DA000C9B2DFB23B46FFF789FC0F490880ED19D5
:108DB000A542D8D304E0082000E004200A49088036
:108DC000094801880020042902D0082900D0012088
:108DD00003490870411E8841400001B0F0BDC04603
:108DE000162F0020022F0020142F00200A4A0123F2
:108DF00013700A4A10700A4A11600A4A0021116071
:108E0000042801D105218901102801D11D208101EB
:108E1000054801807047C046032F0020022F002024
:108E2000042F0020102F0020082F0020F0B587B05D
:108E3000994D00262E80994B1B688B4224D1994C6A
:108E40002188202925D1029000920196964C002776
:108E50002760964D964E2878062809D806F08EFB96
:108E60002068401C2060B042F5D38D480421018069
:108E70002F70904C20880107029B31D08848202118
:108E80000180854D019E0BE001204002844908804D
:108E900006E003A8FFF762FE208081488021018060
:108EA0007F4800883F2807DD874988420BDC40283F
:108EB00012D0802810D010E004280DD008280AD045
:108EC000202809D009E001214A02904204D0C902B9
:108ED000884201D001E002262E80288807B0F0BD2C
:108EE000A128019E00D32780009A012A6A4D1ED135
:108EF000187B012856D1DF719F715F711F711F733D
:108F0000587B012804D1DF729F725F721F725F73FA
:108F100003AF38461946FFF79CFDF87320880028F8
:108F200046D01038C1B2A02003AA102344E0002A82
:108F3000B6D1614801780029B2D00270187859780A
:108F4000090208189978DA781202511809040818E9
:108F50005A490978002901D00F21C943884233D2E8
:108F6000274603AC20461946FFF773FDE0733978B6
:108F7000A02010232246FFF7E6FB029A484908800A
:108F800008288DD13888103038801078517809023F
:108F900008189178D2781202511809040818484923
:108FA00008607DE7597B012911D10128A3D0A7E7EB
:108FB000A02003AA10230146FFF7C5FB384908800B
:108FC0003D48009901706BE70120C0025EE73D4813
:108FD0000078012812D103AC20461946FFF739FD6D
:108FE000E073A020B02110232246FFF7ACFB2C49F0
:108FF00008800828E4D133480770E1E718785978E9
:10900000090208189978DA78120251180904081828
:109010002B490968214A12685118884203D2204816
:1090200040210180CCE725490978002901D00F2192
:10903000C94388422DD203AF384619461C46FFF774
:1090400008FDF8731B480178A02010233A46FFF76B
:109050007AFB134908800828B2D1164908881030D5
:1090600008802078617809020818A178E278120255
:109070005118090408181249086008490A6815219E
:109080005143FFF75DF800299AD101200D4908707E
:1090900096E70120C00291E71C2F0020042F00203A
:1090A0001A2F0020002F0020202F0020172F002033
:1090B000818D5B000A2F00200C2F0020032F002041
:1090C000102F0020182F0020FF010000F0B585B000
:1090D0000646434C0027278004921018414A128804
:1090E000904241D201910397404F00200290386096
:1090F0003F4C404D2078052809D806F03FFA3868E3
:10910000401C3860A842F5D33748042101800298FA
:1091100020703948018839480278102A01D0042A81
:1091200032D188190346C033049C651A0F240440C9
:109130001020001B854200DB0546DC09603C01264F
:109140003002E7B27F09052F12D3B443E6B29E3254
:10915000B242234C039F0DD301984218D9B2EBB20F
:109160003046FFF7F0FA05E01F482021018011E0AA
:109170001B4C039F1C49088008280BD1E8B21E4AEB
:1091800011880818108005E0012080021649088027
:10919000134C039F144800881F2809DD202813D092
:1091A00001210A0290420FD0890288420CD00CE0C3
:1091B000042809D0082808D10F480088049988425B
:1091C00001D3022700E001272780208802210143E4
:1091D000022902D1084900220A8005B0F0BDC0462C
:1091E0001C2F0020082F00201A2F0020202F0020E5
:1091F000172F0020818D5B00242F0020022F0020DC
:10920000F0B585B0044600200190042C6FD20BF01D
:10921000CFFF002801D10CF04BF80020009000BFD8
:109220000098401C00900BF0C3FF039003980028A7
:1092300003D0484900988842F2D30398002856D1B9
:10924000042145480BF096FF444845490880210118
:10925000444A515C4900404A505A41490A88012118
:10926000090300F055F902900120049020013D49C6
:1092700040184078002801D100264BE020013949F0
:1092800040184078012802D13548068842E0200184
:1092900034494018407802282AD120014018057925
:1092A0002901304A515C49002B4A505A2C490A88FE
:1092B0000121090300F02CF9064628012A49431828
:1092C0002801284940180289280140180021C76850
:1092D0003046B84706462801224BC018C2882801EC
:1092E000C0188178304600F087F8064612E02DE07D
:1092F00020011C4940184078032804D02001401860
:109300004078132804D1200116494018868801E0CE
:10931000002004900498002818D020011249431816
:109320002001104940180289200140183146C768C1
:109330000298B847019020010A4BC018C28820014A
:10934000C0188178019800F057F80190019805B095
:10935000F0BD000050C300000A0100208813000087
:10936000040100205411020094110200F8B50546D2
:109370000E4614460020009001211C4801751C482F
:10938000007888431A490870084680780821084305
:109390001749887000208871084600780121084329
:1093A0001349087008460572002717E01048007836
:1093B000802108430E49087000BF0E48007D002838
:1093C000FBD000200B4908750948C0892080A41CE7
:1093D0000748C1890098081800907F1CB742E5D360
:1093E00031460098FEF7ACFE80B2F8BD4061004007
:1093F000005004404060004010B50346012908D1E8
:10940000094CA41A9C4202D99C18A0B20BE0064851
:1094100009E0022906D1934202DD9C1AA0B202E0C3
:10942000002000E0184610BDFFFF000010B5044604
:109430000121202002F00AF80020324908700121A1
:1094400031480175002031490875152016F0B8FD26
:109450002C488078E17808432A498870084680784B
:1094600021780843274988702078802806D108464B
:109470000079E17949000843224908712148807840
:10948000E17A08431F498870A078002803D1084674
:10949000007908710FE0A078012806D119480079F9
:1094A000602108431749087105E0164800798021BA
:1094B00008431449087113488079217908431149F8
:1094C000887108468079617908430E498871207A4D
:1094D000C872607A88720846007838218843094942
:1094E0000870084600786178C9000843054908708B
:1094F000A07A0873084600780121084301490870E2
:1095000010BD000000500440406100404060004039
:10951000F8B504460E461746002E01D100250FE08F
:10952000A64201DC3D460BE00094009C20467843B7
:10953000009031460098FEF703FE0090009885B237
:109540002846F8BD0146042904D28A00024BD218ED
:10955000508800E000207047F428002001460429CC
:1095600003D28A00024B985C00E0002070470000A4
:10957000F4280020FFB587B004460898844203DA37
:109580000A988068002802D12448019042E0089897
:10959000001B82B20292002625460A9880680021AC
:1095A0002F463A463346049605910690FEF722FE72
:1095B00005460E46002328463146029AFEF7EAFD8C
:1095C00005460E46304600210A46494050400143B8
:1095D00002D0124801901DE003950A98C068039DCF
:1095E000A84202D30020019014E00A98C1680398B1
:1095F000401A039009990398FEF7A2FD039003987F
:10960000000C0004002802D00448019002E00398F6
:1096100080B2019001980BB0F0BD0000FFFF000088
:1096200010B5084800788021884306490870012158
:1096300005480175002005490875152016F0C0FC85
:1096400010BD0000005004404061004040600040F8
:10965000F8B505460E4614461F4621462846FEF735
:1096600085FD80B2F8BD0000FFB587B006460A98B8
:109670004068002801D1029035E00A9801684068EE
:1096800008180390002534460021274603980695C4
:109690000491059038462946049B059AFEF7AAFDD9
:1096A00004460D460A984068024600230190204671
:1096B0002946FEF76FFD04460D4600232046294645
:1096C000099AFEF767FD04460D46284607492140E2
:1096D000002359405840014303D00448C04302903E
:1096E00001E0A0B2029002980BB0F0BD0000FFFFB5
:1096F00010B5FE4800688079030016F047FC0705A6
:109700009ED8F5F4F3F2F100F848006840790300C0
:1097100016F03CFC0805138A2A8A468A638A12F0EE
:10972000E1FC0020F1490968C873F04800684079FD
:10973000401CEE49096848717DE0ED494969EB4AF2
:109740001268D27A885C12F045FDE84800684079DA
:10975000401CE64909684871E44800684079401CAB
:10976000E2490968487166E00AF010F8002810D153
:1097700012F030FDDD4800684079401CDB49096883
:109780004871DA4800684079401CD8490968487136
:1097900005E012F0D1FC0020D449096848714AE084
:1097A00009F0F4FF002811D1112012F013FDCF4869
:1097B00000684079401CCD4909684871CB48006871
:1097C0004079401CC9490968487105E012F0B4FCB1
:1097D0000020C649096848712DE009F0D7FF00282C
:1097E0001BD1C2480068C07A401CC0490968C872D1
:1097F000BE480068C07ABE49097888420DDB002067
:10980000BA490968C872B94909684862B748006826
:109810008079401CB5490968887112F08DFC0020E0
:10982000B2490968487106E012F086FC0020AF4991
:109830000968487100BF00BF32E3AC480068407C53
:10984000002817D0AA48C068002803D0A848C168DB
:10985000192088470020A54909684862A348006884
:109860008079401CA1490968887100209F490968D6
:1098700048711BE09D480068406A282807D29B4831
:109880000068406A401C9949096848620EE000205F
:10989000964909684862954800688079401C934958
:1098A000096888710020914909684871F8E28F4879
:1098B00000684079030016F069FB080518A42FA47E
:1098C0004CA480A412F00EFC002088490968C873DB
:1098D000864800684079401C84490968487197E0CF
:1098E000D4E2C7E230E25DE194E0814949697F4A10
:1098F0001268D27A885C12F06DFC7C48006840796E
:10990000401C7A4909684871784800684079401CD1
:109910007649096848717BE009F038FF002811D1C9
:10992000012012F057FC714800684079401C6F49D3
:10993000096848716D4800684079401C6B490968A6
:10994000487105E012F0F8FB002068490968487189
:109950005EE009F01BFF002828D164490968C97A34
:1099600024225143634A12688918604A1268D27BE4
:10997000885C12F02FFC5D480068C07B401C5B498E
:109980000968C87359480068C07B242814D3574815
:1099900000684079401C554909684871534800687F
:1099A0004079401C51490968487105E012F0C4FB38
:1099B00000204E49096848712AE009F0E7FE0028B6
:1099C00018D14A480068C07A401C48490968C872E2
:1099D00046480068C07A4649097888420ADB002078
:1099E00042490968C872414800688079401C3F4973
:1099F0000968887112F0A0FB00203C490968487191
:109A000006E012F099FB002038490968487100BF50
:109A100000BF45E2354800684079030016F0B6FA09
:109A20000A0614B92BB948B978B995B912F05AFB9E
:109A300000202E490968C8732C4800684079401CF2
:109A40002A4909684871ABE029494969274A1268DF
:109A5000D27A885C12F0BEFB244800684079401C32
:109A6000224909684871214800684079401C1F4913
:109A70000968487194E009F089FE002811D14A2054
:109A800012F0A8FB194800684079401C1749096882
:109A90004871164800684079401C144909684871AB
:109AA00005E012F049FB002010490968487177E091
:109AB00009F06CFE002824D1FF2012F08BFB0B482C
:109AC0000068C07B401C09490968C87307480068E2
:109AD000C07B24281BD3054800684079401C0349FB
:109AE0000968487101480068407905E0D007002006
:109AF000E82E0020CC070020401CEA490968487184
:109B000005E012F019FB0020E6490968487147E0BA
:109B100009F03CFE002811D1FF2012F05BFBE14868
:109B200000684079401CDF4909684871DD480068D9
:109B30004079401CDB490968487105E012F0FCFAE5
:109B40000020D849096848712AE009F01FFE002862
:109B500018D1D4480068C07A401CD2490968C8723C
:109B6000D0480068C07AD049097888420ADB0020D2
:109B7000CC490968C872CB4800688079401CC94943
:109B80000968887112F0D8FA0020C649096848713E
:109B900006E012F0D1FA0020C2490968487100BFFE
:109BA00000BF7DE1BF4800684079030016F0EEF980
:109BB0000C0715C32CC349C366C382C39FC312F0ED
:109BC00091FA0020B7490968C873B648006840791F
:109BD000401CB44909684871B4E0B3494969B14AC5
:109BE0001268D27A885C12F0F5FAAE4800684079C3
:109BF000401CAC4909684871AA4800684079401C7B
:109C0000A849096848719DE009F0C0FD002811D1FC
:109C1000772012F0DFFAA34800684079401CA14980
:109C2000096848719F4800684079401C9D4909684F
:109C3000487105E012F080FA00209A4909684871DD
:109C400080E009F0A3FD002811D10C2012F0C2FA27
:109C5000944800684079401C9249096848719148CD
:109C600000684079401C8F490968487105E012F08E
:109C700063FA00208B490968487163E009F086FDAA
:109C8000002810D112F0A6FA864800684079401CDE
:109C9000844909684871834800684079401C8149BB
:109CA0000968487105E012F047FA00207D4909680B
:109CB000487147E009F06AFD002811D1132012F025
:109CC00089FA784800684079401C764909684871EB
:109CD000744800684079401C72490968487105E081
:109CE00012F02AFA00206F49096848712AE009F049
:109CF0004DFD002818D16B480068C07A401C6949A6
:109D00000968C87267480068C07A6749097888425C
:109D10000ADB002063490968C872624800688079DC
:109D2000401C60490968887112F006FA00205D49FC
:109D30000968487106E012F0FFF9002059490968E6
:109D4000487100BF00BFABE056480068407903008F
:109D500016F01CF9080513872A874787638712F0D6
:109D6000C1F900204F490968C8734E48006840791E
:109D7000401C4C49096848717AE04B494969494A95
:109D80001268D27A885C12F025FA46480068407959
:109D9000401C444909684871424800684079401CA9
:109DA00040490968487163E009F0F0FC002811D1CE
:109DB000492012F00FFA3B4800684079401C3949AD
:109DC00009684871374800684079401C354909687E
:109DD000487105E012F0B0F9002032490968487175
:109DE00046E009F0D3FC002810D112F0F3F92D4819
:109DF00000684079401C2B4909684871294800686F
:109E00004079401C27490968487105E012F094F92F
:109E100000202449096848712AE009F0B7FC0028AD
:109E200018D120480068C07A401C1E490968C872D1
:109E30001C480068C07A1C49097888420ADB002067
:109E400018490968C872174800688079401C15498C
:109E50000968887112F070F9002012490968487188
:109E600006E012F069F900200E490968487100BF48
:109E700000BF15E000200B4909688871094909688D
:109E80004871062007490968C87009E012F054F9C2
:109E9000002004490968487102490968887100BFB7
:109EA00000BF10BDD0070020E82E002010B56A4882
:109EB00000684079030016F069F8090610C627C645
:109EC00044C6608EC60012F00DF963480068407900
:109ED000401C614909684871BCE0604949695E4AB3
:109EE0001268D27A885C12F075F95B480068407994
:109EF000401C594909684871574800684079401C1E
:109F0000554909684871A5E009F040FC002811D1C5
:109F10007F2012F05FF9504800684079401C4E499C
:109F2000096848714C4800684079401C4A490968F2
:109F3000487105E012F000F90020474909684871AE
:109F400088E009F023FC002810D112F043F94248C0
:109F500000684079401C4049096848713E480068E3
:109F60004079401C3C490968487105E012F0E4F86A
:109F700000203949096848716CE009F007FC0028A5
:109F800022D135480068C07A401C33490968C8723C
:109F900031480068C07A3149097888420FDB0020D7
:109FA0002D490968C8722C4800684079401C2A492C
:109FB00009684871002028490968486208E00020C3
:109FC00025490968487103E0002023490968487160
:109FD00012F0B2F83EE020480068407C002816D01D
:109FE0001E48C068002803D01C48C1681920884753
:109FF00000201949096848621749096848711649DB
:10A0000009688871052014490968C8701AE0124867
:10A010000068406A282807D20F480068406A401C40
:10A020000D49096848620DE000200B490968486243
:10A030000949096848710849096888710520064975
:10A040000968C87006E012F077F800200249096834
:10A05000487100BF00BF10BDD0070020E82E0020CF
:10A0600010B50024F7480068807A01287ED1F548B1
:10A070000068C07900287AD0F2480068807900280A
:10A0800004D0012874D0022873D191E1ED48006812
:10A09000007B24286ED2EB480068C07901287AD171
:10A0A000002475E0E7480068C07A24214843E64967
:10A0B00009684018E3490968097B415CE148006888
:10A0C000C07A24225043E14A12688018DD4A12689F
:10A0D000127B805C814229D0DA480068C07A242152
:10A0E0004843DA4909684018D6490968097B415C48
:10A0F000D4480068C07A24225043D34A126880189A
:10A10000D04A1268127B8154CE480068407B2428D4
:10A1100005D3CC480068007BCA4909684873C94820
:10A120000068007BC7490968887308E0C548006873
:10A13000407B242803D20120C24909688871C148A4
:10A140000068007B401CBF4909680873BD4800686F
:10A15000007B242808D3BB480068407B242803D216
:10A160000120B84909688871B64805E0D3E1CDE11E
:10A1700069E0BAE138E00EE00068007B242804D2F0
:10A18000B04800688079012800D103E0601CC4B2A7
:10A19000242C87D356E0002413E0AA480068C07A34
:10A1A00024214843A94909684018015DA548006871
:10A1B000C07A24225043A44A126880180155601CBA
:10A1C000C4B2242CE9D300209E4909684873232097
:10A1D0009C490968887301209A490968887124207C
:10A1E0009849096808732DE00020964909680873AA
:10A1F00094480068C07A401C92490968C872914826
:10A200000068C07A92490978884217DB8D48006857
:10A21000007C012804D102208A490968887106E07F
:10A22000002088490968887186490968C87100203A
:10A2300084490968C8728349096808740020814903
:10A240000968487161E17F4800684079030015F0B2
:10A250009DFE080513A62AA651A68EA601207949BF
:10A260000968087411F03EFF764800684079401C88
:10A2700074490968487199E075494969714A1268D9
:10A28000D27A885C11F0A6FF6E4800684079401CC5
:10A290006C49096848716B4800684079401C6949FD
:10A2A0000968487182E009F071FA00281BD16549FC
:10A2B0000968497B491CC8B211F08CFF61480068ED
:10A2C000407B60490968C8735E4800684079401C5B
:10A2D0005C49096848715B4800684079401C5949ED
:10A2E0000968487105E011F027FF00205549096809
:10A2F00048715BE009F04AFA00282BD151490968FE
:10A30000C97A24225143504A126889184D4A12686A
:10A31000D27B885C11F05EFF4A480068C07B401C1D
:10A3200048490968C87347480068C07B45490968BF
:10A33000897B88421ADD434800684079401C4149C6
:10A34000096848713F4800684079401C3D490968E8
:10A3500048710BE011F0F0FE3A480068407B394943
:10A360000968C87300203749096848711EE009F080
:10A370000DFA00280CD1334909688871242031492D
:10A380000968C8732F49096848732E49096888739A
:10A3900011F0D2FE00202B490968487106E011F047
:10A3A000CBFE002027490968487100BF00BFACE020
:10A3B000244800684079030015F0E8FD08050F8E79
:10A3C000268E4C8E688E11F08DFE1E4800684079F6
:10A3D000401C1C490968487185E01D494969194AB2
:10A3E0001268D27A885C11F0F5FE16480068407950
:10A3F000401C144909684871124800684079401CA3
:10A400001049096848716EE009F0C0F9002811D1BF
:10A41000492011F0DFFE0B4800684079401C0949D3
:10A4200009684871074800684079401C0549096877
:10A43000487105E011F080FE00200249096848716A
:10A4400051E00000D0070020CC070020C807002002
:10A45000E82E002009F09AF9002810D111F0BAFE78
:10A460009C4800684079401C9A490968487199489D
:10A4700000684079401C97490968487105E011F06F
:10A480005BFE00209349096848712CE009F07EF9D1
:10A4900000281AD18F480068C07A401C8D4909688D
:10A4A000C8728C480068C07A8B49097888420CDBF6
:10A4B000002088490968C8728649096888718549F9
:10A4C0000968487183490968C87111F035FE002098
:10A4D00080490968487106E011F02EFE00207D4990
:10A4E0000968487100BF00BF0FE011F025FE002091
:10A4F0007849096848717749096888717549096818
:10A50000087374490968C87200BFE2E0002071490D
:10A5100009688872DDE06F480068807A0228F4D10B
:10A520006C480068007A002879D06A480068407951
:10A53000030015F02BFD0B0711BB25BB41545EBB7F
:10A540007590BB0011F0CEFD624800684079401C58
:10A55000604909684871B7E05F494969087811F0B6
:10A5600039FE5C4800684079401C5A4909684871C6
:10A57000584800684079401C564909684871A3E072
:10A5800009F004F9002810D111F024FE51480068A8
:10A590004079401C4F49096848714E48006840792D
:10A5A000401C4C490968487105E011F0C5FD0020C8
:10A5B00048490968487187E009F0E8F8002807D1A0
:10A5C000444800684079401C42490968487103E0EA
:10A5D000002040490968487111F0AEFD74E011F0A7
:10A5E00081FD3C4800684079401C3A49096848713F
:10A5F0006AE0394949690978491CC8B211F0EAFD95
:10A60000344800684079401C324909684871314833
:10A6100000684079401C2F490968487154E054E0B3
:10A6200009F0B4F800280FD111F02EFD294909686E
:10A630008870012011F0A2FD264800684079401C76
:10A6400024490968487105E011F076FD0020214990
:10A650000968487138E01F480068807811280CD1DB
:10A6600000201C4909680872AA201A4909688870E4
:10A67000002018490968487011E0164800684078C1
:10A68000401C144909684870124800684078032843
:10A6900005D309F01BF900200E490968487011F034
:10A6A0004BFD00200B49096848710DE011F044FD95
:10A6B0000020084909684871064909684870AA20BD
:10A6C00004490968887000BF03E000200149096857
:10A6D000887210BDD0070020E82E0020F0B5054696
:10A6E0000C4616461F462088482806DA3A46294670
:10A6F000304604F081FF012800D0F0BD2088C00062
:10A700002E502088401C208000BFF6E710B502467E
:10A710009000074BC018405C002802D00320C043C3
:10A7200010BD01209300024C1B1958540020F7E77C
:10A73000682A002070B5002508E06D1C1B48854282
:10A7400002D20AF0E1FD01E0002503E00AF030FD4D
:10A750000028F2D100BF022100200AF037FD0321BA
:10A7600000200AF033FD052100200AF02FFD07210B
:10A7700000200AF02BFD002408E00020A1000C4A74
:10A780005054A10089184880601CC4B2042CF4D332
:10A7900001200849087000204870052088700020BA
:10A7A000C87005480549088070BD000050C300000E
:10A7B000F428002006010020881300000401002076
:10A7C000F8B58D480078030015F0E0FB0604051687
:10A7D0003D5EFDFC0EE10AF06BFD00208649C8706D
:10A7E000487008468078002802D10320087002E0F3
:10A7F000022081490870FDE07F488078002804D05D
:10A800007D488078401E7C4988700AF0D1FC002881
:10A810000BD10AF04DFD00207749C87008468078BA
:10A8200000280FD1032008700CE07348C078401C4A
:10A830007149C8700846C078052803D30520087000
:10A840000AF062FDD6E00AF0B3FC00280ED1042124
:10A850006A480AF08FFC00206749C8704870684851
:10A86000684908800420644908700CE06248C07898
:10A87000401C6149C8700846C078052803D30520EC
:10A8800008700AF041FDB5E05B49497809015E4A6C
:10A89000515C4900594A505A5A490A880121090312
:10A8A000FEF736FE009001255348407800015649D6
:10A8B00040184078002801D100243CE04E48407800
:10A8C0000001514940184078012802D14D480488C0
:10A8D00031E04948407800014B494018407802284F
:10A8E00012D1454949780901474A89180879FEF784
:10A8F00029FE0446404949780901434A89180879E4
:10A90000FEF72CFE054616E03B48407800013E4924
:10A9100040184078032806D0374840780001401896
:10A920004078132806D13448407800013649401851
:10A93000848800E00025002D2FD02F4840780001AA
:10A94000324943182C48407800012F4940180289A9
:10A9500029484078000140182146C7680098B84748
:10A960000646254840780001274BC018C288224877
:10A9700040780001C01881783046FEF73DFD06465C
:10A980001D484078800022494018468001201A491D
:10A99000497889001E4A50540AE000201649497837
:10A9A00089001B4A89184880134949788900505406
:10A9B00011484078401C10494870084640780428E7
:10A9C00009D301E013E007E00AF072FC00200A4915
:10A9D0004870032008700DE00AF0EAFB002803D15C
:10A9E00001200549087001E00AF08EFC02E0FFF743
:10A9F000A1FE00BF00BFF8BD060100200A01002033
:10AA00008813000004010020541102009411020078
:10AA1000F428002010B50AF095FB002405E0002082
:10AA2000A100074A5054601CC4B2042CF7D3002084
:10AA3000044908700520887003480449088010BD47
:10AA4000F4280020060100208813000004010020E3
:10AA500070B50446002000F0AFF8002000F0DAF8EE
:10AA6000002000F09BF8002000F0C4F8002000F067
:10AA700087F8002000F0AEF800BF012000F08EF84B
:10AA8000012000F0B7F8002521E0002000F086F852
:10AA9000002000F0AFF880202040002806D00120E0
:10AAA00000F08AF8012000F0B5F805E0002000F081
:10AAB00083F8002000F0AEF800BF012000F06EF82F
:10AAC000012000F097F86006040E681CC5B2082D3E
:10AAD000DBDB012000F054F8012000F07BF870BDB2
:10AAE00070B504460D46012000F066F8012000F024
:10AAF00091F8002000F052F8002000F07BF80020D0
:10AB000000F03EF8002000F065F800BF012000F0E2
:10AB100045F8012000F06EF8002628E0002000F043
:10AB20003DF8002000F066F880202040002803D087
:10AB3000012000F041F802E0002000F03DF8802004
:10AB40002840002803D0012000F064F802E0002033
:10AB500000F060F800BF012000F020F8012000F0B4
:10AB600049F86006040E6806050E701CC6B2082E71
:10AB7000D4DB012000F004F8012000F02BF870BDB8
:10AB800010B50446002C04D0812103200AF04EFCAD
:10AB900003E0802103200AF049FC10BD10B50446F3
:10ABA000002C04D0812104200AF040FC03E0802125
:10ABB00004200AF03BFC10BD10B50446002C04D064
:10ABC000812102200AF032FC03E0802102200AF0F9
:10ABD0002DFC10BD10B50446002C04D08121044882
:10ABE0000AF024FC03E0802101480AF01FFC10BD9C
:10ABF0000107000010B50446002C05D08121072074
:10AC000000020AF013FC04E08021072000020AF091
:10AC10000DFC10BD10B50446002C04D08121044861
:10AC20000AF004FC03E0802101480AF0FFFB10BD9C
:10AC30000207000010B5F920FFF70AFF8820FFF790
:10AC400007FF9020FFF704FF9820FFF701FF08217E
:10AC50000846FFF745FFE820FFF7FAFE12210846F5
:10AC6000FFF73EFFA020FFF7F3FE70210846FFF735
:10AC700037FFA820FFF7ECFE70210846FFF730FFF2
:10AC8000B020FFF7E5FE70210846FFF729FFB82046
:10AC9000FFF7DEFE00210846FFF722FFC020FFF786
:10ACA000D7FE00210846FFF71BFFC820FFF7D0FEA4
:10ACB00000210846FFF714FFD020FFF7C9FE2F211F
:10ACC0000846FFF70DFFD820FFF7C2FE2F210846E8
:10ACD000FFF706FFE020FFF7BBFE2F210846FFF736
:10ACE000FFFE4020FFF7B4FE00210846FFF7F8FE04
:10ACF0000A20FFF7ADFE002405E000210846FFF71B
:10AD0000EFFE601CC4B25A2CF7DB00240AE00020DE
:10AD10000B4908550B4908550B4908550B4908556F
:10AD2000601CC4B25A2CF2DB8120FFF791FE002098
:10AD3000074908708870C8700871487010BD00001D
:10AD40001C26002076260020D02600202A2700205E
:10AD5000D300002010B58020FFF77AFE10BD000060
:10AD60000020044908700120034908700020487041
:10AD700070470000D8000020D300002010B54848DC
:10AD8000007800287AD046488078030015F0FEF855
:10AD90000604434A535A687E414800794149085C99
:10ADA0003F490979404A515C884209D13C480079C1
:10ADB0003E49085C3A4909793D4A515C88421BD0BA
:10ADC000374800793749085C35490979364A505483
:10ADD000334800793549085C31490979344A50547F
:10ADE0002F48C078002803D004202D49887011E036
:10ADF00001202B4988700DE000202949C8700846C1
:10AE00000079401C0871084600795A2802DB0020AE
:10AE10000871087041E04020FFF71AFE0220204927
:10AE200088703AE01E4A11791079FFF759FE032025
:10AE30001B49887031E00A20FFF70AFE04201849F8
:10AE400088702AE0164A1279194B995C144A1279D3
:10AE5000154B985CFFF744FE0520114988701CE0F3
:10AE60000F480079401C0E490871084600795A289D
:10AE700005DB002008710870C87003E00EE00120B7
:10AE80000749C87000200649887006E00020044980
:10AE900008708870C870087100BF00BF10BD000046
:10AEA000D30000201C26002076260020D02600207B
:10AEB0002A27002010B511F04BFD012837D10720BB
:10AEC00009F01EFA002810D01C480078052805DA81
:10AED0001A480078401C1949087016E005201749E7
:10AEE00008700020164908700FE015480078052802
:10AEF00005DA13480078401C1149087005E0052068
:10AF00000F49087000200D4908700C48007805288A
:10AF100006D1FF22A5320021012013F007FA0BE031
:10AF20004B22D2000021012013F000FA04E000229D
:10AF30001146012013F0FAF910BD00001D00002099
:10AF40001C00002000200349087248708870486087
:10AF5000704700001C0A002058221152704710B59B
:10AF600004460121022000F071FA0021022000F0C5
:10AF70006DFA10BD014600205322525C10231A4086
:10AF8000002A08D05322525C0C231A409210032A44
:10AF900018D1032016E05422525A0123DB031A4031
:10AFA000002A0ED05322525C0C231A409210032A1E
:10AFB00005D05322525C9207920F032A01D102203E
:10AFC00000E0012070470246002058239B5A0B40A6
:10AFD000002B01D0012000E0002070470146002234
:10AFE0006020405AFF231B0218400005020F100189
:10AFF000014BC018704700000055044010B5002AEE
:10B000000AD056231B5A0C0223435624235256239C
:10B010001B5A8B43235209E056231B5A0C02A343AD
:10B020005624235256231B5A0B43235210BD0000B3
:10B03000F8B504460D46012700263448844203D162
:10B040000121022000F002FA2878401EA07020881A
:10B05000FF210131084320802088400840002080E3
:10B06000A878401EC1B25A20015568790007000C2B
:10B07000E97909020843A97908435C210853288922
:10B0800081B240200153A868C000C10C4220015386
:10B09000A88981B244200153E868C000C10C462051
:10B0A0000153288A81B2482001532869C000C10C8D
:10B0B0004A200153A88A81B24C2001536869C0001C
:10B0C000C10C4E2001535020005B2979090208432E
:10B0D000502108535020005B2979884350210853A0
:10B0E00000E0761C5020005B4007400F2979884221
:10B0F00002D007488642F4D15020005B4007400F41
:10B100002979884200D000273846F8BD0054044011
:10B11000FFFF000030B5034600201C898C4209DD8A
:10B12000082A05D218244C431D682C19A05C02E0A3
:10B13000002000E0002030BD10B5024613898B428C
:10B1400005DD18234B431468E318987C00E00020C9
:10B1500010BD0146FF22C889C007C00F00280AD0D1
:10B160000120C88100E0521EC889C007C00F002816
:10B1700001D0002AF7D1C889C007C00F00280FD11D
:10B180000220C8810420C881487A400840004872E3
:10B19000487A38239843487200204872012070474B
:10B1A0000020FCE70246507A012318435072507A7F
:10B1B0000B78DB0018435072087A012808D1888880
:10B1C00050814868000C0123DB031843908108E09C
:10B1D000087A002805D15081486880001A4B184031
:10B1E0009081487A012804D1507A40231843507244
:10B1F00006E0487A002803D1507A402398435072E1
:10B200000878002811D1C87A1072087B1070487B2A
:10B210005070887B9070CB7BD370087C10714B7C16
:10B220005371887C9071CB7CD371887A002803D0CD
:10B230000120C002D08101E00820D081FF20013030
:10B24000D081012070470000FC1F0000002904D0BD
:10B25000427A80231A43427203E0427A80239A435F
:10B260004272704730B5024600200F4B5024A45A5A
:10B270000D022C435025AC525024A45A8C43AC529E
:10B2800000E05B1E5024A45A6407640F8C4201D076
:10B29000002BF6D15024A45A6407640F002C01D06F
:10B2A000002000E0012030BDFFFF0000827A8023F3
:10B2B0001A40802A00D081727047000070B50446A1
:10B2C00000250023002D02D0012660200653042013
:10B2D000C88188890126F6033040002808D0012063
:10B2E00010728889C004C0084E893043506006E05F
:10B2F0000020107288890F4E304080105060087A0C
:10B30000D072002304E0CE5C10460C30C6545B1CA7
:10B31000D07A9842F7DCC88904263040002804D14E
:10B32000C889F6023040002801D0002070BDD07AD4
:10B33000FCE70000FC1F0000027C80231A40802AEA
:10B3400000D00174704710B50246FF23D089C007B2
:10B35000C00F00280AD00120D08100E05B1ED089F8
:10B36000C007C00F002801D0002BF7D1D089C0073B
:10B37000C00F002801D0002010BD507A01242043C6
:10B380005072507A3824A0435072C87A1072487AAA
:10B3900000280FD1087B1070487B5070887B90701C
:10B3A000CC7BD470087C10714C7C5471887C90717B
:10B3B000CC7CD471FF200130D0814000D081107A44
:10B3C000DAE70000F8B504460D460020002C00D155
:10B3D00000BF002A00D100BF012C01D1412630431B
:10B3E000012A01D112263043022C01D1C02630435C
:10B3F000022A01D130263043134E307076788027F0
:10B40000BE43114F7E70012C08D1FF2100BF0E4EAC
:10B41000B3781E460E4033468B42F8D10A4E7678FA
:10B420004027BE43084F7E70012A0BD100260096AC
:10B4300003E000BF009E761C0096FF276937009E40
:10B44000BE42F6D9F8BD000000040240002905D034
:10B45000054A12780243044B1A7004E0024A12783B
:10B460008243014B1A70704720040240002905D026
:10B47000054A927E0243044B9A7604E0024A927E89
:10B480008243014B9A76704700080240012006492A
:10B49000087000BF04480078802108400028F9D0D7
:10B4A0000120024908707047000C0240A0010020F2
:10B4B00070B5034614460020002B01D1C0B202E053
:10B4C00005468035E8B2012902D1051DE8B206E043
:10B4D000022903D105460835E8B200E0C0B2012CCC
:10B4E00002D1851CE8B200E0C0B2084DA870AD786A
:10B4F00001263543054EB570002201E000BF521C05
:10B500007D252D01AA42F9D970BD0000000C024032
:10B5100070B500242448007920210840002801D07B
:10B52000224D3FE000F046F8054621480078802192
:10B530000840002836D01E4880780840002801D0F6
:10B540001A4D02E000F036F80546194880780007E9
:10B55000840F022C01DBAD0804E0012C01D16D0841
:10B5600000E000BF124880788007C00F002801D09B
:10B570002D0101E00C2045430D4800784007840F61
:10B58000002C02D1601CC4B207E0032C03D1601C64
:10B590004006040E01E06006040E21462846FCF732
:10B5A000CFFD0546284670BD0004024000127A0017
:10B5B000000C024000B5C0229178F82211401C4ACC
:10B5C00012781143EA2923D00ADC0A46E03A130034
:10B5D00014F0DCFC0A181C20242A2A2A2A161A2A0B
:10B5E000ED291FD004DCEB2916D0EC291CD117E083
:10B5F000F02903D0F82917D10E4817E00E4815E0BE
:10B600000E4813E00E4811E00E480FE00E480DE022
:10B610000E480BE00E4809E00E4807E00E4805E032
:10B620000E4803E00E4801E00D4800BF00BF00BD1A
:10B63000201C02400090D003006CDC020048E801AE
:10B6400000366E010024F400001BB70000127A00DF
:10B65000808D5B0000093D00C0C62D0080841E0067
:10B6600040420F0010B50446204600F077FD002050
:10B6700010BD000010B5A8211348FCF711FE1248B8
:10B68000124908601248486007200881002088722B
:10B6900007220F490D4800F065FA00210B48FFF71B
:10B6A00005FEA0210B48FCF7FBFD0A480A4948604B
:10B6B0000A4B05220A49084800F0C0FB55210648FC
:10B6C000FFF73AFE10BD00004808002028080020BF
:10B6D0008C0D0200F00800203408002065B6000040
:10B6E000000D02000C4A127812060B4B5B781B040B
:10B6F0001A43094B9B781B021A43074BDB781A430A
:10B70000104642084240D20083085A401146034A7C
:10B710005140034A116070471707002001020000E2
:10B720001C070020F8B504460F46A07A4006400EDC
:10B73000002874D10025ACE018206843216808185F
:10B74000407C01283CD10121182068432268101850
:10B75000017400260CE0182068432168081808309E
:10B76000815D18206843226810188155701CC6B28C
:10B77000082EF0D3002118206843226810180174A5
:10B780001820684322681018417418206843226802
:10B7900010184161182068432268101881742C2009
:10B7A000684361680818406A002809D018236B4371
:10B7B0002268D0182C236B436268D218516A8847DC
:10B7C00018206843216808184069FF21C94388424E
:10B7D0005DD818206843216808184069C1191820ED
:10B7E00068432268101841611820684321680818CE
:10B7F00041692C206843626810188069814246D3F1
:10B800001820684321680818807C55283FD05521AE
:10B8100018206843226810188174002624E03CE058
:10B820001820684321680818805D2C2169436268EC
:10B8300051181031895D0840182169432268511858
:10B8400088551820684321680818805D2C216943B9
:10B85000626851180831895D0843182169432268DC
:10B8600051188855701CC6B2082ED9D32C206843B5
:10B8700061680818806A002809D018236B43226881
:10B88000D0182C236B436268D218916A8847681CD1
:10B8900085B22089A84200DD4EE7F8BD10B5044608
:10B8A000002014F0D7FE022841D12148007800285A
:10B8B00002D101201E4908701D48007801281FD1BF
:10B8C0001B484078401C1A49487021465A20FCF712
:10B8D00037FC17494978884229D800201449487014
:10B8E00008468078401C8870084680780A2803D370
:10B8F0000020887002200870002014F0DBFE16E0A3
:10B900000B480078022812D109484078401C0849A9
:10B91000487021467D20C000FCF712FC044949789C
:10B92000884204D800200249487014F0C3FE10BDBC
:10B930007400002000B587B0002168460171042121
:10B9400041710C480290411003910B4904910591FB
:10B950000A480690FFF78EFE01A814F00FFF00F0D2
:10B9600023FB00F00FF80021054809F0CBFD07B0DC
:10B9700000BD0000FFFF1F00FFFFFF1FEDBB000029
:10B980000205000010B5FF20023072494860002017
:10B9900008720120087000204872012088726E48E9
:10B9A000FFF7D7FB6B496C48FFF7FCFB01216A48A6
:10B9B000FFF74CFC69486749486000200872012085
:10B9C0000870002048720120887263481030FFF729
:10B9D000C0FB604960481030FFF7E4FB01215E487E
:10B9E0001030FFF733FC5D48401E5A494860002084
:10B9F00008720120087000204872012088725648A1
:10BA00005030FFF7A6FB534953485030FFF7CAFBAD
:10BA1000012151485030FFF719FC5048C1384D49B9
:10BA20004860002008720120087000204872012040
:10BA3000887249484030FFF78CFB46494648403001
:10BA4000FFF7B0FB012144484030FFF7FFFBFF2028
:10BA50001230404948600020087201200870002020
:10BA60004872012088723C486030FFF772FB394908
:10BA700039486030FFF796FB012137486030FFF707
:10BA8000E5FBFF2021303349486000200872012087
:10BA9000087000204872012088722F48A030FFF7FC
:10BAA00058FB2C492C48A030FFF77CFB01212A4889
:10BAB000A030FFF7CBFB29488F382649486000208B
:10BAC0000872012008700020487201208872224804
:10BAD000E030FFF73EFB1F491F48E030FFF762FBF5
:10BAE00001211D48E030FFF7B1FB3F20400119491B
:10BAF0004860002008720120087000204872012070
:10BB0000887215482030FFF724FB12491248203074
:10BB1000FFF748FB012110482030FFF797FB104842
:10BB20000C4948600020087201200870002048720B
:10BB30000120887208483030FFF70BFB05490648A2
:10BB40003030FFF72FFB012103483030FFF77EFB39
:10BB500010BD00002C2A00201055044002040000F3
:10BB6000DF070000F0B50B46144643600481002156
:10BB700036E0002216E02C254D4346687519AD5C71
:10BB800018274F430668F619B5542C254D434668CF
:10BB90007519AD5C18274F430668F6190836B55479
:10BBA000551CEAB2082AE6D3002518274F43066839
:10BBB000F619357418274F430668F6197574182757
:10BBC0004F430668F619B57418274F430668F619EF
:10BBD000F57418274F430668F61975614D1CA9B214
:10BBE00005898D42C5DC00258572F0BD70B504461F
:10BBF000606800F029FE0546E27A23460C332946A8
:10BC0000094800F0E9FD09496068884203D0491CF1
:10BC10006068884206D1E17AA28890B222460C324E
:10BC200003F02AF870BD000028080020DF0700009C
:10BC3000F8B5054600262C46002C11D000BF03E0C5
:10BC4000FF20A055701CC6B2082EF9D304F048FF9F
:10BC5000C000082108400746206888433843206018
:10BC6000F8BDF8B5054600262C46002C2DD000BFA7
:10BC700003E0FF20A055701CC6B2082EF9D305F0D2
:10BC800053F807122088000A00023843208005F08C
:10BC90004BF80002FF21090208400746208888432C
:10BCA0003843208005F042F907126088000A00023C
:10BCB0003843608005F03AF90002FF21090208408C
:10BCC00007466088884338436080F8BD70B50546F4
:10BCD00000262C46002C2CD000BF03E0FF20A055EE
:10BCE000701CC6B2082EF9D305F036F901280AD126
:10BCF00031202070012060705920A0700820E07071
:10BD00000020207115E005F027F902280AD1312022
:10BD10002070012060705920A0700820E070012080
:10BD2000207106E0002020706070A070E07002209A
:10BD3000207170BDFEB5054600260020019001F07F
:10BD400023FD0A210090FCF7FBF9074604F0FCFEF6
:10BD50000A210090FCF70AFA80B201902C46002CD0
:10BD60003AD000BF03E0FF20A055701CC6B2082ED9
:10BD7000F9D3FF21090260688843390C0902FF22C8
:10BD80001202114008436060110260688843390A5A
:10BD90000904120211400843606060680002000A52
:10BDA0003906090E09060843606004F0D3FFFF2836
:10BDB00006DDFF21090420688843401820600BE05D
:10BDC00004F0C8FF0004FF21090408400090206827
:10BDD0008843009908432060FEBDFEB50546002655
:10BDE00000200190002704F083FC64210090FCF700
:10BDF000BDF980B20190002001F0E8FC87B22C462A
:10BE0000002C1AD000BF03E0FF20A055701CC6B262
:10BE1000082EF9D3FF210904206888433912090448
:10BE2000FF22120411400843206020680002000A2B
:10BE30003906090E090608432060FEBDFFB581B032
:10BE400004460F4600250026002000902760039836
:10BE500020810498E0600020207400BF9DE01C2039
:10BE60006843216808586A01616888501C2068434B
:10BE70002168081880686A016168891848601C2078
:10BE800068432168081840686A01616889188860F9
:10BE90001C20684321680818C0686A016168891815
:10BEA000C8601C20684321680818007C6A0161682A
:10BEB000891808741C20684321680818407C6A01AE
:10BEC0006168891848741C20684321680818807CC0
:10BED0006A016168891888831C20684321680818F2
:10BEE000C07C6A0161688918887400206A016168F1
:10BEF0008918C8741C206843216808184068002805
:10BF000013D01C20684321680818C07C002805D184
:10BF1000401E6A0161688918C8831AE00020C04386
:10BF20006A0161688918C88313E01C20684321688E
:10BF30000818C07C002805D000206A0161688918B3
:10BF4000C88306E000206A0161688918C88301205F
:10BF50000090002607E000216A0160688018143014
:10BF60008155701CC6B2690160684018808BB04270
:10BF7000F1DC1C20684321680818406900280AD0B9
:10BF80006B016268D218104614301C236B43226880
:10BF9000D21851698847681CC5B22089A84200DDC3
:10BFA0005DE7009805B0F0BD00B58BB0684807901C
:10BFB000002108A801706846017608A84170002099
:10BFC00064498872082108A8C170002004E000229A
:10BFD00009A90A54411CC8B208A9C9788142F6DCF3
:10BFE0005D48FFF7B6F806A95B48FFF7DBF858484D
:10BFF000401C0790002108A801706846017608A837
:10C000004170002053498872082108A8C17000209F
:10C0100004E0002209A90A54411CC8B208A9C97841
:10C020008142F6DC4C484030FFF793F806A94A48B5
:10C030004030FFF7B7F8452000010790002108A81D
:10C0400001706846017608A8417000204149887255
:10C05000082108A8C170002004E0002209A90A54A0
:10C06000411CC8B208A9C9788142F6DC3A48503070
:10C07000FFF76FF806A938485030FFF793F8112002
:10C0800040010790002108A801706846017608A8C1
:10C09000417000202F498872082108A8C170002033
:10C0A00004E0002209A90A54411CC8B208A9C978B1
:10C0B0008142F6DC28482030FFF74BF806A92648D5
:10C0C0002030FFF76FF80B20C0010790002108A86F
:10C0D00001706846017608A8417000201D498872E9
:10C0E000082108A8C170002004E0002209A90A5410
:10C0F000411CC8B208A9C9788142F6DC16486030F4
:10C10000FFF727F806A914486030FFF74BF8FD2029
:10C11000C000029000216846017301714173817370
:10C120000821C173002004E0002204A90A54411C24
:10C13000C8B26946C97B8142F6DC07481030FFF778
:10C1400008F801A904481030FFF72CF80BB000BD27
:10C15000EE0600002C2A00208055044030B585B042
:10C160000446002520680190A1796846C172617972
:10C17000417200210172017000BF05E020460830C5
:10C18000415D03A841556D1C6846C07AA842F5D8A8
:10C190000B22D2010199881A914226D007DC184857
:10C1A000081A1CD023210901401A24D111E0FF38BC
:10C1B0006F38002802D001281DD104E069461148DB
:10C1C000FFF7C1F818E069460E484030FFF7BBF8AA
:10C1D00012E069460B485030FFF7B5F80CE06946AD
:10C1E00008482030FFF7AFF806E0694605486030A0
:10C1F000FFF7A9F800E000BF00BF05B030BD0000A8
:10C200002002000080550440F0B585B004460F467A
:10C2100000250026207C4006400E55287ED100BF18
:10C2200076E1690160684018807C002877D1690157
:10C230006068401840686A016168891889688842A6
:10C2400009D26901606840184068C0196A016168D4
:10C25000891848605AE1690160684018C068AF49B0
:10C26000884208D8690160684018C068401C6A01AB
:10C2700061688918C860690160684018C07C00283E
:10C2800021D1002607E000216A016068801814307F
:10C290008155701CC6B2690160684018808BB0423D
:10C2A000F1DC1C20684321680818406900280AD086
:10C2B0006B016268D218104614301C236B4322684D
:10C2C000D218516988476901606840580090690137
:10C2D00060684018017C6846017100214171690164
:10C2E00060684018017F6846817169016068401884
:10C2F000417C6846C171002608E069016068401809
:10C300001430815D02A88155701CC6B26901606855
:10C310004018808BB042F0DCE06801E0FCE01DE0FA
:10C32000002806D06846E16888476A016168891874
:10C33000C874690160684018C07C002804D16A0193
:10C34000616889184860E1E06901606840184068E8
:10C35000C01B6A01616889184860D7E0690160689C
:10C36000401880680028EED0690160684018C08BD2
:10C370000028E8D0690160684018C08B6A016168D4
:10C380008918C968884207D1690160684018C08B64
:10C390006249C94388427DD169016068401840689C
:10C3A0006A01616889188968884209D269016068F0
:10C3B00040184068C0196A01616889184860A5E0A2
:10C3C00000206A0161688918486069016068401846
:10C3D000C0685249884208D8690160684018C0683E
:10C3E000401C6A0161688918C860002607E00021C6
:10C3F0006A016068801814308155701CC6B26901EA
:10C4000060684018808BB042F1DC1C2068432168D2
:10C410000818406900280AD06B016268D2181046DB
:10C4200014301C236B432268D21851698847690174
:10C43000606840580090690160684018017C684657
:10C44000017100214171690160684018017F6846EF
:10C450008171690160684018417C6846C17100269D
:10C4600008E06901606840181430815D02A88155B8
:10C47000701CC6B2690160684018808BB042F0DC65
:10C48000E068002808D06846E16888476A0161686A
:10C49000891800E015E0C874690160684018C07C24
:10C4A000002804D16A016168891848602EE069019A
:10C4B000606840184068C01B6A016168891848605C
:10C4C00024E01C20684321680818406800280FD029
:10C4D0000020C0436A0161688918C8831C20684332
:10C4E0002168081840686A0161688918886008E056
:10C4F00000206A0161688918C8836A016168891827
:10C50000886000206A0161688918C860681CC5B22B
:10C510002089A84200DD84E605B0F0BD0000FFFFE1
:10C520007CB500BF19212C480078FBF709FE0446B2
:10C530002A4860432A4A8118002201200DF028F879
:10C5400020460A2250436430001981B200220120A3
:10C550000EF0C0FF01200A2262431219D1B20A2252
:10C56000624312190090D0B201231A4609F0DEFA94
:10C57000BA220721002006F0A1FF012000900190BF
:10C580000B20604382B20B20604381B20023012064
:10C590000EF07CFD6F20604381B201200FF040FA65
:10C5A000104860430246032101200BF079FD00256D
:10C5B00005E0012128460BF0ADFC681CC5B20F2D2B
:10C5C000F7DB21460B2251436431C8B20FF08CFCDB
:10C5D0000FF074FC7CBD00006F000020672B000092
:10C5E000A0860100FCB10100002005490870054942
:10C5F00008700549087005490870054908707047BA
:10C6000070000020710000206F0000206E000020EC
:10C610006D000020F0B589B000BF00BF00BF00BFB3
:10C6200000BF00BF00BF00BF00BF00BF03215C48C8
:10C630000078FBF79BFD5B494843029003210120F2
:10C64000029A0BF02DFD052155480078FBF778FD87
:10C650000446E1B201200BF0EBFA032150480078C8
:10C66000FBF784FD0B214843643080B20690E1B2B1
:10C6700001231846069A09F033FD494909788A00D2
:10C6800088180621FBF772FDFF21F531484380B27F
:10C6900007900798FBF76AFDC7B2394601200AF0F8
:10C6A00003FA03213E480078FBF760FD0B21484365
:10C6B000643080B208900022012008990EF00AFF31
:10C6C000032137480078FBF751FD37494843374984
:10C6D000401803900022012003990CF059FF032118
:10C6E0002F480078FBF742FD0B21484380B20490AD
:10C6F00003212B480078FBF739FD0B21484386B214
:10C700000120F1B20090049AD0B201231A4609F038
:10C710000DFABA220721002006F0D0FE032120489E
:10C720000078FBF723FD0B21484385B201200090E0
:10C7300000232A46294601900EF0A8FC0321184840
:10C740000078FBF713FD6F21484380B2059001206C
:10C7500005990FF065F9164800783C2805DA144869
:10C760000078401C1249087002E03C201049087013
:10C770000F4800781D2805DC09480078401C08494E
:10C7800008700BE006480078002802D104490870C0
:10C7900004E003480078401E0149087009B0F0BD6C
:10C7A00070000020FCB10100672B0000A086010092
:10C7B00071000020002000BF06E00021044A11544F
:10C7C000044A1154411CC8B25A28F6DB70470000D5
:10C7D0001C260020D0260020FFB581B004460F465D
:10C7E0003D462089A8422DDD18206843216808189D
:10C7F000007C002826D1002609E00498815D1820DD
:10C8000068432268101808308155701CC6B2082E83
:10C81000F3D30121182068432268101841742C209A
:10C82000684361680818006A00280BD018236B431E
:10C830002268D218104608302C236B436268D21845
:10C84000116A884705B0F0BD01460720124BCA1A8D
:10C85000994211D008DCCA1FFA3A002A14D0102AD3
:10C860000CD01F2A14D10DE0322A0FD0C02A07D0D5
:10C87000C12A0DD100200DE001200BE0022009E0CB
:10C88000032007E0042005E0052003E0062001E086
:10C89000072000BF00BF70474103000010B50446E9
:10C8A0007D21C90061430846322103F0C3FE10BD5B
:10C8B000FF200B4908700020C0430A4908800A493C
:10C8C0000880FF2009490870094908700949087063
:10C8D0000020094908600949086009490860704753
:10C8E0005400002056000020580000205A0000206C
:10C8F0005B0000205C000020480000204C0000206D
:10C900005000002001480068704700004C000020E3
:10C9100001480068704700004800002010B5054934
:10C9200009886522514308466421FBF71FFC80B249
:10C9300010BD00005600002001480078704700003C
:10C940005B00002001480078704700005400002080
:10C9500010B50FF0FDFF01282CD100F063F8012085
:10C9600000F066F803F0CAFE044600F043F804F055
:10C97000C9F8044600F04AF804F010FB012805D17C
:10C9800000F03EF8012000F047F805E0002000F03C
:10C9900037F8002000F040F80020134908601348E1
:10C9A0000068134988421ED210480068801C0F4955
:10C9B000086018E000200D4908600B4800680C4929
:10C9C000884204D208480068801C0749086000209B
:10C9D00000F028F8012000F02BF8002000F00AF801
:10C9E000002000F013F810BD4C000020480000208B
:10C9F000FFFFFF7F014908807047000056000020BC
:10CA000001490870704700005B0000200149088060
:10CA1000704700005800002001490870704700006E
:10CA20005C0000200149087070470000540000209D
:10CA300001490870704700005A0000200021014A97
:10CA40001171704700600040002201494A7570472B
:10CA500000600040002201494A76704700600040B3
:10CA60000021014A11727047006000400021014A14
:10CA700011737047006000400021014A1174704733
:10CA8000006000400021014A1175704700600040BD
:10CA90000021014A117670470060004000220149E0
:10CAA0004A73704700600040002201494A74704791
:10CAB0000060004010B51C4C1C49206888421ED103
:10CAC00006221B49201DFBF7F6FB002817D1112277
:10CAD000184920460A30FBF7EEFB00280FD106224A
:10CAE000154920461B30FBF7E6FB002807D106223C
:10CAF000124920462130FBF7DEFB00280DD000F064
:10CB000089FE0A480E490860074813F004FF0C4AE2
:10CB10002821054813F02AFF04E02822214608486E
:10CB2000FBF7A5FB10BD0000000250007AA7A55A34
:10CB30002D070020330700202707002021070020B1
:10CB4000382E00200020084908700849087001208C
:10CB5000074908700020074908700748074908601E
:10CB600000200749087070470F0700200E070020BB
:10CB700011070020160700202506000044070020AA
:10CB80002007002070B5054600BF91206843044689
:10CB90000A212046FBF7D4FA0446641D204670BDE6
:10CBA00070B5A8B0054600240026A0216846FBF712
:10CBB00077FB00F09FFC1E490A681421694350501E
:10CBC00000211B480268142068431018416018486F
:10CBD00002681420684310188160154840680028D6
:10CBE00024D000BF17E06006060E282E00D316E002
:10CBF0000F480168142060430858B1006A4650503D
:10CC00000B4801681420604308184168701C8000BC
:10CC10001150601CC4B20648007AA042E3DC00BF99
:10CC200062000348694643680220984728B070BDF7
:10CC3000B02E002030B5A9B000240025A02101A805
:10CC4000FBF72EFB00BF25E06006050E00F052FC4E
:10CC50001F490A6814216143505000211C48026892
:10CC60001420604310184160194802681420604382
:10CC700010188160282D0BD21548016814206043DC
:10CC80000858A90001AA50500021681C80001150CA
:10CC9000601CC4B20E48007AA042D5DC0C48406843
:10CCA000002813D00A48007A4000282806D30848F4
:10CCB000282201A943680220984707E00448007A27
:10CCC0004200034801A943680220984729B030BDBB
:10CCD000B02E002010B50FF03BFE01287ED1FFF7EB
:10CCE00017FE5549884216D20F2054494871887161
:10CCF00008468078002801D1052048704F48807888
:10CD0000052802D100204D49487000204B49087287
:10CD10004872087035E0FA204849487188714849DE
:10CD2000088803F013FE4648807800280CD1434958
:10CD3000087008464079C87008468079087100205C
:10CD40008870487048721CE001203C490870084611
:10CD5000407A022805D1012048720020C87008716D
:10CD60000FE03648407A00280BD102203349487240
:10CD700008464078887008464079C870084680792F
:10CD800008712E4880782D494978884213DD0020AB
:10CD90002A49C87008460079401C08710846007985
:10CDA0008979884222DB002024490871084680786E
:10CDB000401E88701AE021488078204949788842CE
:10CDC00014DA00201D4908710846C078401CC8705C
:10CDD0000846C0784979884208DB00E01EE0002060
:10CDE0001649C87008468078401C887014488078BE
:10CDF000002803D10120114908721BE01048008867
:10CE0000732803DB02200D49087213E00C480088E8
:10CE100070280FDC0020094908720BE00020074948
:10CE2000087008464079C87008468079087100206B
:10CE30000872487210BD0000B80B00009009002075
:10CE4000780000200020044988704870C87008717C
:10CE500008724872704700009009002000200649BF
:10CE600008808870054988704870FA20C870087179
:10CE70000020087248727047780000209009002056
:10CE800070B503F06BFC044603F07AFC05460FF026
:10CE90005FFD01282ED105211A48FEF74DF95528CE
:10CEA00004D1002018498870088027E0012D04D1A2
:10CEB000002015498870088020E001201249887000
:10CEC0001248844202DB201A84B200E000240A21C6
:10CED0002046FBF74BF9052901DB601D84B20C48A5
:10CEE000844200DD04460A212046FBF73FF906494B
:10CEF000088003E00020044988700880FFF7EAFEFC
:10CF000070BD00002808002078000020AA0A000058
:10CF1000C60700001CB500200090019000F0EAFA5E
:10CF20000B49086000200B49096808600A4800683E
:10CF300000280CD00749096808680A21FBF700F9A6
:10CF40000090012269460520034B1B6898471CBDD1
:10CF5000E0070020D4070020DC070020002008495B
:10CF6000488008490880084908800849087008492D
:10CF700088720849088048800120087170470000C5
:10CF8000300000202000002022000020240000208B
:10CF90000C08002028000020F8B503F0C1FB07466C
:10CFA00003F0D0FB0090FFF7CDFC012860D10521F4
:10CFB000C548FEF7C1F8552802D00098012807D1CE
:10CFC0000020C2490870C2490880C249887256E0F0
:10CFD000BE480078002810D10120BC4908703D46A9
:10CFE0002846E917890F091889030D0CBA488542AC
:10CFF00000DD0546B648058041E0B648807A40002D
:10D00000B4490F520846867A0EE07000B1490D5AB5
:10D01000701E4000085A7100AE4A5052701E400007
:10D0200011460D52701EC6B2002E08DD7000A949CF
:10D03000095A701E4000A74A105A8142E5DBA548F4
:10D04000807A401CA34988720846807A052816DB3E
:10D05000002088720846C5882846E917890F0918F4
:10D060008D109D48854200DD05469948058006E003
:10D07000002096490870964908809649887294481D
:10D08000058896480088A84257DA94480088281AEC
:10D0900084B292480079012827D190484088A04264
:10D0A0000BDA8E4840880A308C4948800846408810
:10D0B000A04204DD0846448001E088484480874857
:10D0C000448803212046FBF751F884B2192C00DA7A
:10D0D0001924824800880019804908800846008881
:10D0E000A84201DD08460580CDE07C484088142830
:10D0F00005DD7A48408814387849488002E00020ED
:10D10000764948807548448803212046FBF72EF86D
:10D1100084B2192C03DA012070490871B3E06F481A
:10D120000088A04205DD6D480088001B6B4908801F
:10D13000A9E0002069490880A5E068480088A84265
:10D1400059DD66480088401B84B264480079012894
:10D1500027D162484088142805DD6048408814388B
:10D160005E49488002E000205C4948805B48448872
:10D1700003212046FAF7FAFF84B2192C03DA0220C1
:10D18000564908717FE055480088001953490880C6
:10D19000084600885049884275DD08464F49088096
:10D1A00071E04E484088A0420BDA4C4840880A3073
:10D1B0004A49488008464088A04204DD0846448029
:10D1C00001E0464844804548448803212046FAF758
:10D1D000CDFF84B2192C00DA19244048008829199F
:10D1E000884202DA3D4805804DE03C480088001B3B
:10D1F0003A49088047E03948448803212046FAF735
:10D20000B5FF84B2192C3EDD34484088142805DD72
:10D210003248408814383149488002E000202F49C4
:10D2200048802E48448803212046FAF79FFF84B2A5
:10D230002A480079012813D1192C03DA0220274942
:10D24000087120E025480088001924490880084614
:10D2500000882149884216DD08462049088012E0EE
:10D26000192C03DA01201D4908710CE01B480088C5
:10D27000A04205DD19480088001B1849088002E01B
:10D2800000201649088016480088502804DC1348FE
:10D2900000881349088016E0104800881049098862
:10D2A000884204DD0D4800880D4908800BE00B48DA
:10D2B00000880B490988081A84B2502C03DB074800
:10D2C000008807490880F8BD2808002024000020B5
:10D2D000200000200C080020E02E00002800002084
:10D2E0002200002010B5044664204443A1212046BA
:10D2F000FAF726FF0446204610BD00007CB5002446
:10D3000000200190009000F03FFA05460A21FAF74C
:10D3100017FF044601226946042000F053FE0098DE
:10D32000401C002814D17D20C0002018114908603D
:10D33000084600680190012201A9032000F08EFE3A
:10D340000120009001226946042000F087FE0FE0D2
:10D35000009801280CD17D200001201805490860A3
:10D36000084600680190012201A9032000F076FE22
:10D370007CBD00002801002010B501200F49087075
:10D3800000200F49096808600D49096848600C4988
:10D390000968886000F07EF9FFF7BCFDFFF74AFCE2
:10D3A00008480068002807D00122054801680831B4
:10D3B0000020044B1B68984710BD0000AD070020FB
:10D3C000A8070020A407002010B5184800681849D5
:10D3D000884229D117480068002804D01548006801
:10D3E00080471549087015480068002804D0134884
:10D3F000006880471249087012480068002804D06D
:10D4000010480068804710490880104800680028CC
:10D4100005D00E48006880470D49088002E00D489D
:10D420000B49088000F078F810BD0000B807002014
:10D430007856341294070020AC070020980700208B
:10D44000AE0700209C070020B0070020A0070020A6
:10D45000B20700201027000010B50023174C2360EE
:10D46000174C2370174C2370174C2370174C2380D4
:10D47000174C2380174C2370174C13682360174CEC
:10D4800053682360164C93682360164CD36823605E
:10D49000154C1369236000280CD0144B1860134CF2
:10D4A0000B682468A3600023104C246823600F4C91
:10D4B000246863600E4B014C236010BDB807002048
:10D4C000B4070020AC070020AE070020B007002002
:10D4D000B2070020AD070020940700209807002025
:10D4E0009C070020A0070020A4070020A807002018
:10D4F00078563412054800680549884203D105482A
:10D500000068806870470020C043FBE7B807002030
:10D5100078563412A807002070B500240025002694
:10D520003048007801285CD12F480078002858D175
:10D530002E480078012854D12D4805882D490988A6
:10D54000694308462C49FAF7FBFD85B2E12000014A
:10D55000854207D81921694308460921FAF7F0FDE9
:10D56000044600E0244C254800680068001923495F
:10D57000096808602148006800682049096849680E
:10D58000884207D31D48006800681C49096849683B
:10D59000461A0AE01948006840680021C943081A81
:10D5A0001649096809684018461C1548864218D370
:10D5B000344601462046FAF7C3FD04460F4800688A
:10D5C00041680F48604308180C4909684860012009
:10D5D0000C49087009480068806800190749096803
:10D5E000886070BDAC070020AD070020AE070020AA
:10D5F000B0070020B207002010270000A807002075
:10D60000A0860100B407002000220C4B1A600C4BCE
:10D610000A681A600B4B4A681A600B4B8A681A60DA
:10D620000A4BCA681A600A4B0A691A60002801D0BE
:10D63000084A1060084A014B1A607047B80700207A
:10D6400094070020980700209C070020A0070020D6
:10D65000A4070020A80700207856341210B50A4805
:10D66000006800280ED00948007801280AD100205F
:10D670000649087001220648016808310020024B63
:10D680001B68984710BD0000A4070020B4070020C5
:10D69000A80700201CB50020009001900024FFF78F
:10D6A00029FF04460E480068046000200C49096800
:10D6B00048600B49096888600A48006800280DD056
:10D6C00007480068006800900548006840680190BD
:10D6D000022269460120034B1B6898471CBD0000CD
:10D6E000BC070020C0070020F8B505460C461646CA
:10D6F0000027002D17D00E480560FFF7FBFE0746F8
:10D700002068B84203D90A480068076003E0084966
:10D71000206809680860064960680968486004492B
:10D72000A0680968C8600348066000F005F8F8BD05
:10D73000BC070020C007002070B500240025FFF7BB
:10D74000D9FE04460F4800680068A04200D903E0F3
:10D750000C4800680068251A0A48006840684019AB
:10D7600008490968886007480068806805490968B1
:10D77000C968884205D903480068C068014909683A
:10D78000886070BDBC070020014800688068704751
:10D79000BC070020002801D0024A1060024A116034
:10D7A00070470000BC070020C0070020054900208A
:10D7B00005E00A1D135C044A1354421CD0B2202811
:10D7C000F7DB704700065000642E00200146104829
:10D7D000026814204843101882680D48036814201A
:10D7E00048431818C06882420BD9094802681420BF
:10D7F00048431018C26806480368142048431818A4
:10D8000082600348026814204843101880687047FB
:10D81000B02E00200021002005E01A4A135C1A4AAD
:10D820001354421CD0B20628F7DB1121002006E079
:10D83000164A135C144A921D1354421CD0B28842FB
:10D84000F6DB002006E0124A135C0F4A173213542D
:10D85000421CD0B20628F6DB002006E00D4A135C1D
:10D86000094A1D321354421CD0B20628F6DB0020B0
:10D8700005E00023044A23321354421CD0B201288D
:10D88000F7DB70472D0700203C2E002033070020D7
:10D89000270700202107002038B50446002000900B
:10D8A000009401226946052000F0D8FB38BD000035
:10D8B00008B50020009001226946062000F082FB96
:10D8C00068460078094908736846407848730846F6
:10D8D000007B074908730548407B48730348807BF9
:10D8E00088730248C07BC87308BD00000C28002064
:10D8F000381F002008B5002000900122694606204C
:10D9000000F060FB684600780E490873684640786E
:10D91000487300200C490860486008724872887299
:10D9200003F0E4F80849C8720648007B087305480C
:10D93000407B48730348807B88730248C07BC87370
:10D9400008BD00000C280020381F002038B5002436
:10D950000025002000900121FE48FDF7EDFB552831
:10D9600008D002F051FFFC49087302F061FFFA4948
:10D97000487306E0F948007BF7490873F748407B95
:10D980004873F548007B00281ED1F5480068F5492A
:10D99000884208D8F2480068401CF149086000201D
:10D9A000ED49087359E0ED48007B022807D0EB48A9
:10D9B000007B032803D00320E74908734DE0E748C4
:10D9C000007BE549087348E0E348007B01281ED14D
:10D9D000E3480068E349884208D8E1480068401CF1
:10D9E000DF4908600120DC49087336E0DB48007B32
:10D9F000022807D0D948007B032803D00320D6494A
:10DA000008732AE0D548007BD349087325E0D24843
:10DA1000007B02280FD10020D149086002F01EFFD0
:10DA200000281AD002F01AFF401C002815D002204E
:10DA3000C949087311E0C848007B032806D10020BB
:10DA4000C74908600320C449087306E00020C449A0
:10DA50000860C248007BC0490873BF48407B00286B
:10DA60001ED1C1480068BF49884208D8BE48006836
:10DA7000401CBD4908600020B749487359E0B748C9
:10DA8000407B022807D0B548407B032803D0032001
:10DA9000B14948734DE0B148407BAF49487348E015
:10DAA000AD48407B01281ED1AF480068AD4988428F
:10DAB00008D8AD480068401CAB4908600120A64961
:10DAC000487336E0A548407B022807D0A348407B36
:10DAD000032803D00320A04948732AE09F48007B15
:10DAE0009D49487325E09C48407B02280FD10020C7
:10DAF0009D49086002F0D0FE00281AD002F0CCFE4A
:10DB0000401C002815D002209349487311E0924828
:10DB1000407B032806D100209349086003208E49EA
:10DB2000487306E00020904908608C48007B8A49D1
:10DB300048738948007B8949097B884205D186481A
:10DB4000407B8649497B884246D08348007B834995
:10DB5000097B884202D001207F4988737E48407B40
:10DB60007E49497B884202D001207B49C8737A48AC
:10DB7000007B022803D07848007B032803D1764835
:10DB8000007B764908737448407B022803D07248B2
:10DB9000407B032803D17048407B704948736E482E
:10DBA000007B02280BD06C48007B032807D06A4812
:10DBB000407B022803D06848407B03280CD167488B
:10DBC000017B684601706548417B684641700122CF
:10DBD0006946062000F042FA02F088FF5E49C872EA
:10DBE00002F01CFE044602F02FFE0546FEF7AAFED8
:10DBF000012873D101215748FDF79EFA552807D116
:10DC00000020554908724872086048608872B5E083
:10DC1000FF2C01D0FF2D62D1FF2C2AD1FF2D28D05F
:10DC200000204D4908720120487250480860FF20CA
:10DC300014306843486048686621FAF781FA46491B
:10DC40004860084640684949884202D90846424926
:10DC5000486041484068AA2803D33F484068FA28F2
:10DC600003D901203C49887288E000203A49887233
:10DC700084E0FF2C2AD0FF2D28D1012036490872DC
:10DC80000020487239484860FF2014306043086023
:10DC900008686621FAF754FA2F49086008460068B8
:10DCA0003249884202D908462B4908602A48006850
:10DCB000AA2803D328480068E62803D9012026496A
:10DCC00088725BE000202449887257E02748224987
:10DCD000086048600020087248724FE089E0012027
:10DCE0001D4908724872FF201430604308600868BC
:10DCF0006621FAF725FA18490860084600681B49AA
:10DD0000884202D9084614490860FF20143068434D
:10DD10001149486048686621FAF712FA0E494860CE
:10DD2000084640681149884202D908460A494860B5
:10DD300009480068AA280BD307480068E62807D8D6
:10DD400005484068AA2803D303484068FA2812D936
:10DD500001200DE028080020381F00200C2800209A
:10DD6000C400002070170000C8000020DE0300007F
:10DD70002449887202E00020224988722148007BF1
:10DD8000002802D11F49887315E01E48007B012836
:10DD900002D11C4988730EE01A48007B022802D188
:10DDA0001849887307E01748007B032803D11549F9
:10DDB0008873154808601348407B002802D1114938
:10DDC000C8731DE00F48407B012802D10D49C8737C
:10DDD00016E00C48407B022802D10A49C8730FE0C4
:10DDE0000848407B03280BD10649C87306484860A1
:10DDF00006E0002003490872487208604860887293
:10DE000038BD0000381F0020DE030000FFB583B0DE
:10DE100006460D46174600240020029000BF14203D
:10DE2000784380190190002E57D00198002854D0D3
:10DE30002B4806602A49069848600846077200BFCA
:10DE400045E0FFF757FB02902001295802988142D4
:10DE500004D820012858401C002806D120490298E7
:10DE60000A6814216143505006E0200129581C48DB
:10DE70000268142060431150200140194068401C82
:10DE8000002807D1002116480268142060431018AA
:10DE9000416008E0200140194168114802681420DF
:10DEA0006043101841602001401981680C480268E5
:10DEB000142060431018C16020014019017B0848FC
:10DEC00002681420604310180161601CC4B2044849
:10DED000007AA042B5DC00F005F807B0F0BD000004
:10DEE000B02E002070B5002400250026FFF702FBAD
:10DEF000054600BF4EE02A480168142060430858D8
:10DF0000A84239D8264801681420604308582E1AC0
:10DF1000234801681420604308184068811920488C
:10DF2000026814206043101881601D4801681420A5
:10DF30006043081881681A4802681420604310186A
:10DF4000C068814224D9164801681420604308182B
:10DF50000069002803D02046FEF722FE18E0104892
:10DF60000168142060430818C1680D480268142035
:10DF70006043101881600BE0094801681420604379
:10DF80000818406806490A681421614351188860DE
:10DF9000601CC4B20248007AA042ACDC70BD000034
:10DFA000B02E002010B500BF14244C4323180028C5
:10DFB00005D0002B03D0024C20606260217210BD9E
:10DFC000B02E0020F8B505460E4614462B0011F081
:10DFD000DDFF0705131A21282F363D001D48FAF7EB
:10DFE000BDFD1D4908701B48FAF772F90746642108
:10DFF000FAF7A6F830602AE0A004020C3146162099
:10E00000FAF7A6FE23E0A004020C31464820FAF7F6
:10E010009FFE1CE0A004020C31468020FAF798FE17
:10E0200015E0A004020C3146A020FAF791FE0EE0A4
:10E03000A004020C3146B020FAF78AFE07E0600423
:10E04000020C3146C020FAF783FE00E000BF00BF9B
:10E050000020F8BDFE270020DD00002070B5054639
:10E060000E4614462B0011F091FF07051D242B329C
:10E07000393F46003068002802D1FAF70DFC10E065
:10E0800064223168514308461C49FAF72BF90020F5
:10E090001B490870012264211848FAF7C7FE184985
:10E0A000087029E0A004020C31461620FBF70EF898
:10E0B00022E0A004020C31464820FBF707F81BE0E1
:10E0C000A004020C31468020FBF700F814E0A00405
:10E0D000020C3146A020FAF7F9FF0DE0A2B231465A
:10E0E000B020FAF7F3FF07E06004020C3146C020CD
:10E0F000FAF7ECFF00E000BF00BF70BDF027002082
:10E10000DC00002000B5AFB050211BA8FAF7C8F81A
:10E1100000201A90142115A8FAF7C2F800201290D6
:10E12000139014901190402101A8FAF7B9F800203B
:10E1300000905149086001221BA9FFF743FF1B987B
:10E14000401C002801D11A9001E01B981A904B48FE
:10E1500015904B4816904B481790002018904A484D
:10E16000199015AA1AA94948FFF776F902221CA9A5
:10E170000120FFF727FF1C98401C002801D11290B6
:10E1800001E01C9812901C98401C002801D11390AB
:10E1900001E01D9813903E48149012A93D48199A29
:10E1A000FFF7A2FA08221EA90220FFF70BFF1E9814
:10E1B000401C002801D1019001E01E9801901F9899
:10E1C000029035480390012069460874801E05902E
:10E1D00032490791012101A80177881E09902F4932
:10E1E0000B91012109A80173881E0D902B490F91F5
:10E1F00001210DA80173042201A92948199BFFF7E9
:10E2000005FE01221BA90320FFF7DCFE25491B9810
:10E2100008601B98401C002806D1FF20F5300860DC
:10E2200001220320FFF71AFF01221BA90520FFF797
:10E23000C9FE1B98401C002807D101201A4988609C
:10E24000012208310520FFF709FF01221BA9062042
:10E25000FFF7B8FE1B98401C002808D10021684633
:10E2600001704170012269460620FFF7F7FE0F4852
:10E27000014908602FB000BDE000002045C9000042
:10E2800039C900001DC900005DE00000842700209E
:10E2900076841E00902700200F2700009F86010033
:10E2A000A0270020280100200C280020A33AA55A0E
:10E2B00000B585B014216846F9F7F2FF00200F4938
:10E2C00008600F4800900F4801900F48029000200E
:10E2D00003900E48049069460D48FFF795F90D48E4
:10E2E0000499FFF757FA04210B48049AFFF75AFEE6
:10E2F0000A480249086005B000BD0000E0000020A7
:10E3000045C9000039C900001DC900005DE00000DA
:10E310008427002090270020A0270020A33AA55A98
:10E3200000200B4908800B4908800B490880012018
:10E330000A49087000200A4908730A490880488081
:10E3400001200871002006494880088070470000BD
:10E35000380000203A0000203C0000203E00002051
:10E360001808002040000020FEB502F013FA0090CB
:10E3700002F01AFA0190FEF7E5FA01286BD10521A7
:10E38000D448FCF7D9FE552807D10020D24908709F
:10E39000D2490880D249888067E00198012807D1D6
:10E3A0000020CD490870CD490880CD4988805CE0C7
:10E3B000C9480078002808D10120C7490870009D8D
:10E3C0000A206843C54908804FE0009881B2C448DC
:10E3D000007B4200C248801D8152801F067B11E0F5
:10E3E0007100BF48801D455A701E4100BC48801D09
:10E3F000415A72008152701E4100B948801D455239
:10E40000701EC6B2002E0ADD7100B548801D415A4B
:10E41000701E4200B248801D805A8142E0DBB04845
:10E42000007B401CAE4908730846007B032807DBCD
:10E4300000200873084605890A206843A749088018
:10E440000020A74908804880A448008888800120CF
:10E45000A149087009E000209F4908709F49088081
:10E460009F4908804880087388809C4805889D489B
:10E470000088A84256D29B480088281A84B299483E
:10E480000079012826D197484088A0420BDA9548A8
:10E490004088801C9349488008464088A04204DD9B
:10E4A0000846448001E08F4844808E484488032118
:10E4B0002046F9F75BFE84B2022C00DA0224894878
:10E4C000008800198749088008460088A84200D9BA
:10E4D0000D80CDE083484088062805DD81484088CE
:10E4E000801F8049488002E000207E4948807D48A6
:10E4F000448803212046F9F739FE84B2022C03DA5E
:10E50000012078490871B3E076480088A04205DD13
:10E5100074480088001B73490880A9E000207149F5
:10E520000880A5E06F480088A84259D96D48008846
:10E53000401B84B26B480079012827D16948408884
:10E54000062805DD67484088801F6649488002E04C
:10E550000020644948806348448803212046F9F735
:10E5600005FE84B2022C03DA02205E4908717FE0C6
:10E570005C48008800195B490880084600885A49B1
:10E58000884275DD08465749088071E05548408843
:10E59000A0420BDA53484088801C52494880084604
:10E5A0004088A04204DD0846448001E04D48448094
:10E5B0004C48448803212046F9F7D8FD84B2022C48
:10E5C00000DA0224474800882919884202D24549C6
:10E5D0000D804DE043480088001B4249088047E019
:10E5E0004048448803212046F9F7C0FD84B2022C3C
:10E5F0003EDD3C484088062805DD3A484088801FBB
:10E600003849488002E0002036494880354844882F
:10E6100003212046F9F7AAFD84B232480079012887
:10E6200013D1022C03DA02202E49087120E02D4874
:10E63000008800192B490880084600882A4988422A
:10E6400016DD08462749088012E0022C03DA012073
:10E65000244908710CE023480088A04205DD2148C8
:10E660000088001B1F49088002E000201D49088027
:10E670001C4800881D490988884203DA1948008827
:10E680000F2804DA17480088184908800AE015485E
:10E69000008816490988081A0F2803DB11480088EA
:10E6A00012490880114807880B48007800280DD0CF
:10E6B0006C20474364213846F9F742FD07460A4873
:10E6C000874200D907460A490F8002E00020084926
:10E6D0000880FEBD280800203E00002038000020F1
:10E6E0001808002040000020C60700003C00002061
:10E6F0003A000020002007490880074908800749A0
:10E700000880488001200871002005494880088061
:10E71000704700003A0000203C000020400000202C
:10E7200018080020002004490870044908700021DE
:10E7300003480176704700007C0000207D00002027
:10E74000FC09002070B500250024FEF7FBF8012825
:10E7500063D103213448FCF7EFFC552808D1002091
:10E76000324908703249087000213248017659E078
:10E770002F480078002807D102F0ACF82B49087028
:10E7800001202B4908704DE001202949087002F052
:10E79000A1F82849097E8900264A603A5050254848
:10E7A000047E10E0A000234960390D5C601E8000EB
:10E7B0000858A1001F4A603A5050601E8000114660
:10E7C0000D50601EC4B2002C0ADDA000194960394A
:10E7D0000958601E8000174A603A10588142E1D300
:10E7E0001448007E401CC1B212480176007E1E28EB
:10E7F00018DB00210F48017601466039896B02461B
:10E80000603AD26B89180246603A126C881803216C
:10E81000F9F796FC0549087004E0002003490870E8
:10E820000349087070BD0000280800207C0000200B
:10E830007D000020FC090020F0B5A9B004460E467A
:10E840000025002700202890A0216846F9F728FD20
:10E85000FEF750FE26490A681421614350502448AF
:10E860000168142060430818C068B0420CD22048E8
:10E870000168142060430818C1681D48026814200C
:10E8800060431018416005E0194801681420604396
:10E890000818466016484068002826D0002517E072
:10E8A0006806070E282F00D316E0114801681420CF
:10E8B00068430858B9006A4650500D480168142052
:10E8C000684308184168781C80001150681CC5B264
:10E8D0000748007AA842E3DC00BF6A0004486946A2
:10E8E00043680220984701202890289829B0F0BD5D
:10E8F000B02E002010B500F0F5FD00F0D7F810F0B4
:10E9000075FA00F00DFB00F001F810BD70B541483C
:10E910000078912800D070BD00F0BEF8012876D1B3
:10E920003D4800883D49088008468078F0218843AA
:10E9300020303A498870084680780009000135493E
:10E94000097A0907090F0843344988703148807AE9
:10E95000401E3049887208460089401C08810846DC
:10E960000089C988884216DA08202C498872002458
:10E970000EE0284841882848001D415C2748C01CFB
:10E98000015524484088401C22494880601CC4B27C
:10E99000072CEEDB2DE01F4800891E49C9888842FC
:10E9A0001CD11C4800791B498978401AC5B2681CE3
:10E9B0001A49887200240EE0164841881648001D46
:10E9C000415C1648C01C015512484088401C114942
:10E9D0004880601CC4B2AC42EEDB0AE000F00EFDE1
:10E9E00000200C4908700C490888092100F0B8F98A
:10E9F00091E7012000F0C4FC084A917A1088921C2B
:10EA000000F070F905490888002100F0C1F800BF46
:10EA100081E70000EC2B0020882B0020182B002021
:10EA20001B49097E002932D01949897E0C225143A5
:10EA3000174A515A174A118000200CE01449897E68
:10EA40000C225143124A8918891C0A5C1149891CFD
:10EA50000A54411CC8B20828F0DB0D49897E0C22FB
:10EA600051430B4A8918897A0A4A91720121D1725D
:10EA70000749097E491E064A11761146897E491CBE
:10EA800091761146897E022901DB0021917670473B
:10EA9000E42A00200C2B00200349487B012802D1E6
:10EAA0000021014A51737047FC2B002010B53348F8
:10EAB0004068002861D13148007B030011F066FAFC
:10EAC00007590512212E3D4A59002D48007800288B
:10EAD00007D000202A4908702A490888012100F03F
:10EAE0003FF947E026480078002809D00020244953
:10EAF000087025494A8808880123091D00F040F95B
:10EB000038E01F480078002807D000201C49087012
:10EB10001C490888022100F023F92BE018480078EE
:10EB2000002809D000201649087017494A8808882B
:10EB30000923091D00F024F91CE011480078002881
:10EB400007D000200E4908700E490888092100F0FE
:10EB500007F90FE00A480078002809D0002008498A
:10EB6000087009494A8808880323091D00F008F93C
:10EB700000E000BF00BF00F041FC10BDFC2B0020F6
:10EB8000EC2B0020882B0020242B00207047000055
:10EB900070B504460D4634480088A04263D1002D6C
:10EBA00061D13248007822284ED004DC20283DD0A4
:10EBB000212856D141E0902802D0912851D115E06A
:10EBC0002A48C08801280AD100202849087000F08E
:10EBD00015FC27490888002100F0C2F805E0032051
:10EBE00000F0CEFBA020214908703BE01F480089BF
:10EBF0001E49C98888420AD100201C49087000F0CB
:10EC0000FDFB1B490888002100F0AAF80DE0174819
:10EC1000807A002806D000F0F1FB1449087B00F050
:10EC200091FB02E0032000F0ABFB1BE0062000F0AC
:10EC3000A7FB11200D49087014E0062000F0A0FB8E
:10EC400011200A4908700DE000200849087000F002
:10EC5000D5FB08494A8808880923091D00F090F867
:10EC600000E000BF00BF70BD002B0020EC2B002097
:10EC7000882B0020242B002070B50346184C247EDE
:10EC8000022C00DB70BD164C647E0C256C43144DC9
:10EC90002B5300200AE0155C114C647E0C26744353
:10ECA0000F4EA419A41C2554441CE0B28842F2D390
:10ECB0000B4C647E0C267443094EA419A172344691
:10ECC000247E641C35462C762C46647E641C6C764F
:10ECD0002C46647E022C01DB00246C7600BFD1E759
:10ECE000E42A0020F0B585B007460D4616461A48BE
:10ECF0000780002406E031781748801C0155761CF7
:10ED0000601CC4B2AC42F6DB2C4605E0AA211248D6
:10ED1000801C0155601CC4B2082CF7DB0E4800882B
:10ED2000019008216846C172002141720172017090
:10ED3000002406E00848801C015D03A80155601C02
:10ED4000C4B2082CF6DB69460448FCF7FCFA012043
:10ED50000149887205B0F0BD002B00209055044099
:10ED600070B504460D46294620460FF061FF70BD80
:10ED700070B504460D46294620460FF067FF70BD6A
:10ED8000F8B504460D4616461F463B463246294610
:10ED900020460FF05CFFF8BDF8B507460E46154655
:10EDA0005C480078002804D009213846FFF7D8FFD6
:10EDB000F8BD002D01D0602D04DD09213846FFF794
:10EDC000CFFFF5E7544807804580002406E03178FE
:10EDD0005148001D0155761C601CC4B2AC42F6DBE4
:10EDE00000204C49487008468580FF2088727F20AB
:10EDF00008730846808808282EDA0120C880084653
:10EE00008088488001200881434800884349088061
:10EE100008468078F0218843404988700846807809
:10EE2000000900013B4909790907090F08433B49DB
:10EE3000887038480079401C8872002407E0364802
:10EE4000001D015D3548C01C0155601CC4B231482D
:10EE50008088A042F3DC4AE00721681CF9F786F9B4
:10EE6000002907D0072128460830F9F77FF92949FA
:10EE7000C88005E00721681CF9F778F92549C880A2
:10EE8000062024494880012008812348008823491E
:10EE9000088008468078F021884310301F49887028
:10EEA00008468078000900011A4989880905090F78
:10EEB00008431A49887008464088FF2109028843A0
:10EEC000144989880902FF2212021140084313499C
:10EED000488008208872002407E00F48001D015D6B
:10EEE0000E48001D0155601CC4B2062CF5DB012044
:10EEF00000F046FA094A917A1088921CFFF7F2FE58
:10EF0000902004490870054908880021FFF740FE59
:10EF100000BF4DE7EC2B0020882B0020182B002091
:10EF200010B5FFF77DFD1448C07A002822D01248A2
:10EF300080780009002806D0012807D002280AD0CE
:10EF4000032810D10CE000F0A5F90FE000F09EF8C6
:10EF500000F062FA0AE000F011F800F05DFA05E056
:10EF600000F000F902E0FFF711FE00BF00BF002033
:10EF70000149C87210BD00000C2B002010B540489C
:10EF80000078112800D010BD3E4800883F2149017B
:10EF9000884200D0F7E73B4880780007000F3849E7
:10EFA000097A0907090F88420CD0002034490870FB
:10EFB00000F024FA34494A8808880423091DFFF721
:10EFC000DFFEE0E72E480089401C2D4908810846F5
:10EFD000807A401E887208460089C98888421BDAF8
:10EFE0002848807A082800D0CDE700240EE0254884
:10EFF000C01C015D224842882348001D81542048DE
:10F000004088401C1E494880601CC4B2072CEEDBBF
:10F01000062000F0B5F930E0194880881849498881
:10F02000401A1849897A884203DA1648807A0828F3
:10F0300000D0A8E700240EE01248C01C015D104873
:10F0400042881148001D8154601CC4B20C4840889D
:10F05000401C0B4948800A484088094989888842F1
:10F06000EADB00200649087000F0C8F906494A8822
:10F0700008880023091DFFF783FE00BF83E7000017
:10F08000EC2B00200C2B0020242B002070B53248E4
:10F09000007880210840802800D170BD2F4800886A
:10F0A0003F214901884200D0F7E72C48807A0828A0
:10F0B00000D0F2E72948807805072D0F2D02274858
:10F0C0004088000A0543082D00DAE6E700202249BF
:10F0D0004870062048800846858001200881082065
:10F0E00088720020C8728988481C0721F9F73EF809
:10F0F000002909D018498988084608300721F9F7FE
:10F1000035F81549C88007E013498988481C07214C
:10F11000F9F72CF81049C880104800881049088079
:10F1200008464580002407E00C48001D015D0C489E
:10F13000001D0155601CC4B2062CF5DB042000F054
:10F140001FF9102004490870054A51881088FFF7FC
:10F150000FFE00BFA1E70000EC2B00200C2B0020CD
:10F16000242B002010B548480078A02808D0464835
:10F170000078912804D044480078A12800D010BD20
:10F18000424800883F21490188420AD04049088806
:10F190000921FFF7E5FD00F031F900203A49087038
:10F1A000EDE73A48807A08280AD0394908880921C9
:10F1B000FFF7D6FD00F022F9002033490870DEE7A2
:10F1C000324880780007000F002804D001282DD095
:10F1D00002284BD136E02C484078002800D050E07F
:10F1E0002A48C078002803D101202749487003E04D
:10F1F0002648C078244988722348007891280BD08B
:10F2000022480079002803D101201F49087303E038
:10F210001E4800791C49087391201B49087000F0B2
:10F22000EDF81949087B00F08DF82AE0164840787F
:10F23000002800D025E0A12013490870032000F029
:10F240009FF81EE010484078002800D019E00E48D2
:10F250000078A02809D10E4908880821FFF780FD11
:10F2600000F0CCF80020084908700AE00849088836
:10F270000521FFF775FD00F0C1F800200249087074
:10F2800000BF00BF00BF7AE7EC2B00200C2B002052
:10F29000882B002010B5284800788021084080285D
:10F2A00000D110BD24480078002806D023480088EB
:10F2B0003F214901884200D0F3E72048807A1F4966
:10F2C00089780907090F884203DD1C48807A0828DD
:10F2D00000D0E6E7194880780007000F002805D025
:10F2E000164880780007000F072800DDD9E713488B
:10F2F000008813490880114880780007000F488073
:10F30000002407E00D48C01C015D0D48001D01559B
:10F31000601CC4B20A484088A042F3DC00200649C1
:10F32000087000F06BF806494A8808880023091D18
:10F33000FFF726FD00BFB4E7EC2B00200C2B0020CC
:10F34000242B00207F2805DC7D21C90041430A4A87
:10F3500091600DE0F12808DBF92806DC0107090FB0
:10F3600064225143044A916002E00449024A9160D8
:10F370000221014A51737047FC2B002018F0010054
:10F3800000B5030010F002FE0729050B11171D231D
:10F3900029000121144A11731449516022E002210D
:10F3A000114A1173114951601CE003210E4A117377
:10F3B0000F49516016E004210B4A11730D49516049
:10F3C00010E00521084A1173002151600AE006216E
:10F3D000054A11730849516004E00021024A117383
:10F3E000516000BF00BF00BDFC2B0020A8610000E1
:10F3F000F824010028230000F04902000020014900
:10F4000008737047FC2B0020024909880918014A3B
:10F4100011807047FC2B002010B52F480078102871
:10F4200018D12E48408860280ADD2D4880780009D0
:10F430000001801C2A49887022202749087025E095
:10F44000274880780009000125498870202022493A
:10F4500008701BE020480078112816D11E48807AD9
:10F46000002800D010BD1C484078002800D0F9E7E3
:10F470000820194988721A48807800090001184943
:10F48000887020201449087000E0EBE7FD20C000E0
:10F490001349088008468078F021884330301049AD
:10F4A00088700846C0780020C8700846007914208B
:10F4B0000871032088720220FFF762FF084A917AE0
:10F4C0001088921CFFF70EFC054908880021FFF701
:10F4D0005FFB00BFC6E70000EC2B0020242B0020C0
:10F4E000182B0020244A118852888A4242D0224A8E
:10F4F00052888A4204DA204A52888A1A90B207E077
:10F500001D4A52880023DB439A1A521C521890B2AB
:10F51000194A5180127B002A10D0174A5268002ADB
:10F520000CD0154A5268824205D9134A5268121A01
:10F53000114B5A6002E000220F4B5A600E4A527B78
:10F54000022A17D10C4A9268002A0CD00A4A926803
:10F55000824205D9084A9268121A074B9A6002E063
:10F560000022054B9A60044A9268002A02D10122C7
:10F57000014B5A7370470000FC2B002010B506F0B9
:10F580009BF810BD00BF704710B504468020204393
:10F5900001460320400205F049FF10BD10B51021BF
:10F5A0000320400205F042FF10BD000010B5022408
:10F5B000024805F08BFF0446204610BD01060000FE
:10F5C00010B50021014805F031FF10BD0106000013
:10F5D00010B50446802020430146024805F026FF6E
:10F5E00010BD00000106000010B51021014805F013
:10F5F0001DFF10BD0106000030B503460C4600217A
:10F6000001250D48834201D0002B01D1022030BDDD
:10F61000012A01D10120FAE7002108E0C8002058A2
:10F62000984202D100252846F1E7481C81B2914258
:10F63000F4DB2846EBE70000FFFF0000002000BFDE
:10F6400014E00021C200134B9950C200D2189180DF
:10F65000C200114B9950C200D2189180C2000F4BCA
:10F660009950C200D2189180411C88B24828E8DB2A
:10F670000B490C4A11600C495160002191600B4903
:10F6800011610B49D16000210A4A11800A4A1170A8
:10F69000704700005C1F00209C210020DC2300201C
:10F6A000690B0100481F0020050C0100AF0C010090
:10F6B000A10C0100CE000020D2000020F0B585B0E2
:10F6C0000646674F3846039002900025002400202C
:10F6D0000190009063480068002803D061490868E1
:10F6E000804707465F484068002803D05D49486866
:10F6F000804703905B488068002803D05949886898
:10F700008047029057480069002803D0554908698E
:10F71000804700905348C068002803D05149C8680A
:10F7200080470546482D00DD48250098002876D002
:10F73000002D74DD4C480088A8420BDA2B463A466F
:10F7400049494A48FAF7CAFF2B4647494748039AAE
:10F75000FAF7C4FF44480088002833DD4248008897
:10F76000A84202D1002040490880002415E0E000B2
:10F770003F490858E1003D4A515888420BD0E0000B
:10F7800011460858E1003A4A5050E0001146085826
:10F79000E100384A5050601C84B2AC42E7DB0120E3
:10F7A000354908702C460BE00020E100314A5050EA
:10F7B000E1002F4A5050E1002C4A5050601C84B2A6
:10F7C000482CF1DB2B4800682549884246D029485F
:10F7D00080882A49884205DA264880888019254988
:10F7E00088803BE00020234988800846006801901B
:10F7F000012D33DD002408E0601CC0001D490858BD
:10F80000E1001C4A5050601C84B2681EA042F3DC28
:10F81000691EC900174A019850501FE0FFE70020F9
:10F8200015490870002414E00020E100114A5050EE
:10F83000E10089188880E1000C4A5050E1008918E5
:10F840008880E1000A4A5050E10089188880601CD5
:10F8500084B2482CE8DB00200349088005B0F0BDE5
:10F86000FFFF0000481F0020CE0000209C21002048
:10F87000DC2300205C1F0020D20000208813000041
:10F8800001460020704700002E480078401C2D499A
:10F8900008702D480078401C2B4908702B480078D0
:10F8A000401C2A4908702A480068401C2849086002
:10F8B00008460068FF219131884202D9002024497E
:10F8C000086020480078C82802D900201D49087027
:10F8D0001D480078842802D900201B4908701B4865
:10F8E0000078502802D90020184908701948184992
:10F8F0000968405C18490870184812490978405C4A
:10F9000017490870174810490978405C1649087073
:10F9100016480E490978405C154908701548094990
:10F920000978405C14490870144806490978405C1D
:10F9300013490870134803490978405C124908705C
:10F94000704700005307002054070020550700208F
:10F9500058070020EB1402004C0700207B16020021
:10F960004D070020431702004E0700208F180200A9
:10F9700050070020C71702004F070020DF180200C1
:10F9800051070020A71902005207002010B582007D
:10F99000054BD218525C012A04D100228300024C8C
:10F9A0001B195A5410BD0000682A002010B50446E7
:10F9B000204600F049FA204600F002F810BD000091
:10F9C00010B50446B248007800287DD1B1480088BF
:10F9D000B149884278DAB148007800284FD0B04861
:10F9E0000078002803D0AB480088AE490880AE48B4
:10F9F0000078002818D1A7480188AA480088193043
:10FA0000814206D30120A8490870A2480088A54970
:10FA10000880A0480088A349098888421CDA9D48CC
:10FA20000088A049088017E09E480188994800880E
:10FA30001930814206D300209B4908709548008800
:10FA4000984908809348008896490988884203DDD0
:10FA5000904800889349088093480078002857D13F
:10FA600092480078042803D08D480078002807D0F9
:10FA700088480088822803DA05208C490870A1E0B4
:10FA80008A480078032803D085480078002809D0E8
:10FA900080480088FF211931884203DA0420834915
:10FAA00008708FE081480078022803D07C480078F5
:10FAB00000280AD077480088FF21AF31884204DA55
:10FAC00003207A4908707DE0E0E07848007801285A
:10FAD00003D073480078002808D06E480088744925
:10FAE000884203DA0220714908706BE06F480078A1
:10FAF000002803D06A480078002863D06548008851
:10FB00003721090188425DDA01206849087059E00F
:10FB100065480078012855D164480078012803D051
:10FB20005F480078002809D05A4800883721090129
:10FB3000884203DB00205D49087043E05B480078A1
:10FB4000022803D056480078002808D05148008881
:10FB50005749884203DB01205449087032E053487A
:10FB60000078032803D04E480078002809D049487F
:10FB70000088FF21AF31884203DB02204B49087027
:10FB800020E04A480078042803D04548007800283F
:10FB900009D040480088FF211931884203DB032047
:10FBA000424908700EE041480078052803D03C48DF
:10FBB0000078002806D037480088822802DB04201D
:10FBC0003A490870FCF7A4FE3349643988425DD392
:10FBD0003848006800193749086031480078002823
:10FBE00008D000202E490870324908602F4800785C
:10FBF0003149087000F082FD00281FD12D480068AF
:10FC00002E49884239D300202A4908602A480078C2
:10FC100026490978884205DA27480078401C264999
:10FC200008702AE02448007820490978884224DDB9
:10FC300021480078401E204908701EE01D480068D9
:10FC40001F49884219D300201A4908601A480078D1
:10FC500016490978884205DA17480078401C164989
:10FC600008700AE01448007810490978884204DDD9
:10FC700011480078401E104908700F4800780B4961
:10FC80000978884202D100200A49086010BD0000AE
:10FC90000B000020020000201C0C000012000020BD
:10FCA00008000020040000200A00002006000020B8
:10FCB000760200001800002007000020C05D000050
:10FCC000407E050000200B4908700B490870012098
:10FCD0000A4908700A49087000200A4908700A4950
:10FCE00008700A4908800A4908800A4908800A49B8
:10FCF0000870704706000020070000200800002060
:10FD0000090000200A0000200B0000200C00002049
:10FD10000E000020100000201200002000200B49DF
:10FD200008700B49087001200A4908700A490870D8
:10FD300000200A4908700A4908700A4908800A49DF
:10FD400008800A4908800A490870704706000020A8
:10FD50000700002008000020090000200A00002001
:10FD60000B0000200C0000200E00002010000020DE
:10FD700012000020F1B500272D480078002804D09B
:10FD80000320F9F7DFFB2B4908802B48008819284E
:10FD900047D300202849088028480078142829D211
:10FDA0000320F9F7CFFB0746002407E06000244951
:10FDB000085AB84200DD05E0601CC4B21F48007854
:10FDC0008442F3DB00BF1D48057808E0681E400050
:10FDD0001B49085A69001A4A5052681EC5B2A5420A
:10FDE000F4DC600016490F5214480078401C134997
:10FDF000087016E00026052405E060001049085A46
:10FE00008619601CC4B20F2CF7D30A213046F8F7CC
:10FE100097F908490880002008490870012009491D
:10FE20000870054801880098081803490880F8BD43
:10FE30000900002002000020160000200000002021
:10FE4000E4070020120000203A4909881E2928DA18
:10FE50000021394A1180394A118039490988394AC3
:10FE6000914207DC38490978002914D034490988BF
:10FE7000914210DD0121354A11700021344A117080
:10FE8000344A1170304A11700121334A1170002137
:10FE9000324A11704CE02A4909880918284A118011
:10FEA00046E024490988274A643291422BDB00212D
:10FEB000234A1180214A11801F490988AF2212016B
:10FEC000914207DC20490978002916D01A4909888F
:10FED000914212DD02211D4A117000211C4A11704D
:10FEE00005211C4A11700021174A117001211A4A7C
:10FEF00011700021194A11701AE00F490988091878
:10FF00000D4A118014E000210D4A11800A4A118027
:10FF10000A4909880B4A914205DD00210B4A1170FC
:10FF2000094A117004E0054909880918034A11803B
:10FF30007047000002000020100000200C0000208C
:10FF40000E000020B80B0000090000200B0000206C
:10FF50000600002007000020080000200A00002002
:10FF60000148007870470000900900200148007A9D
:10FF70007047000090090020014880787047000019
:10FF80009009002001480088704700007800002098
:10FF9000F8B50023002500950024002200BF94E05E
:10FFA00001259D40ACB20D8825400095009DA542DD
:10FFB0006FD11A468D79012D0DD1464D032636029B
:10FFC000AD192D5C012696403543424E03273F0272
:10FFD000F61935540CE03F4D03263602AD192D5C61
:10FFE00001269640B5433B4E03273F02F619355490
:10FFF000CD78002D4ED1374D60352D5CCE78002E5A
:020000040001F9
:1000000001D1012600E000269640B543314E60360E
:1000100035548D78002D2ED12E4D19267601AD192F
:100020002D5C8E78002E01D1012600E0002696403E
:10003000B543284E19277F01F61935540D79002D47
:100040000ED1244D50352D5C0E79002E01D10126A4
:1000500000E000269640B5431E4E5036355423E04E
:100060001C4D50352D5C0E7996403543EEB2194D3E
:1000700050352E5418E0174D19267601AD192D5C18
:100080008E7896403543134E19277F01F619355463
:100090000AE018E00F4D60352D5CCE789640354370
:1000A000EEB20C4D60352E544D79012D0AD1094D1B
:1000B00030352D5C012696403543EEB2054D303586
:1000C0002E5400E000BF5D1CABB2082B00DA67E7DE
:1000D000F8BD000000000440FFB5074615461E4667
:1000E00000243846019900F01FF8002802D00120B2
:1000F00004B0F0BD00240CE00A2060430949085C0C
:10010000B04204D12946204600F05EF807E0601CAA
:1001100084B20A2060430349085C0028ECD100BF88
:100120000020E5E7AC0100200246002A03D1402967
:1001300001DD01207047032A03D1022901DD0120DE
:10014000F8E7042A03D1202901DD0120F2E7052A7E
:1001500003D1202901DD0120ECE70C2A03D110296D
:1001600001DD0120E6E70D2A05D1012903DD402943
:1001700001DA0120DEE70E2A03D1202901D1012076
:10018000D8E70020D6E7000010B5064A03231B027B
:10019000D218125C8A43034B032424021B191A54FD
:1001A00010BD00000000044010B5064A03231B02E6
:1001B000D218125C0A43034B032424021B191A545D
:1001C00010BD00000000044070B502460020B1E000
:1001D0000A2353435A4C1B195B1C440004191B1976
:1001E0009B788B427DD10A235343554C1B195B1CD2
:1001F000440004191B195B78082B33D10A2353439D
:100200004F4C1B195B1C440004191B574D4C4E4DA1
:100210006419E35C012423430A245443484D6419C0
:10022000641C450045196457464D474EAD192B5582
:100230000A235343424C1B195B1C440004191B57EF
:10024000404C35466419E35C022423430A2454439A
:100250003B4D6419641C450045196457394DAD196F
:100260002B5564E00A235343354C1B195B1C440097
:1002700004191B195B78092B34D10A235343304CE2
:100280001B195B1C440004191B572E4C2E4D64197E
:10029000E35C402423430A245443294D6419641C1D
:1002A000450045196457274D274EAD192B550A2394
:1002B0005343234C1B195B1C440004191B57214C4E
:1002C00035466419E35C8024A3430A2454431C4D3F
:1002D0006419641C4500451964571A4DAD192B5516
:1002E00025E025E00A235343154C1B195B1C4400F1
:1002F00004191B57134C144D6419E35C0A2454432E
:100300000F4D6419641C4500451964196578012472
:10031000AC402343DCB20A235343094D5B195B1CF9
:10032000450045195B57074D074EAD19EC5404E0E5
:10033000431CD8B2032800DA4AE700BF70BD0000B2
:10034000AC0100200000044075080000F8B500244E
:10035000FCF7F8FA012861D100F088FB0446BA22C4
:100360000721002003F0AAF8012C21D100F0A2FC03
:1003700000280ED000F0AEFB054600F09FFB0646BD
:1003800001200346024629460090304605F0CEFB88
:1003900050E000F09FFB054600F090FB0646012070
:1003A0000023024629460090304605F0BFFB41E09D
:1003B000022C21D100F07EFC00280ED000F08AFB38
:1003C000054600F07BFB064601200346024629460F
:1003D0000090304605F0AAFB2CE000F07BFB0546C0
:1003E00000F06CFB0646002001231A4629460090C7
:1003F000304605F09BFB1DE000F05CFC054600F07C
:1004000069FB064600F05AFB0746012003462A46D0
:1004100031460090384605F089FB0BE0002003468A
:1004200002460146009005F081FB0022072110469C
:1004300003F044F8F8BD0000F0B585B0002473481F
:100440000078012824D1FCF77DFA012812D1FCF7AD
:1004500067F800BF0BE0182C02D1601CC4B204E0A6
:10046000BA222146002003F029F8601CC4B2242CD3
:10047000F1DBC8E0FCF79EF9002406E000222146EB
:10048000104603F01BF8601CC4B2242CF6DBBAE063
:10049000FCF758FA01287DD1FCF73AFA5C4988420A
:1004A0007FD35C480088032805DA5A480088401C3E
:1004B0005849088011E000205649088000F004FBEC
:1004C000064600F01FFB07460A21F7F739FE0546EE
:1004D0003246294601200AF0FDFF00F043FD0646A2
:1004E00000F0DCFC0A210390F7F72AFE054600F035
:1004F000EBFA07463246294609F04AF8FFF726FF8D
:1005000000F0A2FA05462946012007F091FB00F011
:10051000F3FA0646FF21F531F7F728FEC5B2294662
:10052000012006F0C1FAFFF71BFD0546FFF72AFD83
:100530000646FFF721FD07462B4632463946012085
:1005400005F0CEFD00F0E0F80546294601200BF04D
:1005500067FA00F0C3FC054600F0BEFB064600F05B
:10056000C5FA074600F0C0FC039000F0BBFB3B4619
:1005700000960195029001460120039A0AF086FD3B
:1005800000F080FC054600F077FC064600F080FC99
:10059000074601E008E004E02A46314607F080FD06
:1005A00031E0FCF737F82EE0FCF704F900222321B4
:1005B000104602F083FF00222221104602F07EFF47
:1005C00000220721104602F079FF00220821104680
:1005D00002F074FF00220921104602F06FFF002292
:1005E0000A21104602F06AFF00221321104602F091
:1005F00065FF00221121104602F060FF0022122147
:10060000104602F05BFF05B0F0BD000001010020C4
:10061000B80B00007200002001490860704700001C
:100620008007002002480068401C014908607047AC
:100630007C070020F3B581B0064600200E49086013
:1006400000F01EF8044600F01BF805462F1B30464C
:10065000029903F0D5FE00900AE000F011F805467B
:100660002F1B06480068002802D004480068804715
:1006700000988742F1D3FEBD7C0700208007002050
:1006800001480068704700007C0700200B4909788A
:10069000012901D101200FE008490978022901D17F
:1006A000022009E005490978032901D1042003E06B
:1006B0000121024A1170012070470000110700203B
:1006C00010B5094B1B8899B20A12C8B2D343313313
:1006D000064C2370C3432333637013465633A37011
:1006E00003467133E37010BD440700201707002054
:1006F0000148008870470000200000200148008861
:100700007047000038000020014800787047000062
:100710007C00002001480078704700007D00002028
:1007200010B5002205210648FAF7F4FC0402012264
:1007300005210348FAF7EEFC201880B210BD000036
:100740002808002010B5062205210348FAF7E2FC2C
:10075000C006C00F10BD00002808002010B50422FC
:1007600005210648FAF7D6FC040205221146034883
:10077000FAF7D0FC201880B210BD00002808002035
:1007800010B5062205210248FAF7C4FCC01110BDBD
:100790002808002010B5022205210248FAF7BAFC09
:1007A00010BD00002808002010B5062205210348CE
:1007B000FAF7B0FC8006C00F10BD0000280800202A
:1007C00010B5042202210348FAF7A4FCC007C00FA9
:1007D00010BD00002808002010B5052202210348A2
:1007E000FAF798FCC007C00F10BD000028080020D1
:1007F00010B5002204210348FAF78CFC4006400F94
:1008000010BD00002808002010B504220121024874
:10081000FAF780FC801110BD2808002010B50022D6
:1008200001210248FAF776FC10BD000028080020DC
:1008300010B5052201210348FAF76CFC8007800FF0
:1008400010BD00002808002010B501221146024802
:10085000FAF760FC10BD00002808002010B5002247
:1008600006210C48FAF756FC040201220621094829
:10087000FAF750FC20180402022206210548FAF774
:1008800049FC20180402032206210248FAF742FC20
:10089000201810BD2808002010B5042206210C489D
:1008A000FAF738FC0402052206210948FAF732FC5F
:1008B00020180402062211460548FAF72BFC2018DE
:1008C0000402072206210248FAF724FC201810BD72
:1008D0002808002010B5022203210248FAF71AFC6A
:1008E00010BD00002808002010B503220021024896
:1008F000FAF710FC10BD00002808002010B50022F7
:1009000011460248FAF706FC10BD00002808002036
:1009100010B5042200210248FAF7FCFB10BD0000CC
:100920002808002010B5012200210248FAF7F2FB46
:1009300010BD00002808002010B505220021024843
:10094000FAF7E8FB10BD000028080020322815DA6D
:100950003C498978012903DD01213A4A517070E050
:1009600038498978002905DD2F286ADC0021354ABD
:10097000517066E00021334A517062E03E2817DA78
:10098000322815DB2F498978022903DD02212D4AFF
:10099000517056E02B498978012905DD3B2850DC50
:1009A0000121284A51704CE00121264A517048E04B
:1009B000502817DA3E2815DB22498978032903DD00
:1009C0000321204A51703CE01E498978022905DD47
:1009D0004D2836DC02211B4A517032E00221194AAF
:1009E00051702EE0622817DA502815DB15498978F6
:1009F000042903DD0421134A517022E0114989784A
:100A0000032905DD5F281CDC03210E4A517018E024
:100A100003210C4A517014E073280FDA62280DDBB1
:100A200008498978042905DD70280ADC0421054A73
:100A3000517006E00421034A517002E00521014A89
:100A400051707047900900200148007870470000FD
:100A50000700002001480068704700005C1F00206C
:100A60000148007870470000ED0000200148007840
:100A700070470000EC000020F8B500260024002597
:100A8000FCF782FE07460A21F7F75AFB054609489C
:100A90000068854200D303E006480068461B3446E0
:100AA0007D200001844200D30446034804600068AE
:100AB000F8BD000028010020240100200148007832
:100AC00070470000F90000200148007970470000DD
:100AD0000C2800200148407870470000F9000020F1
:100AE0000148007A704700000C2800200148407936
:100AF000704700000C280020014800887047000063
:100B00002200002010B50024FFF7DEFF00280AD1E4
:100B10000A4800880A49884202DB084607490880DB
:100B20000648048808E005480088FCF7DBFB84B22F
:100B30000448844200DB0446204610BD3A000020F1
:100B4000C6070000CE040000002005490988054AB8
:100B5000914202DB1146024A118001490888704720
:100B60003A000020C6070000F8B50027002500263F
:100B70000024FFF7C3FE0546FFF7D4FE0646F0202B
:100B8000284000110A2805DBF02028400011C01C75
:100B9000044303E0F0202840001104432402280706
:100BA000000F0A2804DB2807000FC01C044302E0E2
:100BB0002807000F04432402F020304000110A28C7
:100BC00005DBF02030400011C01C044303E0F0209E
:100BD00030400011044324023007000F0A2804DBD0
:100BE0003007000FC01C044302E03007000F04432D
:100BF000002C01D10248F8BD27463846FBE700002B
:100C0000FFFF0000F8B50027002500260024FFF7AD
:100C10007FFE0546FFF790FE0646F02028400011B3
:100C20000A2805DBF02028400011C01C044303E023
:100C3000F02028400011044324022807000F0A284E
:100C400004DB2807000FC01C044302E02807000F44
:100C500004432402F020304000110A2805DBF02074
:100C600030400011C01C044303E0F020304000116C
:100C7000044324023007000F0A2804DB3007000F6A
:100C8000C01C044302E03007000F0443002C01D1D4
:100C90000248F8BD27463846FBE70000FFFF00008A
:100CA00010B50024FFF720FE0446204610BD0120A9
:100CB0007047000001480078704700004D07002091
:100CC00001480078704700004F0700200148807BF2
:100CD00070470000381F00200148007A704700006C
:100CE000381F002070B500240E48C07A01280ED1AC
:100CF0000C490868FBF746FF054632356421284653
:100D0000F7F71EFA84B2632C0ADD632408E0054875
:100D10000088401D84B20A212046F7F727FA84B2E2
:100D2000204670BD381F002070B5002407490868B0
:100D3000FBF728FF05460A21F7F702FA84B20448B8
:100D4000844200DD0446204670BD0000381F0020AC
:100D5000DE03000010B5002400F016F8012801D1D0
:100D600003240CE000F010F8022802D1FF243734ED
:100D700005E00A2103480088F7F7F8F984B2204615
:100D800010BD0000020000200148007870470000FC
:100D90000B00002010B50024044804F097FB002845
:100DA00001D0012400E00024204610BD030700000C
:100DB00010B50024044804F089FB002801D0012468
:100DC00000E00024204610BD0507000010B50024F7
:100DD000044804F07BFB002801D0012400E000243B
:100DE000204610BD0707000010B50024062004F0BF
:100DF0006DFB002801D0012400E00024204610BD36
:100E000010B50024052004F061FB002801D0012466
:100E100000E00024204610BD10B50024044804F072
:100E200055FB002801D0012400E00024204610BD1D
:100E30000607000010B50024044804F047FB002812
:100E400001D0012400E00024204610BD030500006D
:100E500010B50024044804F039FB002801D0012417
:100E600000E00024204610BD040500000148807AFF
:100E700070470000381F002001488078704700004C
:100E80001C0A002001484068704700001C0A00202E
:100E900001484078704700001C0A002070B500240B
:100EA000FFF712FE002803D1FCF76EFC04460DE0AC
:100EB000FFF70AFE012806D1FCF766FC0546FCF7A1
:100EC00011FA044602E0FCF75FFC0446204670BDC0
:100ED0000148C07B70470000381F00200148407A5D
:100EE00070470000381F002070B500240E48C07AFB
:100EF00001280ED10C494868FBF744FE05463235FF
:100F000064212846F7F71CF984B2632C0ADD6324B8
:100F100008E005488088401D84B20A212046F7F782
:100F200025F984B2204670BD381F002070B500241A
:100F300007494868FBF726FE05460A21F7F700F93E
:100F400084B20448844200DD0446204670BD00009F
:100F5000381F0020DE0300000148007870470000C1
:100F6000F000002070B50024FFF7AEFD002803D18B
:100F7000FCF72CFC04460FE0FFF7A6FD012807D183
:100F80000020FCF723FC0546FCF7ACF9044603E01F
:100F90000020FCF71BFC0446204670BD0148007889
:100FA000704700003E00002070B505460024032D68
:100FB00000D170BD002D01D0012D1BD18121032056
:100FC000800204F033FA8021134804F02FFA322112
:100FD0001248FFF72FFB002409E0A200104BD218A3
:100FE0009178A200985A04F021FA601CC4B23B2CFC
:100FF000F3DB0FE0022D0DD1002409E0A200094B24
:10100000D2189178A200985A04F010FA601CC4B269
:101010003B2CF3DB00BFCCE702060000A0860100FA
:10102000280B0200140C0200F8B500210024002354
:10103000002200BF0AE001258D40ABB205881D40AB
:101040002C469C4200D10A464D1CA9B21029F2DB65
:101050000588FF2D1FDC284D6D7E0688B543264E82
:10106000757635462D7E0688B543234E3576354652
:101070006D7E8678F607F60F964035431E4E7576E0
:1010800035462D7E867802273E40760896403543C9
:10109000194E357622E0184DED7E0688B543164E82
:1010A000F5763546AD7E0688B543134EB576857820
:1010B000ED07ED0F1646083EB5400F4EF67E354360
:1010C0000D4EF5768578022635406D081646083EA9
:1010D000B540094EB67E3543074EB57600250095DE
:1010E00005E000BF6D462D786D1CEEB200966D4692
:1010F0002D78012DF5D9F8BD206B0440C107C90F2B
:10110000002905D00021394A1171002238490A719D
:1011100002210140002905D00021344A1172002229
:1011200033490A7204210140002905D000212F4AC9
:10113000117300222E490A7308210140002905D0AD
:1011400000212A4A1174002229490A741021014001
:10115000002905D00021254A1175002224490A756D
:1011600020210140002905D00021204A11760022CB
:101170001F490A7640210140002904D000221B4962
:101180004A711B494A7180210140002904D0002284
:1011900016494A7216494A72FF210131014000295D
:1011A00004D0002211494A7311494A7301214902AE
:1011B0000140002904D000220C494A740C494A74A9
:1011C000012189020140002904D0002207494A7503
:1011D00007494A750121C9020140002904D00022B3
:1011E00002494A7602494A76704700000060004092
:1011F00000610040C107C90F002905D001223C4908
:101200000A7100213B4A117102210140002905D0D9
:10121000012237490A720021364A11720421014025
:10122000002905D0012232490A730021314A117385
:1012300008210140002905D001222D490A7400210E
:101240002C4A117410210140002905D0012228499F
:101250000A750021274A117520210140002905D077
:10126000012223490A760021224A117640210140B9
:10127000002905D001221E494A7100221D494A71E8
:1012800080210140002905D0012219494A7200221B
:1012900018494A72FF2101310140002905D001227D
:1012A00013494A73002213494A730121490201403C
:1012B000002905D001220E494A7400220D494A74C2
:1012C000012189020140002905D0012208494A75FF
:1012D000002208494A750121C9020140002905D0B0
:1012E000012203494A76002202494A7670470000EB
:1012F000006100400060004010B50C4800780028F4
:1013000003D00B4A50689168884708484078002805
:1013100003D0084A506891688847044880780028BC
:1013200003D0054A50689168884710BD00600040AE
:10133000FC0200207C040020FC05002010B50848B9
:101340000079002803D0074A10695169884704488A
:101350004079002803D0044A50689168884710BD3E
:1013600000600040FC0200208804002010B50848FE
:10137000007A002803D0074AD069116A88470448D8
:10138000407A002803D0044A50689168884710BD0D
:1013900000600040FC0200209404002010B50848C2
:1013A000007B002803D0074A906AD16A8847044826
:1013B000407B002803D0044A50689168884710BDDC
:1013C00000600040FC020020A004002010B5084886
:1013D000007C002803D0074A506B916B8847044873
:1013E000407C002803D0044A50689168884710BDAB
:1013F00000600040FC020020AC04002010B508484A
:10140000007D002803D0074A106C516C88470448BF
:10141000407D002803D0044A50689168884710BD79
:1014200000600040FC020020B804002010B508480D
:10143000007E002803D0074AD06C116D884704480D
:10144000407E002803D0044A50689168884710BD48
:1014500000600040FC020020C404002010B50848D1
:10146000407F002803D0074A5068916888470448A5
:10147000007F002803D0044A906DD16D884710BDCD
:1014800000600040D0040020FC02002010B5084895
:101490004078002803D0074A50689168884704487C
:1014A0000078002803D0044A506E916E884710BD22
:1014B00020600040DC040020FC02002010B5094838
:1014C0000079002803D0084A106F516F88470548FB
:1014D000001D4078002803D0044A5068916888476E
:1014E00010BD000020600040FC020020E804002045
:1014F00010B5034AD06F78329168884710BD00005C
:10150000FC02002010B5024A50689168884710BD5F
:101510008003002010B50948007C002803D0084A49
:10152000506891688847054810304078002803D0FB
:10153000044A50689168884710BD00002060004050
:101540008C0300200C05002010B5024A50689168F9
:10155000884710BD9803002010B5024A5068916872
:10156000884710BDA403002010B50948007F00285B
:1015700003D0084A50689168884705481C30407875
:10158000002803D0044A50689168884710BD0000C5
:1015900020600040B00300203005002010B50C484A
:1015A0000078002803D00B4A5068916888470848A3
:1015B0004078002803D0084A50689168884704485A
:1015C0008078002803D0054A50689168884710BD8C
:1015D00040600040BC0300203C050020BC06002009
:1015E00010B50D480079002803D00C4A5068916866
:1015F00088470948001D4078002803D0084A5068F1
:10160000916888470448001D8078002803D0054A67
:1016100050689168884710BD40600040C8030020B2
:1016200048050020C806002010B50D48007A0028A3
:1016300003D00C4A506891688847094808304078C0
:10164000002803D0084A5068916888470448083049
:101650008078002803D0054A50689168884710BDFB
:1016600040600040D403002054050020D406002030
:1016700010B50D48007B002803D00C4A50689168D3
:10168000884709480C304078002803D0084A506841
:101690009168884704480C308078002803D0054AB8
:1016A00050689168884710BD40600040E00300200A
:1016B00060050020E006002010B50D48007C0028E1
:1016C00003D00C4A50689168884709481030407828
:1016D000002803D0084A50689168884704481030B1
:1016E0008078002803D0054A50689168884710BD6B
:1016F00040600040EC0300206C050020EC06002058
:1017000010B5024A50689168884710BDF803002060
:1017100010B50948007E002803D0084A5068916837
:101720008847054818304078002803D0044A50689C
:101730009168884710BD000040600040040400200C
:101740008405002010B50948007F002803D0084A0E
:1017500050689168884705481C304078002803D0BD
:10176000044A50689168884710BD000040600040FE
:10177000100400209005002010B5084800780028CB
:1017800003D0074A50689168884704484078002889
:1017900003D0044A50689168884710BD60600040DB
:1017A0001C0400209C05002010B509480079002881
:1017B00003D0084A5068916888470548001D407862
:1017C000002803D0044A50689168884710BD000083
:1017D0006060004028040020A805002010B50948DA
:1017E000007A002803D0084A506891688847054865
:1017F00008304078002803D0044A50689168884730
:1018000010BD00006060004034040020B4050020DA
:1018100010B5024A50689168884710BD4004002006
:1018200010B5024A50689168884710BD4C040020EA
:1018300010B50948007D002803D0084A5068916817
:101840008847054814304078002803D0044A50687F
:101850009168884710BD0000606000405804002077
:10186000D805002010B50948007E002803D0084A9A
:10187000506891688847054818304078002803D0A0
:10188000044A50689168884710BD000060600040BD
:1018900064040020E405002010B50948007F0028FA
:1018A00003D0084A50689168884705481C30407842
:1018B000002803D0044A50689168884710BD000092
:1018C0006060004070040020F005002010B5FE4864
:1018D00000688079002806D001286ED002286DD0DB
:1018E00003286CD104E2F8480068407903000EF048
:1018F0004DFB0A0614BC2BBC47BC67BC9BBC0AF062
:10190000F1FB0020F0490968C873EF48006840798E
:10191000401CED4909684871AEE0EC490969EA4AA2
:101920001268D27A885C0AF055FCE7480068407972
:10193000401CE54909684871E34800684079401C4B
:10194000E1490968487197E001F020FF002810D1B3
:101950000AF040FCDC4800684079401CDA4909681C
:101960004871D94800684079401CD74909684871D6
:1019700005E00AF0E1FB0020D349096848717BE0EB
:1019800001F004FF002811D101200AF023FCCE4809
:1019900000684079401CCC4909684871CA48006811
:1019A0004079401CC8490968487105E00AF0C4FB49
:1019B0000020C549096848715EE05FE0FEE0A3E1F0
:1019C00001F0E4FE002828D1BF490968C97A242221
:1019D0005143BF4A12688918BB4A1268D27B885C9F
:1019E0000AF0F8FBB8480068C07B401CB64909689B
:1019F000C873B5480068C07B242814D3B248006877
:101A00004079401CB04909684871AF480068407986
:101A1000401CAD490968487105E00AF08DFB0020C3
:101A2000A9490968487127E001F0B0FE002815D1E6
:101A3000A5480068C07A401CA3490968C872A2483A
:101A40000068C07AA1490978884207DB00209E49D6
:101A50000968C87201209C49096888710AF06CFB0A
:101A6000002099490968487106E00AF065FB0020EA
:101A700095490968487100BF00BF4FE1924800686E
:101A8000407903000EF082FA080513912A914791DC
:101A900070910AF027FB00208B490968C8738A48B7
:101AA00000684079401C88490968487184E087498A
:101AB0000969854A1268D27A885C0AF08BFB8248F1
:101AC00000684079401C8049096848717E48006878
:101AD0004079401C7C49096848716DE001F056FE70
:101AE000002811D126200AF075FB7748006840795C
:101AF000401C754909684871734800684079401C6A
:101B000071490968487105E00AF016FB00206E492A
:101B10000968487150E001F039FE00281DD101200C
:101B20000AF058FB68480068C07B401C6649096899
:101B3000C87365480068C07B242814D362480068D5
:101B40004079401C6049096848715F4800684079E5
:101B5000401C5D490968487105E00AF0EDFA002073
:101B600059490968487127E001F010FE002815D195
:101B700055480068C07A401C53490968C8725248E9
:101B80000068C07A51490978884207DB00204E4935
:101B90000968C87202204C49096888710AF0CCFAB9
:101BA000002049490968487106E00AF0C5FA00209A
:101BB00045490968487100BF00BFAFE0424800686E
:101BC000407903000EF0E2F90805138B2A8B478B4E
:101BD000638B0AF087FA00203B490968C8733A48CA
:101BE00000684079401C3849096848717EE03749EF
:101BF0000969354A1268D27A885C0AF0EBFA3248F1
:101C000000684079401C3049096848712E480068D6
:101C10004079401C2C490968487167E001F0B6FD25
:101C2000002811D125200AF0D5FA2748006840790C
:101C3000401C254909684871234800684079401CC8
:101C400021490968487105E00AF076FA00201E492A
:101C5000096848714AE001F099FD002810D10AF0A6
:101C6000B9FA194800684079401C17490968487159
:101C7000154800684079401C13490968487105E01F
:101C80000AF05AFA00201049096848712EE001F064
:101C90007DFD002815D10C480068C07A401C0A4917
:101CA0000968C87208480068C07A084909788842FB
:101CB00007DB002004490968C8720320024909684B
:101CC00088710AF039FA05E0D0070020E82E0020DC
:101CD000CC070020002012490968487106E00AF08C
:101CE0002BFA00200E490968487100BF00BF15E0BB
:101CF00000200B4909688871094909684871062064
:101D000007490968C87009E00AF016FA002004497A
:101D10000968487102490968887100BF00BF10BD99
:101D2000D007002010B56A480068407903000EF023
:101D30002DF9090610C627C644C6608EC6000AF0F3
:101D4000D1F9634800684079401C614909684871CD
:101D5000BCE0604909695E4A1268D27A885C0AF080
:101D600039FA5B4800684079401C59490968487154
:101D7000574800684079401C554909684871A5E0FA
:101D800001F004FD002811D14F200AF023FA504839
:101D900000684079401C4E49096848714C48006809
:101DA0004079401C4A490968487105E00AF0C4F9C5
:101DB000002047490968487188E001F0E7FC0028E5
:101DC00010D10AF007FA424800684079401C4049A7
:101DD000096848713E4800684079401C3C490968E0
:101DE000487105E00AF0A8F90020394909684871EE
:101DF0006CE001F0CBFC002822D135480068C07AA5
:101E0000401C33490968C87231480068C07A3149BA
:101E1000097888420FDB00202D490968C8722C48D8
:101E200000684079401C2A49096848710020284907
:101E30000968486208E0002025490968487103E004
:101E400000202349096848710AF076F93EE02048ED
:101E50000068407C002816D01E48C068002803D0C7
:101E60001C48C16819208847002019490968486240
:101E7000174909684871164909688871052014498D
:101E80000968C8701AE012480068406A282807D21A
:101E90000F480068406A401C0D49096848620DE01F
:101EA00000200B49096848620949096848710849D6
:101EB00009688871052006490968C87006E00AF0BB
:101EC0003BF9002002490968487100BF00BF10BDFE
:101ED000D0070020E82E002010B50024F748006845
:101EE000807A01287ED1F5480068C07900287AD030
:101EF000F24800688079002804D0012874D00228B4
:101F000073D191E1ED480068007B24286ED2EB4844
:101F10000068C07901287AD1002475E0E74800689C
:101F2000C07A24214843E64909684018E349096812
:101F3000097B415CE1480068C07A24225043E14AB1
:101F400012688018DD4A1268127B805C814229D0B9
:101F5000DA480068C07A24214843DA490968401801
:101F6000D6490968097B415CD4480068C07A2422BC
:101F70005043D34A12688018D04A1268127B8154A9
:101F8000CE480068407B242805D3CC480068007BFD
:101F9000CA4909684873C9480068007BC74909688D
:101FA000887308E0C5480068407B242803D20120DC
:101FB000C24909688871C1480068007B401CBF495C
:101FC00009680873BD480068007B242808D3BB4813
:101FD0000068407B242803D20120B8490968887131
:101FE000B64805E0D3E1CDE169E0BAE138E00EE0C2
:101FF0000068007B242804D2B0480068807901285A
:1020000000D103E0601CC4B2242C87D356E0002426
:1020100013E0AA480068C07A24214843A949096806
:102020004018015DA5480068C07A24225043A44AA4
:10203000126880180155601CC4B2242CE9D300201A
:102040009E490968487323209C49096888730120C8
:102050009A490968887124209849096808732DE015
:10206000002096490968087394480068C07A401CAB
:1020700092490968C87291480068C07A9249097803
:10208000884217DB8D480068007C012804D10220BB
:102090008A490968887106E00020884909688871C2
:1020A00086490968C871002084490968C872834953
:1020B00009680874002081490968487161E17F4816
:1020C0000068407903000DF061FF080513A62AA6F9
:1020D00051A68EA601207949096808740AF002F811
:1020E000764800684079401C74490968487199E055
:1020F00075490969714A1268D27A885C0AF06AF8EF
:102100006E4800684079401C6C49096848716B480A
:1021100000684079401C69490968487182E001F013
:1021200035FB00281BD165490968497B491CC8B2A9
:102130000AF050F861480068407B60490968C8733C
:102140005E4800684079401C5C49096848715B48FA
:1021500000684079401C59490968487105E009F058
:10216000EBFF00205549096848715BE001F00EFB68
:1021700000282BD151490968C97A24225143504A79
:10218000126889184D4A1268D27B885C0AF022F8DE
:102190004A480068C07B401C48490968C8734748E2
:1021A0000068C07B45490968897B88421ADD43483D
:1021B00000684079401C4149096848713F480068FF
:1021C0004079401C3D49096848710BE009F0B4FFB3
:1021D0003A480068407B39490968C873002037498C
:1021E000096848711EE001F0D1FA00280CD133498A
:1021F00009688871242031490968C8732F49096822
:1022000048732E490968887309F096FF00202B490E
:102210000968487106E009F08FFF00202749096826
:10222000487100BF00BFACE024480068407903005B
:102230000DF0ACFE08050F8E268E4C8E688E09F0D0
:1022400051FF1E4800684079401C1C4909684871CC
:1022500085E01D490969194A1268D27A885C09F03B
:10226000B9FF164800684079401C14490968487154
:10227000124800684079401C1049096848716EE0B6
:1022800001F084FA002811D1252009F0A3FF0B48A2
:1022900000684079401C094909684871074800688E
:1022A0004079401C05490968487105E009F044FF80
:1022B000002002490968487151E00000D007002061
:1022C000CC070020C8070020E82E002001F05EFAAD
:1022D000002810D109F07EFF644800684079401C56
:1022E000624909684871614800684079401C5F494B
:1022F0000968487105E009F01FFF00205B49096883
:1023000048712CE001F042FA00281AD157480068C1
:10231000C07A401C55490968C87254480068C07AA0
:102320005349097888420CDB002050490968C8727B
:102330004E49096888714D49096848714B490968D7
:10234000C87109F0F9FE002048490968487106E0A3
:1023500009F0F2FE002045490968487100BF00BF3E
:102360000FE009F0E9FE00204049096848713F4943
:10237000096888713D49096808733C490968C87251
:1023800000BF71E000203949096888726CE0374865
:102390000068807A022867D134480068007A0028F3
:1023A0005ED0324800684079002804D001280CD063
:1023B000032846D11BE009F095FE2C4800684079BF
:1023C000401C2A490968487149E0002009F002FFD1
:1023D000264800684079401C244909684871234810
:1023E00000684079401C21490968487137E009F0CC
:1023F00043FE002812D11D4800684078401C1B494C
:1024000009684870194800684078032812D301F021
:102410005DFA00201549096848700BE00020134957
:1024200009680872AA2011490968887000200F49BC
:102430000968487009F080FE00200C49096848715D
:102440000DE009F079FE0020084909684871074944
:1024500009684870AA2005490968887000BF03E030
:10246000002002490968887210BD0000D0070020D2
:10247000E82E0020F8B504460D4600260C206043E7
:102480001D49085C002801D00120F8BD0C206043E4
:102490001949401885600C20604340188068002866
:1024A00001D10120F1E701210C206043124A1154AF
:1024B00000222046E317DB0E1B185B115B01E31AB9
:1024C0009B000E4FDB19E717FF0E3F197F11DA55FE
:1024D0000DF08EFD00222046E317DB0E1B185B116A
:1024E0005B01E31A9F00064BFB18E717FF0E3F192D
:1024F0007F11DA553046C8E7FC020020006000403A
:102500000061004000BFFEE709480088401C084900
:102510000880084600880749884208DD0648007898
:10252000002804D0084602490880012088707047BE
:10253000E8000020DC050000EC00002010B5154884
:102540008078012824D11448007801280CD1134840
:102550000078012808D1002011498870084602F04F
:1025600083FD00200D4908700B48007802280CD12B
:102570000C480078012808D10020094988700846D5
:1025800002F072FD0020074908700020024908701F
:1025900010BD0000E8000020EC000020EE0000204C
:1025A000F9000020EF0000207047000010B500F097
:1025B00077FE012803D1002001490880887010BDF2
:1025C000E8000020F0B505460E46174600243A46BE
:1025D0003146284600F072FE00BF42E00020210193
:1025E000394A126850522101374A126889184880C6
:1025F00000212001344A1268801881802001324A6B
:1026000012688018C18020012F4A12688018017258
:1026100020012D4A12688018417220012A4A12684E
:10262000801881722001284A12688018C172002027
:102630002101254A12688918087300212001224AC5
:10264000126880184173002021011F4A12688918FE
:102650008873002120011C4A12688018C173601C15
:10266000C4B21A484078A042B8DC6420184909680E
:1026700008807D20C0001649096848801548144923
:10268000096888807D20000111490968C8801049C7
:102690000968088110480E49096848810F480C49AB
:1026A0000968888140000A490968C88132200849C0
:1026B00009680882FF20F530054909684882044905
:1026C00009688882F0BD0000900700208407002080
:1026D0008C0700204C04000010270000307500001B
:1026E00038B5002404E0002013490855601C84B26A
:1026F000282CF8D301216846417001706A460F49C1
:102700000D48FFF75FFF7D21C900322000F0C6F9B8
:102710000B490C4800F0E0F90948643000F072F908
:102720000748C83000F07EF9074800F091F90748E3
:1027300000F0A4F938BD00001C280020E0100200C1
:1027400028230000B80B00005424000010270000CC
:1027500010B528480078002803D1012025490870C9
:1027600046E024480078012810D123480078012849
:1027700008D1002021498870084602F075FC00202D
:102780001D49087002201B49087031E01948007883
:10279000022810D11A480078012808D100201749D2
:1027A0008870084602F060FC00201549087003207C
:1027B000104908701CE00F480078032803D104205A
:1027C0000C49087014E00B480078042803D1052058
:1027D000084908700CE007480078052803D0054830
:1027E0000078062804D100200249087005490870C5
:1027F00010BD0000EC000020EE000020F9000020D9
:10280000EF000020F0000020F8B50024002500268D
:102810003E48007800281ED13D480078002803D1AA
:1028200001203B49087016E039480078012803D19F
:102830000220374908700EE035480078022803D19D
:1028400003203349087006E031480078032802D19C
:1028500000202F4908702D48007801280ED101244E
:10286000172500262B480123324629460090204692
:1028700001F01AFE01202849087046E0234800783C
:1028800002280FD101243B2500262248401C0123A9
:10289000324629460090204601F006FE01201F49DD
:1028A000087032E01948007803280DD1FEF70CF9C2
:1028B000002803D101201A49087102E000201849BC
:1028C00008710DF035FB20E01048007804280DD188
:1028D000FEF70CF9002803D101201149487102E0EC
:1028E00000200F4948710DF023FB0EE007480078E7
:1028F000052803D106200549087006E00348007842
:10290000062802D1052001490870F8BDEC0000201E
:10291000ED000020F9000020EE000020EF00002074
:102920000C28002010B5044623000DF02FFB095B96
:10293000060E16171819595A5E00F9F7E9FF2C49C7
:10294000884201D3FFF760FF50E0F9F7E1FF284923
:10295000884201D3FFF7FCFE48E047E046E045E04F
:10296000F9F7D6FF2249884239D301F057FD2148B3
:102970000078032814D120480078002810D1FEF7F1
:10298000AFF8002806D101201C4988608868FAF752
:1029900083FF05E00020194988608868FAF77CFF0A
:1029A00014480078012805D113480078002801D187
:1029B000FAF740F910480078052803D101201049A2
:1029C00008700AE00C480078062803D102200C4960
:1029D000087002E000200A4908700BF085F805E055
:1029E00004E003E0FFF790FD00E000BF00BF10BD72
:1029F000B80B0000ED000020EC0000200C280020A7
:102A0000F000002001460020054A126852898A42DF
:102A100001DC012002E0024A1268118170470000C7
:102A20008C07002001460020084A126812898A4259
:102A300001DB012009E0054A126892898A4201DC23
:102A4000012002E0014A1268518170478C07002082
:102A500001460020084A126852898A4201DB01209F
:102A600009E0054A1268D2898A4201DC012002E0AD
:102A7000014A1268918170478C07002001460020AE
:102A8000054A126892898A4201DB012002E0024A6B
:102A90001268D181704700008C0700200246002098
:102AA0000C4B1B681B8A934201DD012010E08A4217
:102AB00001DB01200CE0074B1B689B888B4201DC8B
:102AC000012005E0034B1B681A80024B1B685980EC
:102AD000704700008C070020024600200C4B1B684A
:102AE0001B8A934201DD012010E08A4201DB0120B4
:102AF0000CE0074B1B685B88934201DB012005E07B
:102B0000034B1B689A80024B1B68D98070470000FA
:102B10008C07002070B5044600250C206043FE4958
:102B2000096840184068002807D00C216143FA4A20
:102B3000126889184868804705460C206043F649AA
:102B40000968085C002873D10C206043F2490968C9
:102B500040188068002874D02001F04909684018A6
:102B6000C07A02280AD1032D08D10C206043EA4A1A
:102B70001268801881680120884762E02001E749D7
:102B800009684018C07A02280AD1042D08D10C2007
:102B90006043E14A1268801881680220884750E04B
:102BA0002001DE4909684018C07A02280AD1052DA3
:102BB00008D10C206043D84A12688018816803202D
:102BC00088473EE02001D54909684018C07A0228AC
:102BD0000AD1062D08D10C206043CF4A1268801814
:102BE0008168042088472CE02001CC4909684018FE
:102BF000C07A02280AD1072D08D10C206043C64AAA
:102C0000126880188168052088471AE02001C349AE
:102C100009684018C07A02280BD1082D09D10C2070
:102C20006043BD4A1268801881680620884708E022
:102C30000DE00C206043B84A1268801881680020BB
:102C400088472001B54909684018C5720CE30C207B
:102C50006043B1490968085C012873D10C206043C6
:102C6000AD49096840188068002874D02001AB493C
:102C700009684018C07A03280AD1022D08D10C2017
:102C80006043A54A1268801881680120884762E085
:102C90002001A24909684018C07A04280AD1022DEF
:102CA00008D10C2060439C4A126880188168022079
:102CB000884750E02001994909684018C07A0528E2
:102CC0000AD1022D08D10C206043934A1268801863
:102CD0008168032088473EE0200190490968401838
:102CE000C07A06280AD1022D08D10C2060438A4AF6
:102CF000126880188168042088472CE020018749E9
:102D000009684018C07A07280AD1022D08D10C2082
:102D10006043814A126880188168052088471AE05C
:102D200020017E4909684018C07A08280BD1022D7D
:102D300009D10C206043784A126880188168062007
:102D4000884708E00DE00C206043734A1268801841
:102D50008168002088472001704909684018C572C1
:102D600082E20C2060436C490968085C0228F7D1B4
:102D7000002D7DD1200169490968085A6849096810
:102D8000098A884275DA200164490968085A0A30BC
:102D900081B22001614A1268115220015F4909681D
:102DA000085A5F490968098A884231DB20015B497A
:102DB0000968401840885A4909680988884227DB11
:102DC00020015649096840184088554909684988D2
:102DD00088421DDC00202101504A12688918488071
:102DE00020014E4909684018807A0028B8D10C208B
:102DF000604349490968401880680028B0D00C2019
:102E00006043454A126880188168012088472BE298
:102E1000200142490968085A41490968098A8842DB
:102E20009EDB20013D490968401840883C490968FB
:102E30008988884294DB2001384909684018408815
:102E400037490968C98888428ADC00202101334A51
:102E50001268891848802001304909684018807A32
:102E60000028D4D10C2060432B490968401801E0A8
:102E700063E00BE080680028C9D00C206043264A3C
:102E800012688018816802208847EDE10020210146
:102E9000224A1268891848802101204A126889183C
:102EA000C872002120011D4A12688018C1802001CB
:102EB0001A4A1268801841722001184A1268801854
:102EC0008172184801782001144A12688018017232
:102ED00000202101114A12688918888021010F4AB7
:102EE00012688918087321010C4A126889184873FE
:102EF00021010A4A12688918887300212001074AB3
:102F000012688018C1730C20604303490968401897
:102F100080680028B9D007E08807002090070020CB
:102F20008C070020840700200C206043CF4A1268E1
:102F3000801881680020884796E1012DA5D12001E5
:102F4000CB4909684018C07AA84225D00021200149
:102F5000C74A12688018418000202101C44A1268C3
:102F60008918C8802001C24909684018C572C14843
:102F700000782101BE4A1268891848720020210198
:102F8000BB4A126889188880BA4801782001B84A7B
:102F900012688018017267E12001B549096840187C
:102FA000007AB4490978884220D0B24800782101DB
:102FB000AF4A1268891808722001AD4909684018A3
:102FC000407AAC490978884209D02001A8490968AB
:102FD000401880882101A64A12688918C8800021FB
:102FE0002001A34A12688018818012E02001A049C4
:102FF000096840188088A04988420AD220019C496B
:103000000968401880880A302101994A1268891895
:10301000888020019649096840184088964988426E
:103020000AD2200192490968401840880A302101DB
:103030008F4A12688918488020018D490968401814
:10304000407A8C490978884205D001202101884ABC
:1030500012688918887220018549096840184088DB
:10306000864909680988884204DB00212001804ADA
:103070001268115220017E4909684018807A0028A0
:103080007ED10C2060437949096840188068002887
:1030900077D0200176490968401840887749096847
:1030A0000989884214DB2001714909684018007BB6
:1030B00000280DD10C2060436C4A1268801881688A
:1030C0000320884701202101694A12688918087382
:1030D000200167490968401840886849096849899A
:1030E000884214DB2001624909684018407B0028AF
:1030F0000DD10C2060435D4A12688018816804205D
:103100008847012021015A4A126889184873200112
:103110005749096840184088584909688989884290
:1031200014DB2001524909684018807B00280DD12A
:103130000C2060434D4A126880188168052088473A
:10314000012021014A4A12688918887320014849E0
:1031500009684018408849490968C989884210DBD4
:103160002001434909684018C07B00287CD10C200D
:1031700060433E4A1268801881680620884701E053
:1031800007E03BE001202101394A12688918C87321
:103190006AE02001364909684018407A01282ED19A
:1031A0003448007802282AD12001314909684018A2
:1031B000C08832490968498A884255DB20012C4978
:1031C0000968401880882D490968898A88424BDB44
:1031D0000C2060432549096840188068002843D0C6
:1031E0000C206043214A12688018816807208847B4
:1031F000002021011E4A12688918487234E020011B
:103200001B4909684018407A02282DD119480078D6
:10321000012829D12001164909684018C08817499A
:103220000968898A88421FDB200111490968401812
:10323000808812490968498A884215DB0C2060435E
:103240000A4909684018806800280DD00C206043A6
:10325000064A1268801881680820884700202101EA
:10326000034A12688918487270BD00008807002060
:103270009007002084070020F0FF00008C0700204A
:1032800010B5002400BF04E02046FFF743FC601C9B
:10329000C4B202484078A042F6DC10BD840700208A
:1032A00010B50024044802F011F9002800D000E015
:1032B0000124204610BD00000304000010B5074B98
:1032C00014781C7054785C70054B1960054B1860BD
:1032D00003461833044C236010BD0000840700200F
:1032E000880700208C0700209007002010B50446B6
:1032F000012C09D1BA220C21002000F0DFF80121B5
:10330000022004F007FE08E000220C21104600F025
:10331000D5F80021022004F0FDFD10BD10B50024F9
:1033200004210848F7F708FF552801D1012407E0D8
:10333000042000F0E5FF002801D0002400E0012473
:10334000204610BD2808002010B50446012C09D1E4
:10335000BA221C21002000F0B1F80121062004F05F
:10336000D9FD08E000221C21104600F0A7F800213A
:10337000062004F0CFFD10BD10B50024062000F09B
:10338000BFFF002801D0012400E00024204610BD2A
:1033900010B50446012C09D1BA221721002000F0F3
:1033A0008DF80121042004F0B5FD08E0002217216A
:1033B000104600F083F80021042004F0ABFD10BD9E
:1033C00000200449097A002901D0012000E00020F2
:1033D000704700001C0A002010B50446022C1CD1C6
:1033E00000220D21104600F069F8FDF763FC00286B
:1033F00009D0BA220B21002000F060F801210D2035
:1034000004F088FD47E000220B21104600F056F83A
:1034100000210D2004F07EFD3DE0032C1CD1002294
:103420000B21104600F04AF8FDF744FC002809D0B3
:10343000BA220D21002000F041F801210D2004F0F6
:1034400069FD28E000220D21104600F037F8002128
:103450000D2004F05FFD1EE0012C0ED1BA220D21DB
:10346000002000F02BF800220B21104600F026F877
:1034700001210D2004F04EFD0DE000220D2110462B
:1034800000F01CF800220B21104600F017F8002174
:103490000D2004F03FFD10BD10B50024FCF766FDC3
:1034A000022801D1022406E0FCF760FD012801D1C9
:1034B000032400E00124204610BD000010B5064B97
:1034C0001B78834207DD242905D224234343034C80
:1034D00024681B195A5410BDE82E0020C80700208C
:1034E00010B574480068407903000CF04FFD0B07DD
:1034F00011D325D35A6D77D38DA8D30008F0F2FDF0
:103500006C4800684079401C6A4909684871CFE0FE
:1035100069494969087808F05DFE664800684079A5
:10352000401C644909684871624800684079401C41
:10353000604909684871BBE000F028F9002811D102
:103540007F2008F047FE5B4800684079401C5949DD
:1035500009684871574800684079401C5549096816
:1035600048711DE0534800684078401C5149096883
:10357000487050480068407803280BD300204D491C
:1035800009684870AA204B49096888700320494996
:103590000968C87008F0D0FD0020464909684871E4
:1035A00086E000F0F3F8002807D14248006840792F
:1035B000401C40490968487103E000203D49096802
:1035C000487108F0B9FD73E008F08CFD39480068D7
:1035D0004079401C37490968487169E036494969B2
:1035E0000978491CC8B208F0F5FD324800684079F6
:1035F000401C3049096848712E4800684079401CD9
:103600002C490968487153E000F0C0F800280FD138
:1036100008F03AFD274909688870012008F0AEFDDE
:10362000244800684079401C22490968487105E037
:1036300008F082FD00201F490968487138E01D48E4
:103640000068807818280CD102201A49096808708F
:103650000020184909684870042016490968C87094
:1036600011E0144800684078401C1249096848700D
:10367000104800684078032805D300F027F900209F
:103680000C490968487008F057FD0020094909688D
:1036900048710DE008F050FD0020064909684871A6
:1036A000044909684870AA2002490968887000BF67
:1036B00000BF10BDD0070020E82E002010B5314813
:1036C00000684079002804D001280CD0032848D194
:1036D0001DE008F007FD2B4800684079401C29498F
:1036E000096848714BE028490969087808F072FDBB
:1036F000244800684079401C2249096848712148E3
:1037000000684079401C1F490968487137E000F0A3
:103710003DF800280CD101201A49096808700020E2
:10372000184909684870042016490968C87011E0F2
:10373000144800684078401C1249096848701148D4
:1037400000684078032805D300F0C0F800200D4938
:103750000968487008F0F0FC00200A4909684871BF
:103760000DE008F0E9FC00200649096848710549A8
:1037700009684870AA2003490968887000BF00BF23
:1037800010BD0000D0070020E82E002010B508F082
:1037900073FC04461F4800680078002838D01D4894
:1037A0000068C078042833D3002C09D100211948BF
:1037B0000068C07A8200174800681430815027E002
:1037C00014480068C07A81001248006814304058DC
:1037D0001149884211D20F480068C07A81000D4813
:1037E000006814304058401C0A490968C97A8A00A8
:1037F00008490968143188500AE000F067F8002190
:1038000004480068C07A8200024800681430815081
:10381000204610BDD0070020B80B000000B587B0CF
:10382000012069460871084802900848039008483A
:103830000490084805900848069001A9074800F040
:103840000FF807B000BD0000853B0100B95601002C
:10385000190102004D1102004C11020084280020C1
:10386000F8B506460F46002400253946304600F0DC
:10387000EFF900BF14E000250EE000212420604392
:103880000B4A12688018415524206043094A126887
:1038900080184155681CC5B2242DEED3601CC4B2FB
:1038A00005480078A042E6DC00F010F8F8BD000002
:1038B000C8070020CC070020E82E00200120024984
:1038C0000968087170470000D007002010B500F0AB
:1038D00073F9002003490968087002490968C87033
:1038E00010BD0000D007002007480068C0780628F7
:1038F00008D105480068C079002803D10120024999
:103900000968C87170470000D007002010B55548FD
:103910000068C07803000CF039FB08671D1A171403
:10392000110E056650484068002803D04E48416893
:103930000020884793E000F0E5F890E000F0C6F83A
:103940008DE000F0D1F88AE0FFF7B8FE87E0FFF7DE
:10395000C7FD84E044484068002803D042484168DD
:10396000012088473F480068407C00281AD03E4824
:10397000C068002803D03C48C168C82088470020A0
:10398000384909684862374800680078002804D040
:10399000042034490968C87024E0022031490968CC
:1039A000C8701FE02F480068406A401C2D49096814
:1039B00048622C480068406A7D21C900884211D3C2
:1039C00000202849096848622648006800780028D5
:1039D00004D0042023490968C87003E0022021496B
:1039E0000968C8703BE000BF1F484068002803D04A
:1039F0001D484168002088471A480068407C00281C
:103A000013D01948C068002803D01748C168C820DF
:103A10008847002013490968486212480068C07846
:103A2000401C10490968C87018E00E480068406AD8
:103A3000401C0C49096848620A480068406A7D21B8
:103A4000C90088420AD3002006490968486205482F
:103A50000068C078401C03490968C87000BF00BFF7
:103A600010BD0000D0070020E82E002010B515483A
:103A70000068C078072824D00120124909684874DA
:103A800008E011488068002802D00F498868804704
:103A9000FFF73CFF0B480068C0780628F1D10948C1
:103AA0000068007A0028ECD106480068C079002838
:103AB000E7D104480068807A0028E2D1014909680A
:103AC000487410BDD0070020E82E002010B505482E
:103AD00000680078012802D1FDF7F8FE01E0F5F753
:103AE00007FE10BDD007002010B50548006800781B
:103AF000012802D1FEF716F901E0F6F7D7F910BD5B
:103B0000D007002010B51D480068807A002829D110
:103B10001A480068007A002803D002201749096873
:103B2000887216480068C079002803D00120134924
:103B300009688872114800680079012812D10020B4
:103B40000E49096808710D490968887207200B49F8
:103B50000968C8700A484068002803D008484168CE
:103B600000208847054800680078012802D1FEF748
:103B7000B3F901E0F6F774FA10BD0000D007002099
:103B8000E82E002010B504462146084801F0BAFC92
:103B900007480078002805D1002C03D032210548C1
:103BA000FCF748FD0248047010BD0000010300004E
:103BB0000201002050C30000002024490968487019
:103BC000AA202249096888700020204909684862B3
:103BD0001E49096808711D49096848711B4909682F
:103BE00088711A490968C871184909680872174923
:103BF0000968887215490968C87214490968087308
:103C000024201249096848731049096888730F49CC
:103C10000968C87300200D49096808740B490968D0
:103C200048740A490968887408490968C8740749CA
:103C300009684861002105480068816103480068FF
:103C4000C16102480068016270470000D00700208F
:103C500010B50A780D4B1860034628330C4C2360CE
:103C600024235343044628341B190A4C23600A4C6E
:103C70004B6863608B68A360CB68E3604B696361EA
:103C80000B6923610B78237010BD0000D007002062
:103C9000C8070020CC070020E82E00200748006855
:103CA000C078062808D105480068007A002803D1AA
:103CB000012002490968087270470000D0070020FF
:103CC00010B50446012C09D1BA2220210020FFF7AB
:103CD000F5FB0121084604F01DF908E0002220212F
:103CE0001046FFF7EBFB0021012004F013F910BD93
:103CF00010B50024032000F003FB002801D00124AC
:103D000000E00024204610BD10B50446032C0ED15F
:103D1000BA2215210020FFF7D1FB00221421104602
:103D2000FFF7CCFB01210E2004F0F4F839E0022C5F
:103D30001CD1FCF7BFFF002809D0BA2214210020B3
:103D4000FFF7BCFB01210E2004F0E4F808E000229C
:103D500014211046FFF7B2FB00210E2004F0DAF820
:103D6000002215211046FFF7A9FB1AE0012C0ED105
:103D7000BA2214210020FFF7A1FB01210E2004F03C
:103D8000C9F8002215211046FFF798FB09E0002230
:103D900015211046FFF792FB002214211046FFF771
:103DA0008DFB10BD10B50024F8F7B2FD094988421B
:103DB0000DD3FCF7E9FF002807D1FCF745FE0128E9
:103DC00001DD032404E0022402E0022400E00124D7
:103DD000204610BDB80B000010B50446012C09D1D7
:103DE000BA221D210020FFF769FB0121002004F009
:103DF00091F808E000221D211046FFF75FFB00212B
:103E0000084604F087F810BD10B50024022000F029
:103E100077FA002801D0012400E00024204610BDDC
:103E200010B50446012C09D1BA221E210020FFF74B
:103E300045FB0121092004F06DF808E000221E2155
:103E40001046FFF73BFB0021092004F063F810BD8A
:103E500070B5002400250026FCF7B2FC0546FCF7EF
:103E6000BBFC064602210848F7F766F9552800D141
:103E700008E0012E01D1002404E0012D01D101242C
:103E800000E00024204670BD2808002010B504463C
:103E9000012C09D1BA221F210020FFF70FFB0121BD
:103EA000082004F037F808E000221F211046FFF731
:103EB00005FB0021082004F02DF810BD70B500248A
:103EC0000025FCF707FD054603211A48F7F734F9EA
:103ED000552806D10120184908800020174908807C
:103EE00023E016480088012811D114490880FCF706
:103EF0000BFC762803DA01200F49088015E0FCF757
:103F000003FC782811DB00200B4908800DE001201C
:103F10000A490880FCF7F8FB762803DA01200649F5
:103F2000088002E0002004490880034804882046F5
:103F300070BD000028080020200100202201002080
:103F400010B50446012C09D1BA2221210020FFF727
:103F5000B5FA0121072003F0DDFF08E0002221214E
:103F60001046FFF7ABFA0021072003F0D3FF10BD86
:103F700010B50024FCF780FD002801D1012400E0E9
:103F80000024204610BD10B50446012C09D1BA22E8
:103F900016210020FFF792FA0121032003F0BAFF57
:103FA00008E0002216211046FFF788FA00210320BE
:103FB00003F0B0FF10BD10B50024052000F0A0F9FB
:103FC000002801D0012400E00024204610BD10B5D7
:103FD0000446012C09D1BA2219210020FFF76EFAFC
:103FE0000121052003F096FF3CE0022C17D1FCF7DD
:103FF00061FE002809D0BA2219210020FFF75EFADD
:104000000121052003F086FF2CE000221921104633
:10401000FFF754FA0021052003F07CFF22E0032C77
:1040200017D1FCF74DFE002809D0BA221921002033
:10403000FFF744FA0121052003F06CFF12E0002293
:1040400019211046FFF73AFA0021052003F062FF1C
:1040500008E0002219211046FFF730FA0021052060
:1040600003F058FF10BD000010B50024FCF738FD28
:1040700001282FD104211948F7F75EF8552801D1FE
:10408000012428E0FCF7B4FB01280BD0FCF7B0FBBF
:10409000022807D0FCF7ACFB032803D0FCF7A8FBF1
:1040A000052801D1012416E0FCF7A2FB042801D168
:1040B000022410E0FCF79CFB062801D103240AE04F
:1040C000FCF796FB002803D0FCF792FB072802D1EF
:1040D000002400E00024204610BD00002808002035
:1040E00010B50446012C0ED1BA221B210020FFF787
:1040F000E5F900221A211046FFF7E0F901210A2014
:1041000003F008FF1EE0022C0ED1BA221A21002073
:10411000FFF7D4F900221B211046FFF7CFF9012148
:104120000A2003F0F7FE0DE000221A211046FFF7E7
:10413000C5F900221B211046FFF7C0F900210A2013
:1041400003F0E8FE10BD10B50024FCF78FFE012837
:1041500001D1012400E00224204610BD10B5F8F77B
:10416000F1FB0446204610BD10B5034B082203495D
:10417000034800F013F910BD5D410100EC1002008E
:104180004428002070B506465C488068002804D0AA
:104190005A4988688047054600E000250024A6E0CB
:1041A000564841680C20604308184088A84207D050
:1041B000524841680C2060430818408802287DD18D
:1041C0004E4841680C2060430818806800280CD0D5
:1041D0004A494A680C216143511888688047474919
:1041E0000968E2008918487009E0444841680C20D9
:1041F0006043095C41480068E200801841703F4814
:104200000068E100401840783C490968E200895C98
:1042100088420FD039480068E1004018417837489B
:104220000068E2008154002034490968E2008918DE
:1042300048605AE031480068E100401841782F4852
:1042400042680C2060431018407881421FD12B48EF
:104250000068E10040184168284842680C2060432B
:104260001018808881420BD824480068E10040186B
:104270004068801921490968E2008918486034E0E3
:1042800001201E490968E200891848802DE01B487A
:104290000068E10040184168184842680C206043FB
:1042A0001018C08881420DD814480068E1004018F9
:1042B0004068811911480068E20000E009E08018B8
:1042C000416012E000200D490968E2008918488029
:1042D0000BE0002009490968E200891848800021A4
:1042E00006480068E20080184160601C84B2034800
:1042F0008089A04200DD53E770BD0000A02E0020A1
:104300000146064A92898A4205DD044A1268CB00BA
:10431000D218508800E0002070470000A02E002036
:10432000002000BF14E00D494A680C214143511898
:10433000498801290AD10021084A1268C300D2180D
:104340005180064A1268C300D2185160411C88B2DD
:10435000024989898142E6DC70470000A02E0020D6
:10436000002000BF13E00C494A680C21414351185A
:104370004988002909D1084A1268C300D21851801F
:10438000054A1268C300D2185160411C88B2024924
:1043900089898142E7DC7047A02E0020F0B50446F1
:1043A0000020164DAB6069602C60AA8100BF1FE041
:1043B000124D6E680C254543755D104E3668C7007A
:1043C000F61975700D4D6E680C254543755D0B4EE5
:1043D0003668C700F5550025084E3668C700F6193F
:1043E0007580064E3668C700F6197560451CA8B280
:1043F000024DAD898542DBDCF0BD0000A02E00201F
:1044000070B505460E46002E05D031462846F3F716
:1044100097FE044600E02C46204670BD10B5FCF720
:104420002BFB00280DD107480078012809D005484A
:104430000078032805D004480078002801D1F8F757
:104440005DFF10BDED000020EC00002008B500204D
:104450000090012269460520F9F7B4FD054900984E
:1044600088600020044908700449087004490870F5
:1044700008BD00000C280020EC000020EE00002009
:10448000EF00002008B500200090012269460520B9
:10449000F9F798FD00200349087148710098886079
:1044A00008BD00000C28002070B5049C25789142BE
:1044B00016DD01280AD18D4206DAFF26F61AAE4231
:1044C0000ED3EE18F5B20BE0154609E0022807D12D
:1044D000954204DD9D4203DBEE1AF5B200E00D4685
:1044E000257070BD0D4A4168516081699161C16854
:1044F000D160416A5162016A1162016811604169CB
:10450000516181689160C169D16101691161816AFC
:1045100091620021024A117070470000BC2E0020F9
:10452000C407002010B5FFF7FBFEF8F75DF8002187
:104530000148F6F701FF10BD3408002010B5F8F768
:1045400053F8FFF70DFF09F011FD09F0ADFDFBF782
:10455000B9FBFAF7E7F8FFF779FFF8F773FCF6F71E
:10456000F1FCF9F7A5F955210448F6F7E5FEF8F74F
:10457000A1FAF9F71BF9FBF761F810BD3408002028
:104580001CB500203149087007F05CFD0020FCF7E5
:104590000BFD0CF023F8F7F7CDF955212C48F6F771
:1045A000CBFEF8F787FAF9F701F9F6F7C3F8F6F753
:1045B00041FBE12040020BF053FC00F069FAF6F7F2
:1045C000C1FC07F01DFFF8F70FF8F9F7A9FEF8F79F
:1045D000C5FCF8F743FCFFF7C7FDFEF781F8FFF7CE
:1045E0001DF9FFF743FAF9F78DFDFBF797FBFAF793
:1045F00099F8184AFF219131012009F021FE00228B
:104600001146012009F060FD09F096FC09F04CFD0F
:10461000FFF738FFF9F76EF900200F4988714871EC
:1046200008710120887048701420087007226846BD
:10463000F3F71DFE0199009800F0B4FF022101205C
:1046400000F08CFEFAF7FAFF1CBD0000010100200B
:10465000340800200090D0031201002070470000B1
:1046600010B50446552C03D105494869804702E03E
:1046700003490868804700200249087010BD000007
:10468000BC2E0020C407002010B546480078030067
:104690000BF07CFC0A06111B26303B4650517381FF
:1046A00041484068002802D03F49486880470120BF
:1046B0003C49087000BF3C488068002804D03A4953
:1046C000886880473749087069E03748C068002823
:1046D00002D03549C868804703203249087000BFBE
:1046E00031480069002804D02F49086980472D49C6
:1046F000087054E02C484069002802D02A494869D3
:10470000804700202749087049E027488069002831
:1047100002D025498869804706202249087000BFD9
:104720002148C069002804D01F49C86980471D4935
:10473000087034E000BF1B48007807280AD11A48E7
:10474000006A002802D01849086A804709201549E4
:10475000087011E01348007808280AD11248406A0E
:10476000002802D01049486A804709200D49087086
:1047700002E000200B49087000BF0A4800780028BA
:1047800008D00948806A002804D00749886A804711
:104790000449087003E000200249087000BF00BF10
:1047A00010BD0000C4070020BC2E00207047000090
:1047B00010B500200BF0CEFF08F0E8FC08F03CFD3F
:1047C00008F052FD00F0BEFCF6F7C4FA0220FCF738
:1047D000EBFB002007490870FFF748F9FFF76EF878
:1047E000FFF794F8F6F716F910200AF03FF900F0F9
:1047F000A9FD10BD9801002010B5012408F0A8F80B
:10480000012801D1052407E0F8F77CF80349884224
:1048100001D2012400E00224204610BD204E0000F9
:1048200010B5062408F094F8002800D1002408F000
:1048300095F8012803D008F091F8072800D9092439
:10484000204610BD10B5F6F785FA0022114601206A
:1048500009F06CFD00213B48F6F76EFD002400BF17
:1048600000F02AFF32217D200001FBF7E3FE00204B
:10487000354908700AE00022334801781046FEF7F7
:104880001DFE31480078401C2F4908702E480078E2
:104890002428F0DB00202D49087009E000212B4876
:1048A000007809F051F929480078401C2749087020
:1048B000264800780D28F1DBFFF728F8F5F780FF90
:1048C00007F098FF22480078401C214908700846EC
:1048D0000078052812D300200870FFF705F81D485E
:1048E00000780A2805D300201A490870FFF7D6F986
:1048F00004E018480078401C1649087008F02EF8AB
:104900000128ADD908F02AF80728A9D200200F49BC
:10491000087008E00D48007809F030F90B4800787D
:10492000401C0A490870094800780D28F2DBF6F7A8
:1049300081F955210348F6F7FFFCF7F7B9FF204648
:1049400010BD0000340800201B01002019010020C8
:104950001A0100201C01002010B5032408E000F01B
:10496000ABFE012000F0B2FD002801D0042400E0DD
:10497000F5E700BF204610BD10B5002028490860AB
:1049800007F060FB0120FCF70FFBF6F7D3FF552182
:104990002448F6F7D1FCF8F78DF8F8F707FF0BF08D
:1049A0001DFEF5F7C7FEF9F783FCF6F743F907F0AC
:1049B00031FFF9F7B5FCF9F79DFEF8F7CFFAFFF7ED
:1049C000D3FBFDF78DFEFFF7CBFCFFF73FFDFEF7B6
:1049D00025FFFFF74BF800F05BF8E12040020BF0F9
:1049E0003FFAF6F7AFFAFBF799F9F9F79BFE0E4A93
:1049F000FF219131012009F023FC00221146012002
:104A000009F062FB09F098FA09F04EFBF8F750FF45
:104A10000221012000F0A2FCFAF710FE10BD0000F8
:104A20004C000020340800200090D00370B50646EA
:104A30000D4614460E4806600E4805600E49206873
:104A400008600E49606808600D49A06808600D495B
:104A5000206908600C49E06808600C4960690860DA
:104A600005480068002802D003480068804770BDF0
:104A7000B8000020C0000020A0000020A4000020FA
:104A8000A8000020AC000020B0000020B4000020EE
:104A900000B587B00C4801900C4802900C48039078
:104AA0000020049005900B48069000200A490860F9
:104AB00048600A490860486001AA0121C902084803
:104AC000FFF7B4FF07B000BDE54A0100894E0100C1
:104AD000114E01003D4D010030120020280A002037
:104AE0003817002001207047F3B5C3B00446449E38
:104AF0000020009057E002E0641C761E00BF022EEA
:104B000005D32078EB28F7D160789028F4D1072ED0
:104B100000D24AE0A778FD1CB54200D945E0A81EA6
:104B2000205C0002691E615C08434290042D38D964
:104B3000291FA01C0BF06CFD4299884226D11D480C
:104B40000068002804D0B91EE01C1A4A1268904779
:104B500019480068002824D0E1786846017120795E
:104B600081116846417120798106890E68468171FC
:104B7000381FC1B26846C171C279611D02A8F3F73E
:104B800076FB01A80C49096888470AE000200090DC
:104B900002E00098401C00900098A842F9D3002041
:104BA00000906419761B072EA5D200BF4498801B85
:104BB00045B0F0BDAC000020B4000020F7B5C0B097
:104BC000154600260027E81DFF210131884202DD3D
:104BD000002043B0F0BDEB21684601709021417088
:104BE000281DC1B2684681700021C1704098C1B2D1
:104BF000684601710524002605E04198805D6946FC
:104C00000855641C761CAE42F7DBA11E00A80230DA
:104C10000BF0FEFC0746381269460855641C0F5518
:104C2000641C06480068002805D021466846034AEF
:104C300012689047CDE70020CBE70000A4000020D9
:104C400070B50024002500261B4840681A490968F1
:104C5000884200D170BD18484068174909688842E9
:104C600005D91548406814490968451A07E01248F3
:104C7000006811494968401A012189020D1AFF2D67
:104C800001D9FF2600E02E4600240DE00A48016805
:104C90000830405C0949085507480088401C8005D9
:104CA000800D05490860641CB442EFD3B1B20348DB
:104CB0000BF032F900BFCDE730120020381600208B
:104CC00070B500251A480068002830D0194A1288AB
:104CD000FF230133991A184A1268164B1B88D01803
:104CE000134A126890470546002D20D011480088CD
:104CF000401910490880084601880F480068FFF7EE
:104D0000F3FE0446002C0DDD0A480088844209DACF
:104D100008480088021B0848006801190648006816
:104D2000F3F7A5FA03480088001B0249088070BD0C
:104D3000A8000020BC000020B800002038B50446C0
:104D400000200090A07810280CD120792D490870FF
:104D500008460078012853D1002211462020FFF791
:104D60002DFF4DE0A078122803D120792549087243
:104D700046E0A078052803D12079224988723FE0D7
:104D8000A07802281DD120791E4948720846407A31
:104D9000012806D10090012269460420FFF70EFF8A
:104DA0002EE01848407A02282AD100BFBFF34F8F67
:104DB00015481649C860BFF34F8F00BF00BF00BF42
:104DC000FDE7A07801281BD12079332803D10120E9
:104DD0000C49487005E02079352802D100200949A6
:104DE0004870607907498870607A0006217A090462
:104DF0000843E17909020843A17908430149486061
:104E000038BD00001C0A00200400FA0500ED00E097
:104E100070B503460022002400251A484068194E48
:104E20003668B04201D1002070BD16484068154E6A
:104E30003668B04205D913484068124E3668841B64
:104E400007E0104800680F4E7668801B0126F602C6
:104E5000341AA14201D9254600E00D4600220CE09B
:104E6000084806680830805D985406480088401C51
:104E70004005400D034E3060521CAA42F0D3284634
:104E8000D2E70000280A002070B503460022002463
:104E900015484068144D2D68A84208D31248406850
:104EA000114D2D68401B0125AD022C1A04E00E485F
:104EB00000680D4D6D68441BA14201D9012070BDF1
:104EC00000220CE09D5C084846680830855508388B
:104ED0008088401C8005800D034D6860521C8A420A
:104EE000F0D30020EBE700003012002010B502489C
:104EF000FFF7F8FA10BD0000D41102000021014AAA
:104F00001175704740600040014600BFF020084026
:104F100000110A23584302460807000F8018C0B248
:104F200070470146002204E0501CC2B208460A380D
:104F3000C1B20A29F8DA1007000E084370470000D2
:104F400010B5044601218020F6F780FA607A012826
:104F500005D14248C078102108434049C870607AA2
:104F6000A22805D13E48007F802108433C490877AC
:104F7000607A3B49087700203A4948770846407FE5
:104F80002178084337494877E07B002805D0084658
:104F9000407F20210843334948773248407FC0088A
:104FA000C000A17A08432F4948770846807FF7213F
:104FB00008402C498877E078FFF7B3FF29498874C7
:104FC000A078FFF7AEFF2749C8746078FFF7A9FF04
:104FD000244908752078002805D10846007D2179EC
:104FE000084320490875E079FFF79BFF1D49887544
:104FF0006079FFF796FF1B494875A079FFF791FF8D
:105000001849C875207AFFF78CFF164908760846BC
:10501000807F4006400E8877E07A002806D0084658
:10502000807F402108430F49887703E00D48807F47
:105030000C498877A07BFFF774FF0A498876607B6C
:10504000FFF76FFF0749C876207B08770846807F07
:10505000102188430349887710BD000020040240D6
:1050600060040440404F044010B504461B48807F54
:1050700001210843194988772078FFF752FF174923
:1050800008756078FFF74DFF1449C874A078FFF7E2
:1050900048FF1249887420780C2806DD0846407FB6
:1050A000082108430D49487709E00C48407F0B4927
:1050B00048770846007DE1780843084908750748A5
:1050C000807F400840000549887700BF0348807F03
:1050D000022108400028F9D110BD0000404F0440D3
:1050E00010B500201449087616200AF075FF00213B
:1050F000124801761248407F8021084310494877C2
:105100000846807F012108430D49887700BF0C487D
:10511000807F022108400028F9D00948807F40089C
:1051200040000749887700BF0548807F022108407A
:105130000028F9D110BD00004060004040610040EF
:10514000404F044010B5002007490870002120207E
:10515000F6F77CF90121054801750020044908751E
:1051600015200AF021FF10BD0050044040610040AE
:105170004060004070B504460D46002C14D0002D50
:1051800012D0042D10D800F013F800280CD10026FE
:1051900008E00649885D22460121F4F7E7F8A41CDF
:1051A000701CC6B2AE42F4DB70BD000050110200AC
:1051B00000200549897DC907C90F002901D00120B8
:1051C00000E00020704700000050044030B585B07A
:1051D00005460C4600200390049000900190029038
:1051E000072C0BDC0120A04081B26846818101219F
:1051F000C17303A90220FAF7CBFE3EE0082C01D0D0
:10520000092C0BD10120A04081B268468181012187
:10521000C17303A90120FAF7BBFE2EE00A2C03D0CC
:105220000B2C01D00D2C0BD10120A04081B268467F
:1052300081810121C17303A90020FAF7A9FE1CE0B6
:105240000C2C01D00F2C0BD10120A04081B268465C
:1052500081810121C17303A90E20FAF799FE0CE0A8
:105260000E2C0AD10120A04081B268468181012123
:10527000C17303A90C20FAF78BFE00216846017068
:10528000C17041700121817000210171C1720D2135
:105290008172FF21017200214172F4F7C7F80349BE
:1052A0001520FDF7E7F805B030BD0000FD4E010008
:1052B00010B500201049087515200AF075FE002170
:1052C0000E4801751520002809DB00BF00BFC2068B
:1052D000D20E012191400A4A116000BF00BF00BFF9
:1052E000084880798011032805D00648007880217D
:1052F00008430449087010BD406000404061004010
:1053000000E100E00050044010B5F4F789F910BD49
:1053100010B501231A4600211846F6F753F801226A
:1053200011461046F6F7C4F8F6F7B0F803480BF04C
:1053300047F902480249086010BD00000090D00300
:105340004807002000BF04480069042108430249BF
:10535000086130BF00BF704700ED00E0F3B585B0D5
:105360000546002400270026002003900490EEB29A
:105370002804070E0F2F54DA082E52DA002009E015
:105380000C214143284A515AA94201D1044603E065
:10539000411CC8B21728F3D300BF0120B04086B229
:1053A0000C20604320494018C3780C20604340180B
:1053B0008278F8B231460190FAF78EFE684686810F
:1053C000012181730021C17302214174F8B203A944
:1053D000FAF7DEFD0C216143134A8918C888FBF7F0
:1053E00009FF0C20604310494018C18868460181BC
:1053F00069460698887202A8FBF716FE0C226243E3
:10540000094BD21891680C226243D218042010561E
:10541000FDF730F80C216143034A8918C888FBF76F
:105420006DFE07B0F0BD000068130200FEB5054632
:105430000C460020C0430290EFB22804060E0F2E47
:1054400042DA082F40DA0120B840694608808020FF
:105450002040002816D101208870A007800F022864
:1054600001D1487109E0A007800F012802D16946E7
:10547000487102E0002069464871F0B26946FAF7C7
:1054800087FD1FE00020694688700E20204000281C
:1054900000D000BF10202040002802D169460871CA
:1054A00002E0012069460871E007C00F002802D120
:1054B0006946887102E0012069468871F0B2694648
:1054C000FAF766FD002002900298FEBD30B5014655
:1054D000CAB20C04230E00200F2B0FDA082A0DDAB3
:1054E00001249440A2B2064C03252D026419E45C09
:1054F0001440002C01D0012000E0002030BD00004D
:1055000000000440F8B504460F460020C043009058
:10551000E6B22004050E0F2D11DA082E0FDA012055
:10552000B04086B2002F04D1E8B23146FAF72CFE23
:1055300003E0E8B23146FAF737FE00200090009809
:10554000F8BD00001649897F01221143144A917762
:1055500000BF1349897F022211400029F9D0104968
:10556000897C81700E49C97C41700D49097D0170AB
:105570000B498A7D8271497D01710949CA7D427159
:105580000A7EC271897F49084900054A917700BFA8
:105590000349897F022211400029F9D17047000098
:1055A000404F044003B585B0002001900290039065
:1055B0000490002168464173817E01A8C17068464D
:1055C000417E01A881706846017E4171002101A8D9
:1055D0000171082168460171817D01A8C171684689
:1055E000C17D4172417D01A881716846017D01A89C
:1055F0000172002168468173C17301A881730C2177
:1056000041734121684601740021C17401A8FFF76C
:1056100097FC1A200449888204491620FCF72AFFC7
:1056200000F006F807B000BD204F04400D0702004F
:1056300010B5FFF755FD10BD70B504460D46601E50
:105640000D49884200D90124002C00D101244020BA
:105650000A490870084600786043094948610321F7
:10566000081F0AF0D1FC0020054988610720086165
:105670000448056070BD0000FFFFFF0074010020BA
:1056800000E000E0700100200020C043002809DB9A
:10569000C206D20E01219140054A1160BFF34F8F1F
:1056A000BFF36F8F00BF0020024908618861704717
:1056B00080E100E000E000E010B50AF04BFC10BD16
:1056C0001A20084908722B2048723C2088724D200D
:1056D000C8727F20044909680860AC2003494870FB
:1056E00070470000000402407801002000100240D2
:1056F00010B51C480078012812D11B480078642896
:1057000009DB022019494871087100201649087008
:105710001449087004E014480078401C12490870CD
:105720001348007801281CD112480078012804D1C0
:10573000002010490870104908700F48007832287E
:105740000ADBF7F7FFF900210C48F5F7AFFD55210B
:105750000B48F5F7F1FD04E007480078401C0649C6
:10576000087010BD15070020140700200407002052
:105770000E070020100700200F0700202808002037
:1057800034080020F8B504460D460027002000909C
:1057900003200003204000130090102C04D0122C92
:1057A00002D01148844217D122202840222806D155
:1057B00027073F0F39460098F4F7A8FF0646122046
:1057C000284012280ED12007000F471C39460098A8
:1057D000F4F79CFF064605E02107090F0098F4F74F
:1057E00095FF06463046F8BD10100000F8B5044697
:1057F0000D46002600270120000320400713102C2F
:1058000004D0122C02D00F48844215D12220284007
:10581000222805D12607360F31463846FAF7B6F862
:105820001220284012280CD12007000F461C3146B8
:105830003846FAF7ABF804E02107090F3846FAF7C3
:10584000A5F8F8BD10100000FFB58BB01C46002075
:105850000790069005903848049010210B98084056
:10586000002801D0022707E040210B9808400028BB
:1058700001D0012700E00027002C04D01498047008
:105880000120089001E010200890002548E0002C3D
:1058900008D025466000294A115A0C98F2F750FCAE
:1058A000079006E06800254A115A0C98F2F748FC68
:1058B00007903E4630E0711C0798F2F741FC400823
:1058C00006900D98F2F792FD03900D9A0699881AAA
:1058D000F2F78CFD18490190F2F70DFD0290039943
:1058E000F2F746FD05900598F2F787FD4900490853
:1058F000039102900498F2F780FD49004908019154
:105900000090039B029AF2F78DFD03D20A95099647
:1059100005980490701CC6B27F2ECCDD681CC5B201
:1059200008988542B3DB14990A980870149909986D
:10593000487004980FB0F0BD0000C8427C1402000B
:105940000246412A2ED010DC212A2AD006DC102A59
:1059500045D0122A4BD0202A59D11CE0222A26D029
:10596000232A2AD0402A52D116E081235B01D01A83
:105970009A4228D008DC422A1AD0432A1ED0254851
:105980001018002843D13AE0012822D020281BD04B
:1059900021283CD11EE000BF1F4803890B4303812F
:1059A00036E000BF1C4843890B43438130E000BF11
:1059B000194883890B4383812AE000BF1648C389B5
:1059C0000B43C38124E000BF144883880B438380CA
:1059D0001EE000BF1148C3880B43C38018E00E4887
:1059E00043890B43438103890B43038110E00A4839
:1059F000C3890B43C38183890B43838108E0074834
:105A0000C3880B43C38083880B43838000E000BFBF
:105A100000BF7047F0EFFFFF001104400014044086
:105A2000F0B505460E46412D30D010DC212D2CD08E
:105A300006DC102D51D0122D56D0202D62D11CE045
:105A4000222D2AD0232D30D0402D5BD116E081218C
:105A50004901681A8D4230D008DC422D1ED0432DFA
:105A600024D02A48281800284CD144E001282CD002
:105A7000202823D0212845D128E000BF244F388892
:105A8000314600F049F804463DE000BF204F7888D9
:105A9000314600F041F8044635E000BF1C4FB8889D
:105AA000314600F039F804462DE000BF184FF88861
:105AB000314600F031F8044625E000BF154F388824
:105AC000314600F029F804461DE000BF114F7888E8
:105AD000314600F021F8044615E00D4F7888314634
:105AE00000F01AF804460EE0094FF888314600F03D
:105AF00013F8044607E0074F7888314600F00CF8A9
:105B0000044600E000BF00BF2046F0BDF0EFFFFFFD
:105B100000110440001404400246002013460B40CC
:105B2000002B01D0012000E000207047FFB581B0BC
:105B30000E461746012F07D1F748407D00090001A6
:105B4000C01DF549487505E0F348407D0009000196
:105B5000F1494875049801287ED10A210198F2F78D
:105B6000EFFA0546ED48445DE007C00F002807D076
:105B7000E948007C00090001C01DE749087405E000
:105B8000E548007C00090001E34908740220204038
:105B9000002807D0E048C07BF02188437030DE4900
:105BA000C87305E0DC48C07BF0218843DA49C8733C
:105BB00004202040002807D0D748807C000900013D
:105BC000C01DD549887405E0D348807C00090001D8
:105BD000D149887408202040002807D0CE48407C56
:105BE000F02188437030CC49487405E0CA48407CB5
:105BF000F0218843C849487410202040002807D06D
:105C0000C548407C00090001C01DC349487405E037
:105C1000C148407C00090001BF4948742020204051
:105C2000002807D0BC48007CF02188437030BA4976
:105C3000087405E0B848007CF0218843B649087430
:105C400040202040002808D0B348807CF0218843C1
:105C50007030B149887406E08BE0AF48807CF02159
:105C60008843AD4988740A210198F2F769FA0D4614
:105C7000AA48445DE007C00F002807D0A648807BF3
:105C8000F02188437030A449887305E0A248807BE6
:105C9000F0218843A049887302202040002807D0C3
:105CA0009D48807B00090001C01D9B49887305E069
:105CB0009948807B0009000197498873042020409F
:105CC000002807D09448007DF02188437030924925
:105CD000087505E09048007DF02188438E490875DD
:105CE00008202040002807D08B48007D00090001D3
:105CF000C01D8949087505E08748007D000900013D
:105D00008549087510202040002807D08248C07CB3
:105D1000F021884370308049C87405E07E48C07C1B
:105D2000F02188437C49C87420202040002807D0F7
:105D30007948C07B00090001C01D7749C87305E0A0
:105D40007548C07B000900017349C873402020409A
:105D5000002807D07048C07C00090001C01D6E49B2
:105D6000C87454E06C48C07C000900016A49C874DA
:105D70004DE06948007C0009000167490874084645
:105D8000C07BF02188436449C8730846807C0009C1
:105D9000000188740846407CF02188435E494874BD
:105DA0000846407C0009000148740846007CF02148
:105DB0008843594908740846807CF0218843564935
:105DC00088740846807BF0218843534988730846CD
:105DD000807B0009000188730846007DF02188431C
:105DE0004D4908750846007D000900010875084600
:105DF000C07CF02188434849C8740846C07B00092C
:105E00000001C8730846C07C00090001C8740A98E4
:105E100001287DD10A213046F2F792F905463F4824
:105E2000445DE007C00F002807D03B48407B0009D5
:105E30000001C01D3849487305E03748407B000920
:105E400000013549487302202040002807D032481D
:105E5000007BF021884370302F49087305E02E48FD
:105E6000007BF02188432C4908730420204000283F
:105E700007D02948807DF0218843703026498875F5
:105E800005E02548807DF021884323498875082056
:105E90002040002807D02048807D00090001C01D57
:105EA0001D49887505E01C48807D000900011A49DC
:105EB000887510202040002807D01748407DF02129
:105EC000884370301449487505E01348407DF0213F
:105ED00088431149487520202040002807D00E48EB
:105EE000407BF021884370300B49487305E00A4835
:105EF000407BF02188430849487340202040002817
:105F00000ED00548C07D00090001C01D024900E017
:105F100092E0C8750AE000001C260020C00E0200B6
:105F20006D48C07D000900016B49C8750A213046E3
:105F3000F2F706F90D466948445DE007C00F0028F6
:105F400007D06548C07AF021884370306249C87232
:105F500005E06148C07AF02188435F49C872022099
:105F60002040002807D05C48C07A00090001C01D0D
:105F70005949C87205E05848C07A000900015649DD
:105F8000C87204202040002807D05348407E0009F2
:105F90000001C01D5049487605E04F48407E000989
:105FA00000014D49487608202040002807D04A4883
:105FB000007EF021884370304749087605E0464866
:105FC000007EF021884344490876102020400028B4
:105FD00007D04148007E00090001C01D3E490876F7
:105FE00005E03D48007E000900013B49087620207D
:105FF0002040002807D03848007B00090001C01D60
:106000003549087305E03448007B00090001324936
:10601000087340202040002807D02F48C07DF02181
:10602000884370302C49C87554E02B48C07DF0215E
:1060300088432949C8754DE02748407B0009000185
:10604000254948730846007BF0218843224908739C
:106050000846807DF02188431F4988750846807D69
:106060000009000188750846407DF02188431A49DF
:1060700048750846407BF021884317494873084615
:10608000C07D00090001C8750846C07AF021884328
:106090001149C8720846C07A00090001C872084652
:1060A000407E0009000148760846007EF0218843C2
:1060B000094908760846007E00090001087608466E
:1060C000007B0009000108730846C07DF021884369
:1060D0000149C87505B0F0BD1C260020C00E0200A5
:1060E000FFB581B00E461746019801287ED104986D
:1060F000002828D1FB480078012824D0F6F708FCB6
:10610000F94988421FD3FAF7D5FD00280DD0F7488A
:10611000807DF02188437030F44988750846C07C42
:1061200000090001C01DC8741AE0F048807DF0210C
:1061300088431030ED4988750846C07C000900018D
:10614000401CC8740CE0E948807DF0218843703021
:10615000E64988750846C07C00090001C01DC87466
:10616000E248C07CF02188437030E049C87408469A
:10617000007EF02188437030DC4908760846807D37
:1061800000090001401C88750846407DF0218843C5
:106190001030D64948750846407D00090001401C72
:1061A00048750846007DF02188431030CF490875B6
:1061B0000846007D00090001401C0875330009F005
:1061C000E5FE062E261E140C042FC848007D00098B
:1061D0000001C01DC549087500BFC448007DF021FD
:1061E00088437030C149087500BF00E0AFE1BF4887
:1061F000407D00090001C01DBC49487500BFBB4877
:10620000407DF02188437030B849487500BFB748D9
:10621000807D00090001C01DB449887500BF00E001
:1062200000BF00BF049800285ED1AE480078012866
:106230005AD0F6F76DFBAC49884255D3AB48C07FC6
:10624000F0218843A949C8770846807F00090001EA
:1062500088770846407FF0218843A449487708465C
:10626000007FF0218843A14908770846C07DF021CE
:1062700088439E49C8750846C07F00090001C87759
:106280000846807FF0218843984988770846407FF8
:1062900000090001C01D48770846807EF021884330
:1062A000924988760846807E000900018876084673
:1062B000407E0009000148760846007E0009000182
:1062C00008760846007F0009000108770846C07E6E
:1062D000F02188438549C8760846407EF0218843EE
:1062E000703082494876B8E164213846F1F728FFDA
:1062F0000546012D07D17D48C07FF02188437030CD
:106300007A49C87705E07948C07FF021884377490A
:10631000C8770A213846F1F713FF0A210090F1F7F8
:106320000FFF0D46642F02D37148445D01E07148B0
:10633000445DE007C00F002807D06C48807F00094B
:106340000001C01D6949887705E06848807F000921
:1063500000016649887702202040002807D0634862
:10636000407FF021884370306049487705E05F48FE
:10637000407FF02188435D49487704202040002871
:1063800007D05A48007FF02188437030574908777A
:1063900005E05648007FF0218843544908770820DB
:1063A0002040002807D05148C07DF021884370303C
:1063B0004E49C87505E04D48C07DF02188434B49E2
:1063C000C87510202040002807D04848C07F000929
:1063D0000001C01D4549C87705E04448C07F000959
:1063E00000014249C87720202040002807D03F48BC
:1063F000807FF021884370303C49887705E03B4836
:10640000807FF02188433949887740202040002848
:1064100007D03648407F00090001C01D3349487746
:1064200005E03248407F00090001304948770A21E1
:106430003846F1F785FE0D462D48445DE007C00F54
:10644000002807D02948807EF021884370302749F2
:10645000887605E02548807EF021884323498876A8
:1064600002202040002807D02048807E000900013B
:10647000C01D1E49887605E01C48807E0009000189
:106480001A49887604202040002807D01748407E0B
:1064900000090001C01D1549487605E01348407EFB
:1064A000000900011149487608202040002807D043
:1064B0000E48007E00090001C01D0C49087605E069
:1064C0000A48007E00090001084908761020204093
:1064D000002811D00548007F00090001C01D0349B4
:1064E00008770FE001010020B80B0000F026002023
:1064F000C00E0200D30E02005948007F00090001BF
:106500005749087720202040002807D05448C07EF3
:10651000F021884370305249C87605E05048C07E6B
:10652000F02188434E49C87640202040002807D0FB
:106530004B48407EF02188437030494948768CE0D2
:106540004748407EF02188434549487685E04448E5
:10655000807D00090001424988750846407DF02190
:1065600088433F4948750846407D00090001487549
:106570000846007DF0218843394908750846007DAA
:106580000009000108750846C07C00090001C874B4
:106590000846807DF0218843314988750846C07CD3
:1065A000F02188432E49C8740846007EF0218843B4
:1065B0002B4908760846C07FF02188432849C877D0
:1065C0000846807F0009000188770846407FF02157
:1065D0008843234948770846007FF02188432049B3
:1065E00008770846C07DF02188431D49C8750846D4
:1065F000C07F00090001C8770846807FF0218843EA
:10660000174988770846407F000900014877084607
:10661000807EF0218843124988760846807E0009F2
:10662000000188760846407E000900014876084649
:10663000007E0009000108760846007F000900017D
:1066400008770846C07EF02188430549C876084689
:10665000407EF02188430249487605B0F0BD000035
:10666000F026002010B50146002200200A0EFE4B45
:10667000985CC307DB0F002B07D0FC4BDB7FF024BB
:10668000A3437033F94CE37705E0F84BDB7FF0244C
:10669000A343F64CE37702230340002B07D0F34BD0
:1066A000DB7F1B091B01DB1DF04CE37705E0EF4BA3
:1066B000DB7F1B091B01ED4CE37704230340002B18
:1066C00007D0EA4B9B7F1B091B01DB1DE74CA3771F
:1066D00005E0E64B9B7F1B091B01E44CA3770823D5
:1066E0000340002B09D0E14B20335B781B091B01D1
:1066F000DB1DDE4C2034637007E0DC4B20335B781D
:106700001B091B01D94C2034637010230340002B5C
:1067100009D0D64B20331B78F024A3437033D34CDD
:106720002034237007E0D14B20331B78F024A3439F
:10673000CE4C2034237020230340002B09D0CB4BB8
:1067400020331B781B091B01DB1DC84C2034237030
:1067500007E0C64B20331B781B091B01C34C2034B8
:10676000237040230340002B07D0C04B9B7FF024B5
:10677000A3437033BD4CA37705E0BC4B9B7FF02453
:10678000A343BA4CA377FF231B040B401A0CB64B50
:10679000985CC307DB0F002B07D0B44B1B7F1B0992
:1067A0001B01DB1DB14C237705E0B04B1B7F1B09A0
:1067B0001B01AE4C237702230340002B07D0AB4BC9
:1067C000DB7EF024A3437033A84CE37605E0A74BAF
:1067D000DB7EF024A343A54CE37604230340002B87
:1067E00007D0A24B9B7EF024A34370339F4CA3762B
:1067F00005E09E4B9B7EF024A3439C4CA37608238C
:106800000340002B07D0994B5B7FF024A3437033E8
:10681000964C637705E0954B5B7FF024A343934C44
:10682000637710230340002B07D0904B5B7F1B093D
:106830001B01DB1D8D4C637705E08C4B5B7F1B09D7
:106840001B018A4C637720230340002B07D0874B22
:106850001B7FF024A3437033844C237705E0834BE4
:106860001B7FF024A343814C237740230340002B5C
:1068700007D07E4BDB7E1B091B01DB1D7B4CE376C7
:1068800005E07A4BDB7E1B091B01784CE376FF2386
:106890001B020B401A0A744B985CC307DB0F002BDA
:1068A00007D0724B1B7EF024A34370336F4C2376CA
:1068B00005E06E4B1B7EF024A3436C4C2376022331
:1068C0000340002B07D0694B1B7E1B091B01DB1DFE
:1068D000664C237605E0654B1B7E1B091B01634C50
:1068E000237604230340002B07D0604BDB7D1B097C
:1068F0001B01DB1D5D4CE37505E05C4BDB7D1B097B
:106900001B015A4CE37508230340002B07D0574B5B
:106910009B7E1B091B01DB1D544CA37605E0534BEA
:106920009B7E1B091B01514CA37610230340002BB7
:1069300007D04E4B5B7EF024A34370334B4C637601
:1069400005E04A4B5B7EF024A343484C637620234A
:106950000340002B07D0454B5B7E1B091B01DB1D51
:10696000424C637605E0414B5B7E1B091B013F4CAB
:10697000637640230340002B07D03C4BDB7DF024A3
:10698000A3437033394CE37505E0384BDB7DF024CD
:10699000A343364CE375CAB2334B985CC307DB0F95
:1069A000002B07D0314B1B7DF024A34370332F4CB9
:1069B000237505E02D4B1B7DF024A3432B4C237541
:1069C00002230340002B07D0284B1B7D1B091B0112
:1069D000DB1D264C237505E0244B1B7D1B091B0189
:1069E000224C237504230340002B07D01F4BDB7C74
:1069F0001B091B01DB1D1D4CE37405E01B4BDB7CFD
:106A00001B091B01194CE37408230340002B07D01A
:106A1000164B9B7CF024A3437033144CA37405E005
:106A2000124B9B7CF024A343104CA374102303400F
:106A3000002B07D00D4B5B7DF024A34370330B4C30
:106A4000637505E0094B5B7DF024A343074C637538
:106A500020230340002B0BD0044B5B7D1B091B0143
:106A6000DB1D024C637509E0C00E0200D026002039
:106A70000C4B5B7D1B091B010A4C637540230340D3
:106A8000002B07D0074BDB7CF024A3437033054C6D
:106A9000E37405E0034BDB7CF024A343014CE37477
:106AA00010BD0000D026002000B501287ED1FE4A8E
:106AB000D278F0239A437032FB4BDA701A4612797F
:106AC00012091201D21D1A711A461279F0239A4343
:106AD0007032F54B1A711A46527912091201D21D01
:106AE0005A711A465279F0239A437032EE4B5A711A
:106AF0001A46D27912091201D21DDA711A46D279D8
:106B0000F0239A437032E84BDA711A46527A12092E
:106B10001201D21D5A721A46527AF0239A437032E9
:106B2000E14B5A721A46927AF0239A437032DE4B46
:106B30009A721A469278F0239A437032DA4B9A701E
:106B40001A46D27A12091201D21DDA721A46527806
:106B500012091201D21D5A701A46D27AF0239A43B2
:106B60007032D14BDA721A46203AD27FF0239A4320
:106B70007032CD4B203BDA77CB4A127B12091201DF
:106B8000D21D20331A731A46203A927F120912013D
:106B9000D21D203B9A77C44A127BF0239A4370326D
:106BA000C14B1A731A46203A127F00E0F2E1F0233B
:106BB0009A437032BC4B203B1A77BB4A527B120976
:106BC0001201D21D20335A731A46203AD27E12097E
:106BD0001201D21D203BDA76B44AD278F0239A43D0
:106BE0007032B24BDA701A46127B12091201D21DB2
:106BF0001A731A46127912091201D21D1A711A4615
:106C0000927AF0239A437032A84B9A721A461279FC
:106C1000F0239A437032A54B1A711A465279120921
:106C20001201D21D5A711A46927912091201D21D0F
:106C30009A711A46127A12091201D21D1A721A4654
:106C4000127AF0239A437032984B1A721A46527A8B
:106C500012091201D21D5A72934A92791209120135
:106C6000521C914B9A711A469279F0239A43103232
:106C70008D4B9A711A46127A12091201521C1A721D
:106C80001A46127AF0239A431032874B1A721A4628
:106C9000927A12091201521C9A721A46D27812097B
:106CA0001201521CDA701A46927812091201521C13
:106CB0009A701A465278F0239A4310327A4B5A70DF
:106CC0001A461278F0239A431032774B1A701A46FC
:106CD000127812091201521C1A701A46203AD27FF9
:106CE00012091201521C203BDA771A46927FF023D8
:106CF0009A4310326C4B203B9A771A46527FF0230E
:106D00009A431032684B203B5A771A46527F120939
:106D10001201521C5A771A46127F12091201521C94
:106D20001A771A46D27EF0239A4310325E4B203BEC
:106D3000DA761A46927EF0239A4310325A4B203B61
:106D40009A765A4A127BF0239A431032574B1A73A1
:106D50001A46D27AF0239A431032544BDA721A460A
:106D6000D27A12091201521CDA721A46927A120968
:106D70001201521C9A721A46527AF0239A43103228
:106D80004A4B5A721A465279F0239A431032474BB3
:106D90005A711A46D279F0239A431032434BDA7172
:106DA0000B0009F0F3F819F3E9DFD5CBC1B7ADA3B8
:106DB000998F87786E645A50463E362E261E160EE0
:106DC000F5003A4AD279F0239A437032374BDA71A0
:106DD00000BF364A5279F0239A437032334B5A71CE
:106DE00000BF324A527AF0239A4370322F4B5A72C4
:106DF00000BF2E4A927A12091201D21D2B4B9A72B1
:106E000000BF2A4AD27A12091201D21D274BDA7228
:106E100000BF264AD27AF0239A437032234BDA72AB
:106E200000BF224A127BF0239A4370321F4B1A7321
:106E300000BF1D4A203A927EF0239A4370321A4BCB
:106E4000203B9A7600BF184A203AD27EF0239A431C
:106E50007032154B203BDA7600BF134A203A127F7E
:106E600012091201D21D104B203B1A7700BF0E4AA7
:106E7000203A527F12091201D21D0B4B203B5A7748
:106E800000BF094A203A527FF0239A437032064BE2
:106E9000203B5A7700BF044A203A927FF0239A435E
:106EA0007032014B203B03E03C26002010270020DD
:106EB0009A7700BFDC4AD27F12091201D21DDA4B49
:106EC000DA7700BFD84A2032127812091201D21D97
:106ED000D54B20331A7000BFD34A20321278F023EA
:106EE0009A437032D04B20331A7000BFCE4A203202
:106EF0005278F0239A437032CB4B20335A7000BF44
:106F0000C94A2032927812091201D21DC64B203391
:106F10009A7000BFC44A2032D27812091201D21DE1
:106F2000C14B2033DA7000BFBF4A2032927A120977
:106F30001201D21DBC4B20339A7200BFBA4A2032D4
:106F4000127AF0239A437032B74B20331A7200BF83
:106F5000B54A2032127A12091201D21DB24B2033E7
:106F60001A7200BFB04A20329279F0239A437032ED
:106F7000AD4B20339A7100BFAB4A2032927912098F
:106F80001201D21DA84B20339A7100BF01E0FFE728
:106F900000BF47E1A44A2032D278F0239A43A24BA3
:106FA0002033DA701A461279120912011A711A4640
:106FB0001279F0239A439C4B20331A711A46527966
:106FC000120912015A711A465279F0239A43964BCC
:106FD00020335A711A46D27912091201DA711A460F
:106FE000D279F0239A43904B2033DA711A46527AC1
:106FF000120912015A721A46527AF0239A438A4BA6
:1070000020335A721A46927AF0239A43864B2033E1
:107010009A721A469278F0239A43834B20339A70DF
:107020001A46D27A12091201DA721A4652781209F5
:1070300012015A701A46D27AF0239A437A4B2033BF
:10704000DA72794AD27FF0239A43774BDA771A467D
:107050002032127B1209120120331A73724A927F76
:1070600012091201203B9A771A462032127BF02334
:107070009A436D4B20331A736B4A127FF0239A4365
:10708000694B1A771A462032527B120912012033BB
:107090005A73654AD27E12091201203BDA76634A9E
:1070A000D278F0239A43614BDA701A46127B1209A8
:1070B00012011A731A461279120912011A711A462C
:1070C000927AF0239A43594B9A721A461279F02316
:1070D0009A43564B1A711A465279120912015A7183
:1070E0001A469279120912019A711A46127A1209F5
:1070F00012011A721A46127AF0239A434B4B1A72F3
:107100001A46527A120912015A72474A203292796B
:1071100012091201444B20339A711A469279F023D6
:107120009A43414B20339A711A46127A120912017E
:107130001A721A46127AF0239A433B4B20331A7282
:107140001A46927A120912019A721A46D2781209D4
:107150001201DA701A469278120912019A701A46D0
:107160005278F0239A43304B20335A701A461278E3
:10717000F0239A432C4B20331A701A4612781209C6
:1071800012011A70284AD27F12091201203BDA77C5
:107190001A46927FF0239A43234B9A771A46527FDE
:1071A000F0239A43204B5A771A46527F1209120154
:1071B0005A771A46127F120912011A771A46D27E9E
:1071C000F0239A43184BDA761A46927EF0239A43BC
:1071D000154B9A76154A127BF0239A43134B1A7378
:1071E0001A46D27AF0239A43104BDA721A46D27AB0
:1071F00012091201DA721A46927A120912019A726F
:107200001A46527AF0239A43084B5A721A46527918
:10721000F0239A43054B5A711A46D279F0239A43C8
:10722000024BDA7100BD00001C2600201027002050
:10723000F7B582B006461746002500200190002EC3
:107240007ED1F9F713FC05285FD1F9F733FD00284B
:107250000DD0FA484079F02188437030F7494871E1
:107260000846807800090001C01D88700AE0F348D4
:107270004079F0218843F149487108468078000937
:1072800000018870ED48C07900090001EB49C87120
:107290000846807900090001887108464079000994
:1072A000000148710846007AF0218843E3490872DA
:1072B0000846007A0009000108720846C079F021EA
:1072C0008843DE49C8710846C07800090001C870CB
:1072D00008468078F0218843D8498870084640786D
:1072E000F0218843D54948700846407800090001DC
:1072F0004870084600790009000108710846C07806
:10730000F0218843CD49C87029E2CC484079F0216A
:1073100088437030C94948710846807800090001E7
:10732000C01D88700846C07900090001C871084670
:10733000807900090001887108464079000900E061
:1073400034E0000148710846007AF0218843BB49C7
:1073500008720846007A0009000108720846C079E0
:10736000F0218843B549C8710846C078000900017A
:10737000C87008468078F0218843B0498870084674
:107380004078F0218843AD494870084640780009AC
:10739000000148700846007900090001087108469C
:1073A000C078F0218843A549C870ADE7012E5FD1B0
:1073B000F9F780FC00280DD0A0484079F0218843DF
:1073C00070309E4948710846807800090001C01D50
:1073D00088700AE099484079F021884397494871BC
:1073E000084680780009000188709448C079000937
:1073F00000019249C871084680790009000188712E
:10740000084640790009000148710846007AF021D9
:1074100088438A4908720846007A00090001087208
:107420000846C079F02188438449C8710846C0786D
:1074300000090001C87008468078F02188437F4920
:10744000887008464078F02188437C494870084697
:1074500040780009000148700846007900090001E1
:1074600008710846C078F02188437449C870DAE38F
:10747000022E7DD1F9F7FAFA05287AD1F9F71AFC2C
:10748000002877D0012F76D10A210398F0F758FE13
:107490000546F9F72BFB002802D16948445D01E05D
:1074A0006848445DE007C00F002807D06348C079F2
:1074B00000090001C01D6149C87105E05F48C0793D
:1074C000000900015D49C87102202040002807D052
:1074D0005A48807900090001C01D5849887105E0AB
:1074E00056488079000900015449887104202040E1
:1074F000002807D05148407900090001C01D4F49BC
:10750000487105E04D484079000900014B49487138
:1075100008202040002807D04848007AF0218843FE
:1075200070304649087205E04448007AF0218843EB
:107530004249087210202040002807D03F48007AB6
:1075400000090001C01D3D49087205E03B48007A72
:1075500000090001394908722020204000280BD082
:107560003648C079F021884370303449C87109E049
:10757000AEE242E1F4E0A4E03048C079F021884373
:107580002E49C87140202040002807D02B48407960
:10759000F021884370302949487105E02748407937
:1075A000F0218843254948710A210398F0F7C8FD66
:1075B0000D462348445DE007C00F002807D01F4850
:1075C000C07800090001C01D1C49C87005E01B48B7
:1075D000C078000900011949C87002202040002825
:1075E00007D016488078F02188437030134988709E
:1075F00005E012488078F021884310498870042003
:107600002040002807D00D484078F0218843703092
:107610000A49487005E009484078F0218843074945
:1076200048700820204000280ED004484078000907
:107630000001C01D014948700CE000005C260020DC
:10764000C00E0200D30E0200FE484078000900017F
:10765000FC49487010202040002807D0F9480079E4
:1076600000090001C01DF749087105E0F5480079DF
:1076700000090001F349087120202040002807D0AC
:10768000F048C078F02188437030EE49C87005E0BA
:10769000EC48C078F0218843EA49C8704020204077
:1076A000002807D0E748807800090001C01DE5499F
:1076B0008870B8E2E348807800090001E1498870E9
:1076C000B1E2E0484079F02188437030DD494871EB
:1076D0000846807800090001C01D88700846C079FE
:1076E00000090001C871084680790009000188710D
:1076F000084640790009000148710846007AF021E7
:107700008843D04908720846007A000900010872CF
:107710000846C079F0218843CA49C8710846C07834
:1077200000090001C87008468078F0218843C549E7
:10773000887008464078F0218843C249487008465E
:1077400040780009000148700846007900090001EE
:1077500008710846C078F0218843BA49C87062E2CF
:10776000B8484079F0218843B64948710846807886
:107770000009000188700846C07900090001C8713D
:10778000084680790009000188710846407900099F
:10779000000148710846007AF0218843A94908721F
:1077A0000846007A0009000108720846C079F021F5
:1077B0008843A449C8710846C07800090001C87010
:1077C00008468078F02188439E49887008464078B2
:1077D000F02188439B494870084640780009000121
:1077E0004870084600790009000108710846C07811
:1077F000F02188439349C87015E2012F73D10A2103
:107800000398F0F79DFC0546F9F770F9002802D1BE
:107810008D48445D01E08D48445DE007C00F0028BD
:1078200007D08848C07900090001C01D8549C8718A
:1078300005E08448C079000900018249C87102202E
:107840002040002807D07F48807900090001C01D32
:107850007C49887105E07B488079000900017949FD
:10786000887104202040002807D07648407900091C
:107870000001C01D7349487105E072484079000954
:1078800000017049487108202040002807D06D4849
:10789000007AF021884370306A49087205E069482F
:1078A000007AF021884367490872102020400028A0
:1078B00007D06448007A00090001C01D61490872C0
:1078C00005E06048007A000900015E490872202046
:1078D0002040002808D05B48C079F02188437030F0
:1078E0005849C87106E09DE05648C079F0218843A8
:1078F0005449C87140202040002807D051484079A1
:10790000F021884370304F49487105E04D48407977
:10791000F02188434B4948710A210398F0F710FC85
:107920000D464948445DE007C00F002807D0454890
:10793000C07800090001C01D4249C87005E04148F7
:10794000C078000900013F49C8700220204000288B
:1079500007D03C488078F0218843703039498870DE
:1079600005E038488078F021884336498870042043
:107970002040002807D033484078F02188437030F9
:107980003049487005E02F484078F02188432D4960
:10799000487008202040002807D02A484078000975
:1079A0000001C01D2749487005E0264840780009BD
:1079B00000012449487010202040002807D02148A9
:1079C000007900090001C01D1E49087105E01D482D
:1079D0000079000900011B4908712020204000287F
:1079E00007D01848C078F021884370301549C87016
:1079F00005E01448C078F02188431249C87040203F
:107A00002040002807D00F48807800090001C01DE1
:107A10000C49887007E10B4880780009000109498A
:107A2000887000E107484079F021884370300549AB
:107A300048710846807800090001C01D887008461A
:107A4000C07905E05C260020C00E0200D30E0200C3
:107A500000090001C8710846807900090001887199
:107A6000084640790009000148710846007AF02173
:107A700088436E4908720846007A000900010872BE
:107A80000846C079F02188436849C8710846C07823
:107A900000090001C87008468078F02188436349D6
:107AA000887008464078F02188436049487008464D
:107AB000407800090001487008460079000900017B
:107AC00008710846C078F02188435849C870AAE078
:107AD000032E9FD1F9F7EEF8002858D0534840798B
:107AE000F021884370305149487108468078000978
:107AF0000001C01D88700846C07900090001C01D42
:107B0000C8710846807900090001C01D88710846C7
:107B1000407900090001C01D48710846007AF02133
:107B200088437030414908720846007A0009000114
:107B300008720846C079F021884370303B49C8710B
:107B40000846C07800090001C01DC870084680784A
:107B5000F021884370303549887008464078F0211C
:107B60008843703031494870084640780009000168
:107B7000C01D4870084600790009000108710846D8
:107B8000C078F021884370302849C8704BE02748FE
:107B90004079F021884325494871084680780009DA
:107BA000000188700846C07900090001C8710846C4
:107BB00080790009000188710846407900090001B8
:107BC00048710846007AF02188431849087208462F
:107BD000007A0009000108720846C079F021884344
:107BE0001249C8710846C07800090001C8700846EB
:107BF0008078F02188430D49887008464078F0214C
:107C000088430A49487008464078000900014870D6
:107C1000084600790009000108710846C078F02183
:107C200088430249C87005B0F0BD00005C26002002
:107C300070B505460C46012D7ED1B348407D000944
:107C40000001C01DB04948750846007DF0218843F9
:107C50001030AD4908750846007D00090001401C40
:107C600008750846C07CF02188431030A649C874C6
:107C70000846807CF02188431030A3498874084668
:107C8000807C00090001401C8874F9F77DF8022807
:107C900003D0F9F779F801286ED19C4800780128C3
:107CA0006AD0F4F735FE9A49884265D3F9F702F8AD
:107CB00000282FD09448007DF021884370309249ED
:107CC00008750846007D00090001C01D08750846BA
:107CD000C07CF021884370308B49C8740846807C92
:107CE000F02188437030884988740846807C0009F8
:107CF0000001C01D88740846407DF0218843703023
:107D0000814948750846407CF021884370307E499F
:107D10004874F8E07C48007DF021884310307A49AF
:107D200008750846007D00090001401C08750846DA
:107D3000C07CF021884300E0B8E010307249C8747C
:107D40000846807CF021884310306F4988740846CB
:107D5000807C00090001401C88740846407DF021A9
:107D600088431030684948750846407CF0218843B4
:107D7000103065494874C6E0F8F766FE002826D141
:107D8000F4F7C6FD6249884221D3F8F793FF002833
:107D90000ED05D48407DF021884370305A494875C7
:107DA0000846407CF02188437030574948741CE0F5
:107DB0005548407DF02188431030534948750846A6
:107DC000407CF021884310304F4948740DE04E4804
:107DD000407DF021884370304B4948750846407C0F
:107DE000F0218843703048494874F8F72DFE012887
:107DF0002AD146480078012826D0F4F789FD444965
:107E0000884221D34048407DF021884370303E496C
:107E100048750846407CF021884370303A494874E0
:107E2000F8F748FF002807D03748007DF021884345
:107E300070303549087566E03348007DF02188438D
:107E40001030314908755EE0230008F09FF8062CD9
:107E5000241C140C042D2C48807C00090001C01D3A
:107E60002949887400BF2848807CF02188437030FD
:107E70002549887400BF2448C07CF02188437030B5
:107E80002149C87400BF2048007D00090001C01DC1
:107E90001D49087500BF1C48007DF02188437030E3
:107EA0001949087500BF00E000BF2CE01648407D6E
:107EB000F0218843144948750846007DF021884325
:107EC000114908750846007D00090001087508463B
:107ED000C07CF02188430C49C8740846807CF0219E
:107EE0008843094988740846807C00090001887429
:107EF0000846407D0009000148750846407CF02195
:107F000088430149487470BD3C26002001010020CF
:107F1000B80B000030B50246002901D1002000E076
:107F20000720130008F032F80F09141F2B374350B5
:107F30005D67727C88929FA9B500574B5B7EF024E9
:107F4000A3430401F0252C402343534C6376A1E066
:107F5000524B9B79F024A3430401F0252C4023438A
:107F60004E4CA37196E04D4B2033DB791B091B016E
:107F70000407240F2343494C2034E3718AE0464B25
:107F80002033DB7C1B091B010407240F2343424CD5
:107F90002034E3747EE0404B40331B781B091B0107
:107FA0000407240F23433C4C4034237072E03A4BC7
:107FB0002033DB7FF024A3430401F0252C4023432E
:107FC000354C2034E37765E0334B20335B7BF02482
:107FD000A3430401F0252C4023432F4C203463732A
:107FE00058E02E4B9B791B091B010407240F2343E8
:107FF0002A4CA3714EE0294B9B7CF024A34304013F
:10800000F0252C402343254CA37443E0234BDB7E17
:108010001B091B010407240F2343204CE37639E09E
:108020001D4B2033DB7F1B091B010407240F234357
:10803000194C2034E3772DE0174B9B7E1B091B0165
:108040000407240F2343144CA37623E0134B20335F
:108050009B79F024A3430401F0252C4023430F4CCB
:108060002034A37116E00D4BDB7D1B091B010407B7
:10807000240F2343094CE3750CE0074B20335B7C52
:108080001B091B010407240F2343034C2034637492
:1080900000E000BF00BF30BD1C260020F0260020FD
:1080A000F7B582B00746164600250024FE48007842
:1080B000012804D0F4F72CFCFC49884279D2FC4812
:1080C000407CF02188437030F94948740846807C30
:1080D00000090001C01D88740846007D00090001E8
:1080E000C01D08750846007DF02188437030F049B6
:1080F00008750846807CF02188437030EC4988740C
:108100000846C07C00090001C01DC8740846C07C38
:10811000F02188437030E649C8740846407C000965
:108120000001C01D48740846407D00090001C01DC3
:1081300048750846407DF02188437030DC49487519
:108140000846007CF02188437030D94908740846FD
:10815000007C00090001C01D08740846C07BF021A6
:1081600088437030D249C873BA220A210020FBF735
:10817000A5F9BA2213210020FBF7A0F9BA22112198
:108180000020FBF79BF9BA2212210020FBF796F999
:10819000BA220E210020FBF791F9BA220F2100200C
:1081A000FBF78CF9BA2210210020FBF787F9F4E3E2
:1081B000FFE7039836283DD019DC08287ED007DC7D
:1081C000801E030007F0E2FE0635A8FCFBFAF97EEC
:1081D000102874D006DC092872D00D2871D00E2822
:1081E00070D1FDE333286ED03428F9D170E13F28F7
:1081F0006AD00FDC3738082864D243007B449B8860
:108200005B009F448A009702FF025F005F006503E6
:10821000CB0318004E287BD006DC402879D04128BB
:1082200078D04D28DCD1BBE14F2874D05028D7D16D
:108230004FE100BF00BF9E48407CF02188439C492D
:1082400048740846807C0009000188740846007D57
:1082500000090001C01D08750846007DF021884313
:108260007030934908750846807CF0218843904916
:1082700088740846C07C00090001C01DC874084607
:10828000C07CF02188438A49C8740846407C0009B4
:10829000000148740846407D000900014875084601
:1082A000407DF0218843824948750846007CF021D2
:1082B00088437F4908740846007C06E0A1E2FDE39C
:1082C00037E2D2E3FBE394E028E000090001087400
:1082D0000846C07BF02188437549C873BA220A2139
:1082E0000020FBF7EBF8BA2213210020FBF7E6F899
:1082F00000220E211046FBF7E1F800220F21104664
:10830000FBF7DCF8002210211046FBF7D7F877E2E4
:10831000ABE110E2DDE26DE000BF00BF6448407CED
:10832000F0218843624948740846807C00090001B6
:1083300088740846007D00090001C01D08750846C4
:10834000007DF02188437030594908750846807CCB
:10835000F0218843564988740846C07C0009000112
:10836000C8740846C07CF02188435149C874084647
:10837000407C0009000148740846407D0009000166
:10838000C01D48750846407DF0218843484948751E
:108390000846007CF0218843454908740846007C63
:1083A0000009000108740846C07BF0218843404959
:1083B000C873BA220A21002003E055E1EFE086E00D
:1083C00016E0FBF77BF8BA2213210020FBF776F8C2
:1083D00000220E211046FBF771F800220F211046F3
:1083E000FBF76CF8002210211046FBF767F88EE7C8
:1083F00000BF00BF2E48407CF02188432C494874C0
:108400000846807C00090001C01D88740846007D74
:1084100000090001C01D08750846007DF021884351
:108420007030234908750846807CF02188437030FD
:108430001F4988740846C07C00090001C8740846BA
:10844000C07CF02188431A49C8740846407C000962
:10845000000148740846407D00090001487508463F
:10846000407DF0218843124948750846007CF02180
:1084700088430F4908740846007C0009000108740D
:108480000846C07BF02188430949C873BA220A21F3
:108490000020FBF713F8BA2213210020FBF70EF897
:1084A00000220E21104605E001010020B80B00005B
:1084B0005C260020FBF702F800220F211046FAF795
:1084C000FDFF002210211046FAF7F8FF1FE700BF5A
:1084D00000BFFE48407CF0218843FC4948740846B0
:1084E000807C00090001C01D88740846007D0009D9
:1084F0000001C01D08750846007DF02188437030DA
:10850000F24908750846807CF0218843EF49887459
:108510000846C07C00090001C8740846C07CF021F0
:108520008843EA49C8740846407C00090001C01D20
:1085300048740846407D0009000148750846407DA2
:10854000F0218843E14948750846007CF0218843C2
:10855000DE4908740846007C0009000108740846DA
:10856000C07BF0218843D949C873BA220A21002070
:10857000FAF7A4FFBA2213210020FAF79FFF002286
:108580000E211046FAF79AFF00220F211046FAF743
:1085900095FF002210211046FAF790FFF6E300BF86
:1085A000CA48407CF0218843C84948740846807C0A
:1085B0000009000188740846007D00090001087563
:1085C0000846007DF02188437030C0490875084690
:1085D000807CF0218843BD4988740846C07C00092E
:1085E0000001C8740846C07CF02188437030B74948
:1085F000C8740846407C0009000148740846407D64
:108600000009000148750846407DF0218843AF49C4
:1086100048750846007CF0218843AC490874084638
:10862000007C0009000108740846C07BF0218843E3
:10863000A649C873BA220A210020FAF73FFFBA22DE
:1086400013210020FAF73AFF00220E211046FAF714
:1086500035FF00220F211046FAF730FF00221021CB
:108660001046FAF72BFF91E300BF9848407CF021B9
:108670008843964948740846807C00090001887444
:108680000846007D0009000108750846007DF021BC
:10869000884370308D4908750846807CF0218843F6
:1086A0008A4988740846C07C00090001C8740846DD
:1086B000C07CF02188438549C8740846407C000985
:1086C000000148740846407D0009000148750846CD
:1086D000407DF021884370307C4948750846007C15
:1086E000F0218843794908740846007C000900019C
:1086F00008740846C07BF02188437449C873BA22C5
:108700000A210020FAF7DAFEBA2213210020FAF734
:10871000D5FE00220E211046FAF7D0FE00220F21CE
:108720001046FAF7CBFE002210211046FAF7C6FEDB
:108730002CE300BF00BF6548407CF02188437030C7
:10874000624948740846807C00090001C01D887495
:108750000846007D00090001C01D08750846007D1F
:10876000F02188437030594908750846807CF02113
:108770008843564988740846C07C00090001C874C3
:108780000846C07CF02188435049C8740846407CA4
:108790000009000148740846407D00090001487541
:1087A0000846407DF0218843484948750846007CCA
:1087B000F0218843454908740846007C00090001FF
:1087C00008740846C07BF02188434049C873BA2228
:1087D0000A210020FAF772FEBA2213210020FAF7CC
:1087E0006DFE00220E211046FAF768FE00220F21CE
:1087F0001046FAF763FE002210211046FAF75EFEDB
:10880000C4E200BF3148407CF02188432F494874BE
:108810000846807C0009000188740846007D000934
:10882000000108750846007DF02188437030274913
:1088300008750846807CF0218843244988740846DE
:10884000C07C00090001C8740846C07CF021884340
:1088500070301E49C8740846407C00090001487405
:108860000846407D0009000148750846407DF0211A
:108870008843164948750846007CF021884313490F
:1088800008740846007C0009000108740846C07B93
:10889000F02188430D49C873BA220A210020FAF753
:1088A0000DFEBA2213210020FAF708FE00220E2145
:1088B0001046FAF703FE00220F211046FAF7FEFDDC
:1088C000002210211046FAF7F9FD5FE25C26002035
:1088D00000BFFC48407CF0218843FA4948740846B0
:1088E000807C0009000188740846007D00090001B1
:1088F00008750846007DF02188437030F1490875FD
:108900000846807CF0218843EE4988740846C07C84
:1089100000090001C8740846C07CF0218843E94979
:10892000C8740846407C0009000148740846407D30
:108930000009000148750846407DF02188437030E9
:10894000E04948750846007CF0218843DD490874F9
:108950000846007C0009000108740846C07BF0212D
:108960008843D849C873BA220A210020FAF7A6FD25
:10897000BA2213210020FAF7A1FD00220E21104691
:10898000FAF79CFD00220F211046FAF797FD00220E
:1089900010211046FAF792FDF8E1F8E1C948407C51
:1089A000F02188437030C74948740846807C00092C
:1089B0000001C01D88740846007D00090001C01D2B
:1089C00008750846007DF0218843BE4908750846B1
:1089D000807CF0218843BB4988740846C07C00E055
:1089E000A9E000090001C8740846C07CF021884352
:1089F000B449C8740846407C000900014874084620
:108A0000407D0009000148750846407DF0218843FB
:108A1000AC4948750846007CF0218843A949087490
:108A20000846007C0009000108740846C07BF0215C
:108A30008843A449C873BA220A210020FAF73EFDF0
:108A4000BA2213210020FAF739FD00220E21104628
:108A5000FAF734FD00220F211046FAF72FFD00220D
:108A600010211046FAF72AFD90E19648407CF0214B
:108A70008843944948740846807C00090001887442
:108A80000846007D0009000108750846007DF021B8
:108A900088438C4908750846807CF02188438949C1
:108AA00088740846C07C00090001C8740846C07C70
:108AB000F02188438349C874084601E09EE003E141
:108AC000407C0009000148740846407D000900010F
:108AD00048750846407DF02188437A494875084624
:108AE000007CF0218843774908740846007C00091F
:108AF000000108740846C07BF0218843703071493A
:108B0000C87300220A211046FAF7D8FC002213216C
:108B10001046FAF7D3FCBA220E210020FAF7CEFC59
:108B200000220F211046FAF7C9FC0022102110463E
:108B3000FAF7C4FC2AE16348407CF021884361498C
:108B400048740846807C0009000188740846007D4E
:108B50000009000108750846007DF0218843594945
:108B600008750846807CF021884356498874084679
:108B7000C07C00090001C8740846C07CF02188430D
:108B80005049C8740846407C0009000148740846F2
:108B9000407D0009000148750846407DF02188436A
:108BA000484948750846007CF021884345490874C7
:108BB0000846007C00090001C01D08740846C07BFF
:108BC000F02188433F49C87300220A211046FAF772
:108BD00075FC002213211046FAF770FC00220E21CA
:108BE0001046FAF76BFCBA220F210020FAF766FC58
:108BF000002210211046FAF761FCC7E03148407CA2
:108C0000F02188432F4948740846807C0009000100
:108C100088740846007D0009000108750846007D3B
:108C2000F0218843274908750846807CF021884355
:108C3000244988740846C07C00090001C8740846AD
:108C4000C07CF02188431F49C8740846407C000955
:108C5000000148740846407D000900014875084637
:108C6000407DF0218843174948750846007CF02173
:108C700088437030134908740846007C00090001DD
:108C800008740846C07BF02188430E49C87300224F
:108C90000A211046FAF712FC002213211046FAF7B7
:108CA0000DFC00220E211046FAF708FC00220F21CD
:108CB0001046FAF703FCBA2210210020FAF7FEFB57
:108CC00064E000005C260020FA48407CF0218843E4
:108CD000F84948740846807C0009000188740846F9
:108CE000007D0009000108750846007DF0218843D9
:108CF000F04908750846807CF0218843ED49887466
:108D00000846C07C00090001C8740846C07CF021F8
:108D10008843E849C8740846407C0009000148744B
:108D20000846407D0009000148750846407DF02155
:108D30008843E04948750846007CF0218843DD49B6
:108D400008740846007C0009000108740846C07BCE
:108D5000F0218843D749C87300220A211046FAF748
:108D6000ADFB002213211046FAF7A8FB00220E21CA
:108D70001046FAF7A3FB00220F211046FAF79EFBDC
:108D8000002210211046FAF799FB00BF00BF002F08
:108D900072D0BA2211210020FAF790FBBA221221D8
:108DA0000020FAF78BFBC4480078012804D0F3F7C1
:108DB000AFFDC249884216D2C148807BF02188436A
:108DC0007030BF498873084640300078F0218843EE
:108DD0007030BB4940310870084600780009000136
:108DE000C01D08702DE07D20C000864214D2B4481A
:108DF000807BF0218843B249887308464030007870
:108E0000F02188437030AE49403108700846007840
:108E100000090001087014E0A948807BF021884314
:108E20007030A7498873084640300078F0218843A5
:108E3000A349403108700846007800090001C01DB0
:108E400008707D20C000864205D201463046EFF70B
:108E500077F9054604E09B493046EFF771F905467E
:108E600095480078012804D0F3F752FD93498842D1
:108E700003D29548445D02E0A0E29448445DE007D7
:108E8000C00F002809D08E484030C078000900018A
:108E9000C01D8B494031C87007E089484030C07818
:108EA0000009000186494031C87002202040002896
:108EB00007D08348C07900090001C01D8049C871EE
:108EC00005E07F48C079000900017D49C871042090
:108ED0002040002807D07A48807900090001C01D91
:108EE0007749887105E07648807900090001744966
:108EF000887108202040002807D071484079F0216F
:108F0000884370306E49487105E06D484079F02122
:108F100088436B49487110202040002807D06848DA
:108F2000407900090001C01D6549487105E06448A9
:108F30004079000900016249487120202040002842
:108F400007D05F480079F021884370305C49087190
:108F500005E05B480079F0218843594908714020B9
:108F60002040002807D056488079F021884370308F
:108F70005349887105E052488079F021884350496F
:108F800088717D20C000864207D264213046EFF709
:108F9000D7F805464D48445D17E06421304632302D
:108FA000EFF7CEF87D21C9000090EFF7C9F80191E5
:108FB00064210198EFF7C4F805464548864202D37C
:108FC0004148445D01E04148445D3B480078012848
:108FD00004D0F3F79DFC3949884201D23A48445DF8
:108FE000E007C00F002809D0354840308078F021D4
:108FF0008843703032494031887007E03048403053
:109000008078F02188432E4940318870022020402A
:10901000002807D02A48807A00090001C01D28498D
:10902000887205E02648807A000900012449887288
:1090300004202040002807D02148407A0009000180
:10904000C01D1F49487205E01D48407A0009000113
:109050001B49487208202040002807D01848007A91
:10906000F021884370301649087205E01448007AF0
:10907000F02188431249087210202040002807D0B0
:109080000F48007A00090001C01D0D49087205E073
:109090000B48007A0009000109490872202020408D
:1090A000002817D00648C079F02188437030044961
:1090B000C87115E05C26002001010020B80B0000FB
:1090C000D0260020A0860100C00E0200D30E0200B0
:1090D00010270000FE48C079F0218843FC49C87180
:1090E00040202040002807D0F948407AF0218843EA
:1090F0007030F749487205E0F548407AF02188431E
:10910000F34948727D20C000864210D20A213046C1
:10911000EFF716F80A210190EFF712F80D460A2E24
:1091200002D3EC48445D12E0EB48445D0FE064215B
:1091300030463230EFF704F80A210090EFF700F8DC
:109140000A210190EEF7FCFF0D46E2494C5DE34831
:109150000078012804D0F3F7DBFBE149884201D213
:10916000DC48445DE007C00F002809D0D8484030F3
:10917000807800090001C01DD5494031887007E0A2
:10918000D3484030807800090001D14940318870CF
:1091900002202040002807D0CD48807B0009000134
:1091A000C01DCB49887305E0C948807B00090001D8
:1091B000C749887304202040002807D0C448407B5A
:1091C00000090001C01DC249487305E0C048407B4A
:1091D00000090001BE49487308202040002807D03C
:1091E000BB48007BF02188437030B949087305E023
:1091F000B748007BF0218843B54908731020204010
:10920000002807D0B248C07A00090001C01DB0494B
:10921000C87205E0AE48C07A00090001AC49C872C6
:1092200020202040002807D0A948807AF0218843D8
:109230007030A749887205E0A548807AF0218843FC
:10924000A349887240202040002807D0A048407BD6
:10925000F021884370309E49487305E09C48407B6C
:10926000F02188439A4948737D20C000864207D286
:109270000A213046EEF764FF0D469648445D0BE048
:10928000642130463230EEF75BFF0A210190EEF7A1
:1092900057FF0D468F494C5D90480078012804D057
:1092A000F3F736FB8E49884201D28A48445DE007D5
:1092B000C00F002809D0864840304078F02188430C
:1092C000703083494031487007E081484030407831
:1092D000F02188437E494031487002202040002818
:1092E00009D07B484030407800090001C01D784912
:1092F0004031487007E0764840304078000900016E
:1093000073494031487004202040002807D070483D
:10931000007CF021884370306D49087405E06C488A
:10932000007CF02188436A49087408202040002806
:1093300007D06748007C00090001C01D644908741B
:1093400005E06348007C00090001614908741020B1
:109350002040002807D05E48C07BF0218843703051
:109360005B49C87305E05A48C07BF02188435849DF
:10937000C87320202040002807D05548C07B000932
:109380000001C01D5249C87305E05148C07B000967
:1093900000014F49C87340202040002807D04C48A6
:1093A000407C00090001C01D49494874ECE0484870
:1093B000407C0009000146494874E5E000220A218A
:1093C0001046FAF77BF8002213211046FAF776F8D8
:1093D000002211211046FAF771F8002212211046DE
:1093E000FAF76CF800220E211046FAF767F800220F
:1093F0000F211046FAF762F8002210211046FAF702
:109400005DF833484030C0780009000130494031F0
:10941000C8702F48C079000900014039C87108465A
:10942000807900090001887108464079F02188435D
:1094300027494871084640790009000148710846EB
:109440000079F02188432249087108468079F0218B
:1094500088431F498871084640308078F02188434E
:109460001B49403188701A48807A00090001403950
:1094700088720846407A0009000148720846007A5E
:10948000F0218843124908720846007A0009000159
:1094900008720846C079F02188430D49C871084612
:1094A000407AF02188430A49487208464030807863
:1094B00000090001403188700548807B00090001E7
:1094C000403988730846407B00090001487309E071
:1094D000D0260020C00E0200D30E020001010020A1
:1094E000B80B00000846007BF02188432749087329
:1094F0000846C07A00090001C8720846807AF02147
:109500008843224988720846407BF02188431F49DE
:109510004873084640304078F02188431B49403169
:109520004870084640780009000148701748007CE0
:10953000F0218843154908740846007C00090001A1
:1095400008740846C07BF02188431049C873084658
:10955000C07B00090001C8730846407C0009000177
:1095600048740846807BF021884308498873084680
:1095700040300078F02188430449403108700846A3
:10958000007800090001087005B0F0BDD026002069
:10959000F7B582B007460E460121FF200830FBF7E1
:1095A000B1FF0121FC48FBF7ADFFFC480078012822
:1095B0007ED0F3F7ADF9FA49884279D3F7F756FA36
:1095C000032843D1F7F74CFA002803D0F7F748FAFD
:1095D00001283BD1002F1CD1F7F76CFB00280CD0E1
:1095E000F048407CF0218843EE4948740846807C6E
:1095F00000090001C01D8874EEE0EA48407CF021BB
:109600008843E84948740846807C00090001887452
:10961000E2E0F7F74FFB00280CD0E248407CF02155
:1096200088437030DF4948740846807C0009000197
:109630008874D1E0DB48407CF0218843D9494874E4
:109640000846807C000900018874C5E0F7F708FA35
:10965000002803D0F7F704FA012865D1002F0CD1B8
:10966000D048407CF0218843CE4948740846807C2D
:1096700000090001C01D88740BE0CA48407CF0213D
:1096800088437030C74948740846807C000900014F
:109690008874F7F7E5F9002821D1C2482030C07856
:1096A000F02188437030BF492031C870BD4800E0C8
:1096B00064E0807D00090001203988750846807DBE
:1096C000F0218843B7498875BA2223210020F9F791
:1096D000F5FE002222211046F9F7F0FE7CE0F7F7B4
:1096E000BFF9012878D1AF482030C078F0218843F5
:1096F000AC492031C870AB48807D00090001C01D15
:10970000203988750846807DF02188437030A5494E
:109710008875002223211046F9F7D0FEBA222221B3
:109720000020F9F7CBFE57E09E48407CF0218843AB
:109730009C4948740846807C0009000188740846EA
:109740002030C078F021884396492031C870954870
:10975000807D00090001203988750846807DF02150
:10976000884390498875002223211046F9F7A6FE08
:10977000002222211046F9F7A1FE2DE08948407C05
:10978000F02188437030874948740846807C00097E
:109790000001C01D887408462030C078F02188433D
:1097A000703080492031C8707E48807D00090001FA
:1097B000C01D203988750846807DF02188437030AF
:1097C00078498875BA2223210020F9F777FEBA225A
:1097D00022210020F9F772FEF7F742F9002808D09D
:1097E0006E480078012804D0F3F792F86C4988425B
:1097F00076D26D48864209D96A4820304079F021F6
:109800008843703067492031487107E0654820304F
:109810004079F021884363492031487163493046DB
:10982000EEF78EFC0A210190EEF78AFC0D465E48A9
:10983000401C864202D35E48445D01E05D48445DC1
:10984000E007C00F002809D056482030C078000932
:109850000001C01D53492031C87007E05148203035
:10986000C078000900014F492031C8700220204013
:10987000002809D04B4820308078F0218843703090
:1098800048492031887007E0464820308078F02130
:10989000884344492031887004202040002809D0A2
:1098A000404820304078F021884370303D492031D5
:1098B000487007E03B4820304078F0218843394920
:1098C000203148700820204000280AD03548203038
:1098D000407900090001C01D32492031487108E07B
:1098E000A1E2304820304079000900012D492031A3
:1098F000487110202040002809D02A4820300079E3
:10990000F0218843703027492031087107E025484D
:1099100020300079F021884322492031087120202D
:109920002040002809D01F4820300079000900019C
:10993000C01D1C492031087107E01A482030007909
:1099400000090001174920310871402020400028FB
:1099500009D014482030807800090001C01D114949
:109960002031887007E00F4820308078000900011E
:109970000C49203188707D21C9003046EEF7E0FBAC
:109980000A210190EEF7DCFB0D460848864213D30E
:109990000748445D12E000000505000001010020B9
:1099A000B80B0000D02600209F8601001027000081
:1099B000C00E0200D30E0200F948445DE007C00F5C
:1099C000002807D0F748C07FF02188437030F54960
:1099D000C87705E0F348C07FF0218843F149C87794
:1099E00002202040002807D0EE48C07F0009000177
:1099F000C01DEC49C87705E0EA48C07F00090001B6
:109A0000E849C87704202040002807D0E548807F37
:109A100000090001C01DE349887705E0E148807F27
:109A200000090001DF49887708202040002809D07C
:109A3000DC482030407800090001C01DD9492031A0
:109A4000487007E0D7482030407800090001D54928
:109A50002031487010202040002809D0D148203003
:109A60000078F02188437030CE492031087007E03B
:109A7000CC4820300078F0218843CA492031087052
:109A800020202040002809D0C64820300078000956
:109A90000001C01DC3492031087007E0C1482030D3
:109AA000007800090001BF492031087040202040A3
:109AB000002807D0BB48807FF02188437030B94927
:109AC000887705E0B748807FF0218843B5498877DB
:109AD00064213046EEF734FB0A210190EEF730FBAB
:109AE0000D467D20C000864202D3AF48445D01E0B0
:109AF000AB48445DE007C00F002807D0A948007FAD
:109B000000090001C01DA749087705E0A548007FAE
:109B100000090001A349087702202040002807D04F
:109B2000A048C07EF021884370309E49C87605E089
:109B30009C48C07EF02188439A49C8760420204082
:109B4000002807D09748807EF021884370309549DF
:109B5000887605E09348807EF02188439149887695
:109B600008202040002807D08E48407FF0218843FD
:109B700070308C49487705E08A48407FF02188435F
:109B80008849487710202040002807D08548407F2A
